:020000040000FA
:040000006FD00400B9
:101000006F009044000000000000000090200020CD
:10101000A4220020A9BDF9F55C23002000000000F7
:10102000000000005C230020902000200000000051
:101030000000000090200020000000009020002010
:101040000000000090200020902000209020002030
:101050009020002090200020B82B0020902000201D
:10106000000000009020002090200020EC230020B1
:1010700090200020C22300209020002090200020FB
:101080009020002090200020902000209020002020
:101090009020002001A04111B7170040985F3AC688
:1010A000945F3247E39CE6FE3245410182800111A4
:1010B00013078008F337078093F787083EC20100C3
:1010C0000100B7170040930570052380B70413068D
:1010D00080FA2380C7040100010083C6B70493F699
:1010E000F60DA385D704238007049246F3A6068055
:1010F0000100010093760502D5CEF336078093F602
:10110000860836C4010001002380B7042380C70489
:1011100001000100B70614007D89558D88C70100C4
:1011200001000100010023800704A246F3A6068007
:101130000100010073370780137787083AC6010062
:1011400001002380B7042380C704010001000100CF
:1011500001003727004093061005A303D7802380A2
:101160000704B247F3A70780010001009307800836
:10117000F3B7078093F787083ECE01000100B71749
:101180000040130770052380E704130780FA2380CB
:10119000E7040100010003C7B70413670708A3852C
:1011A000E70423800704F247F3A70780010001004A
:1011B0000561828093760504BDC6F336078093F6F9
:1011C000860836C8010001002380B7042380C704C5
:1011D00001000100B7061400938606047D89558D31
:1011E00088C7010001000100010023800704C246F6
:1011F000F3A6068001000100733707801377870884
:101200003ACA010001002380B7042380C70401000B
:1012100001003727004093062005A303D7802380D1
:101220000704D24781B773370780137787083ACC12
:10123000010001002380B7042380C70401000100DE
:1012400098471367070C98C723800704E24719BF24
:101250000111814601468145114506CE6D24930753
:101260008008F3B7078093F787083EC601000100A6
:10127000B7170040130770052380E704130780FAAF
:101280002380E7040100010003C767041367170008
:101290002383E70423800704B247F3A707800100F4
:1012A0000100F2400561828041118146014681457D
:1012B0001145912C13078008F337078093F78708AF
:1012C0003EC401000100B7170040130670052380DB
:1012D000C704930680FA2380D70401000100FD555E
:1012E0002396B70223800704A245F3A505800100D9
:1012F000010073370780137787083AC601000100A1
:101300002380C7042380D7040100010003C76704BA
:10131000136717002383E70423800704B247F3A76A
:1013200007800100010001A0BD473305F50201005F
:101330007D1575FD8280411122C426C206C6AA848D
:10134000014463179400B2402244924441018280D8
:1013500005041305803E4204C13F4180DDB7000013
:101360009305000273A04580824573901534924026
:101370002242B2424243D2436244F2440255925561
:101380002256B2564257D2576258F25806499649E9
:10139000264AB64A464BD64B664CF64C065D965DE1
:1013A000265EB65E465FD65F09617300203041114C
:1013B000B7170040985F3AC6945F3247E39CE6FE59
:1013C000324541018280B71700401307000323888C
:1013D000E7028547171700002326F7F47300203033
:1013E000411122C406C6370400201C408297F5BF75
:1013F00037370040834747009146BD8B6389D7004C
:1014000099466394D700834757407300203097165E
:10141000000083C6F6F39387160017160000A30991
:10142000F6F203478700973700009387E75CB6978B
:101430002380E700B7E70400BC4F0946894517152C
:1014400000000345C5E98297C9B723030480154707
:101450002303E48001002302A48082808307648048
:10146000E3CE07FE23030480828083076480E3CEFB
:1014700007FE03454480828083076480E3CE07FE35
:101480002302A4808280411126C44AC24EC006C6EF
:101490001377F50BAD47AA892E8995446306F700AB
:1014A00019456537653F8D444E854537FD59FD1417
:1014B00063983401B240A2441249824941018280BA
:1014C000135509011375F50F453F2209CDB70111D9
:1014D00026CC06CEB704080051371545BD37713705
:1014E00069372AC6A53F32459377150089EB136506
:1014F00015001375F50FF240E24405618280FD147A
:10150000E9FC0145CDBF397126DC4ADA4ED852D606
:1015100056D45AD25ED006DE62CE66CCB7E700E083
:101520007D5783AA070022C603AA470023A0E71815
:1015300023A2E718B7170040130770052380E704BC
:10154000130780FA2380E70483C74704930B75FFD2
:10155000B684E20793FBFB0F8546AA892E8B32895E
:1015600037240040E187015763FA76016308D5000C
:101570008946130700026313D5000157D98F93F7EB
:10158000F70FB71C00402382FC0411472303E480BB
:101590001305F00F5D3D094CD135636D7C11B70526
:1015A0000700DA9537870700795563F2E504B387BA
:1015B0009500636EF702370B0800A94733EB65010E
:1015C0006399F90689E48144513D26850DA0DA85A9
:1015D0000945553D05090345F9FFFD14050B693D16
:1015E00081C49377FB0FFDF7DD3569FD7D55B71796
:1015F0000040130770052380E704130780FA238057
:10160000E70403C74704418B2382E704F250B7E79E
:1016100000E023A0571123A24711E254324452594B
:10162000C259325AA25A125B825B724CE24C21615F
:101630008280A5476395F90685691309F00FB30603
:101640009900B3742B01B6941349F9FFB374990050
:10165000856B33796901416B9387F9FFB3F72701F4
:1016600099E363FC340193D94900C147E3E637FFAE
:1016700099BF0569C1697D19D9B71305800D6388C4
:101680006901130500026384790113051008CA85F6
:10169000DD3B353D21DD4E99B3843441D9B7DA8540
:1016A0002D45D533CA94E30099F205097D3BA30F7C
:1016B000A9FED5BF9387F9FF93F7F70F6361FC0C81
:1016C00083C71C0413073008631FF704370708009B
:1016D000636BEB04B3079B00B706100063F5D704F8
:1016E000334BEB0089476393F9068980D549E38C36
:1016F00004ECDA850945413B11090327C9FF9147ED
:101700002320E48003076480E34E07FE2303348133
:10171000FD17EDFBFD14110B81C49377FB0FE9FF5F
:101720007D3371F5E1B5B717004003C75704B7071C
:1017300008001377070219E3B78707007955E378A4
:10174000FBEA33079B00E3FFE7F855B58547E382E3
:10175000F9F2DA852D45053B9389F4FFE38504E62C
:10176000293393F7390091EB83260480032709007E
:1017700093074900E39AE6E43E89CE84F1BFB5477A
:101780006396F9001305900BC93135BDB1471305B8
:10179000B00AE38BF9FE99476391F904B705080095
:1017A000B365BB002D45C53181448D4BA1497539C9
:1017B00063967401832704802320F9008504E3984D
:1017C00034FF8327048013172B016355070023126E
:1017D000F900D5BB2322F900FDB39D476399F902B7
:1017E00081451305B0044531BD442320090023225F
:1017F0000900FD599D3993F77400CA9703C7070084
:10180000FD14398D2380A700E39634FF6DBBA147FB
:101810006392F9046D398144630D0B008D47930485
:10182000C0036308FB009304000563048B01930469
:1018300040041375C507E30895D81945393139397E
:101840000545213126850D3909453D314931E31CD6
:1018500005D669BB91476399F90013056006F53613
:10186000F53E130590090DB7E38F09D4F154A9BBD8
:10187000BD660147173600001306C644938606A6C8
:1018800085458347060093F7F70F91C382800507CC
:10189000E3F9E6FE973700002386B742DDB77D16F1
:1018A0006206618693178601E18763D407000145CC
:1018B0008280931726003307F500AE9718439C43A8
:1018C00063E7E7007D16E37FF7FC7D5582800545E1
:1018D0008280FD15E205E18513978501618793F705
:1018E000F50F63480700FD15139725002A97584305
:1018F00065D7138517006205618582803308B502BC
:101900001C4283A80600B335B502C29733B5070160
:10191000AE98469585486367B5006394A50063E378
:10192000070181480C43C6950CC388C21CC2828043
:1019300081471397870161876343B70082801397BC
:1019400027002A97232007008507E5B7814701472D
:1019500093968701E18663C5B60013351700828030
:1019600093962700AA9694428507558FD5B793D7AB
:1019700055408A07AA979C4305453315B5007D8DD0
:10198000828017F3FFDFE702C33B2A84993705C53E
:10199000931725003E940327C4FF814711EB7D1563
:1019A00016053E954205418517F3FFDF6700A33B0F
:1019B00005838507E5B70145C5BF814713978701B3
:1019C00061876343C700828013972700B386E500D1
:1019D00094422A97850714C3D5B77D16620661869F
:1019E000014793178601E18763D507001335170078
:1019F000828093172600B306F500AE9794429C436D
:101A00007D16B58F5D8FF1BF8A05AA950147636387
:101A1000B500828083A6C5FFF11593D71600D98F34
:101A20009CC11397F601E5B72A8301480147014598
:101A30006343D7008280B387050183A80700B307FB
:101A400006019C43C697AA976384F80033B5170133
:101A50000507B3080301620723A0F8006187110896
:101A6000C1BF2A8301478147014563C3D7008280F4
:101A70003388E50083280800330EE600032E0E00AD
:101A80003388A8403308C8416384080133B508018E
:101A90008507B308E300E20723A00801E1871107E7
:101AA000E9B717F3FFDFE702C3290111B286B28459
:101AB0002E86AA850A8575372A84A6850A857935F2
:101AC00033348000060413351500018D056117F3CA
:101AD000FFDF6700432917F3FFDFE702032441110B
:101AE000AA89AE8A328BB68402C202C402C60144FD
:101AF000131C8401135C8C4163499C02939B14006A
:101B0000FD1B0549138CF4FFF15C33048901620469
:101B10006184634D740592478E04CE9423AEF4FE27
:101B2000410117F3FFDF6700C32213192400B30B31
:101B30002B01014A93172A00D69783A50B008843EF
:101B40007800340050005D3B050A93178A01E18755
:101B5000F11BE351FCFE92474E9905042320F90046
:101B6000A2473EC2B24702C63EC459B7131A890102
:101B7000135A8A41131D240093178A01E18763CF0A
:101B8000970092470A044E941CC0A2470509137996
:101B9000F90F3EC2B24702C63EC485BFB3079A03DF
:101BA00013152A0056950841780034005000050AA4
:101BB000EA97DA978C439933C1B70000197106C2CE
:101BC00012C416C61AC81ECA22CC26CE2AD02ED2BD
:101BD00032D436D63AD83EDA42DC46DECAC0CEC26D
:101BE000D2C4D6C6DAC8DECAE2CCE6CEEAD0EED29D
:101BF000F2D4F6D6FAD8FEDA97050000938505727E
:101C00008841E700050092402242B2424243D2435B
:101C10006244F244025592552256B2564257D25768
:101C20006258F25806499649264AB64A464BD64B60
:101C3000664CF64C065D965D265EB65E465FD65FE8
:101C40000961730020300000972100209381813BBF
:101C500017510020130101BB17F5FFFF1305C53A0B
:101C6000970500209385053A171600201306C6FD38
:101C700063FAC5008322050023A0550011059105D4
:101C8000E3EAC5FE17A501001305C54E9715002010
:101C90009385C5FB171600201306C66563FAC500B9
:101CA0008322050023A0550011059105E3EAC5FE36
:101CB0001715002013050564974500209385854C72
:101CC0006377B500232005001105E36DB5FEFD42E5
:101CD000739002BC8D4273904280B72200009382C1
:101CE000828873900230970200209382A23193E29F
:101CF00032007390523097420000938202F073904A
:101D000012346FC0E42F73002030397101436EC666
:101D100019A0397141536AC866CA62CC5ECE19A057
:101D2000397101535AD056D252D44ED64AD826DAF7
:101D300022DC06DE33016140828241114AC026C2A4
:101D400022C406C68282B24D4101024D924C224C01
:101D5000B24B4101024B924A224AB2494101024927
:101D600092442244B240410182803D432A876373FA
:101D7000C3029377F700BDEFADE5937606FF3D8A8A
:101D8000BA960CC34CC30CC74CC74107E36BD7FED4
:101D900011E28280B306C3408A069702000096963D
:101DA0006780A6002307B700A306B7002306B70085
:101DB000A305B7002305B700A304B7002304B700A9
:101DC000A303B7002303B700A302B7002302B700A1
:101DD000A301B7002301B700A300B7002300B70099
:101DE000828093F5F50F93968500D58D9396050126
:101DF000D58D61B79396270097020000969686824C
:101E0000E78086FA9680C1171D8F3E96E374C3F86B
:101E1000A5B73367B500FD530D8B79E7B7877F7F93
:101E20009387F7F710419441B372F6003363F600DD
:101E3000BE92B3E262006397720C6318D6065041FB
:101E4000D441B372F6003363F600BE92B3E262008F
:101E50006398720A631BD60410459445B372F6006A
:101E60003363F600BE92B3E262006391720A631EAE
:101E7000D6025045D445B372F6003363F600BE92E5
:101E8000B3E26200639A72086311D6021049944962
:101E9000B372F6003363F600BE92B3E2620063935E
:101EA00072085105D105E30FD6F613170601939773
:101EB0000601631CF7001357060193D7060133058B
:101EC000F7409375F50F91E982804183C183330513
:101ED000F7409375F50F91E182801377F70F93F731
:101EE000F70F3305F74082800346050083C60500DF
:101EF000050585056313D60065FA3305D640828053
:101F000011059105E312D6FE014582802105A10548
:101F1000E31CD6FC014582803105B105E316D6FCF1
:101F2000014582804105C105E310D6FC0145828050
:101F3000B717004003C777051377E70FA38BE704B4
:101F4000130700F8A38DE7043D47238CE70413072C
:101F50005003A38CE70403C7A7051377D70F238D7E
:101F6000E7048280B717004003C7E7020D894111DB
:101F70001377C70F498F93068008F3B6068093F650
:101F8000860836C601000100930670052380D70439
:101F9000930680FA2380D704010001002387E7021B
:101FA00023800704B247F3A7078001000100410125
:101FB000828041112A83014E930E407E130F001937
:101FC000930F400663E56E12930800191303400651
:101FD000B3781503854E0D4FA14F337365020D89FC
:101FE0001335150063EFBE121308F6FF7946729899
:101FF0004208135808013307C70213D61700BE075B
:1020000032976146B3F6C60213068070B386C602E5
:102010003697A166F58F42075D8FB716004083C7DC
:10202000F60293F70708A303F1000346710083C784
:10203000F60293F70708E394C7FE83477100B716CB
:10204000004093F7F70F6388071293078008F3B7F0
:10205000078093F787083EC401000100B7170040CE
:10206000930670052380D704930680FA2380D70453
:102070000100010023AA070383C6170393E606089D
:10208000A388D70223800704A247F3A70780010093
:1020900001001166B71700407D16D45BC85F9385B9
:1020A0004703A98EF18EF5FA93068008F3B60680F1
:1020B00093F6860836C6010001009306700523805A
:1020C000D704930680FA2380D7040100010098C149
:1020D00003C7170313670704A388E70223800704D5
:1020E000B247F3A7078001000100410182807D1300
:1020F0003368E3039308E016630E08003368F303C4
:102100009308D016630808009378330093B818003A
:102110009388D81633081E01131E0801135E0E01A2
:1021200055B56393E50305486386080001486303DA
:1021300003002A8871087298FD15131E0801C20554
:10214000135E0E01C18179BD13F8150063F4BF0061
:102150007908D5B713381800E5BF83C7F60293F79F
:102160000708A303F1000346710083C7F60293F743
:102170000708E394C7FE8347710093F7F70FF1DF79
:10218000E9B531714AD966CB06DF22DD26DB4ED7B1
:1021900052D556D35AD15ECF62CD6AC96EC7AA8CCA
:1021A00002D8EF00901C2A8993078008F3B70780B4
:1021B00093F787083EDA01000100B71700401307C4
:1021C00070052380E704130780FA2380E7040100E9
:1021D000010003C7F7021377770FA387E70203C74E
:1021E000F70213678700A387E70223800704D2570B
:1021F000F3A70780010001000545AD33130780C137
:102200003347E902116A93070AE893065002BD6951
:10221000930BA004814A014B1304800893047005BA
:102220007D1AB347F9023307D7023EC0FD873ECC83
:10223000938709A69309803E3347F7023AC27D8708
:102240003AC4334739038549B399990193D9394041
:10225000B306D702B30B7703B3C6F602B3CBFB02C8
:1022600036C6FD8636C893D6FB4136CEB7460F003C
:10227000938606243349D9028566938606FAB39677
:102280009601B389E902130760553309D902930611
:102290000010B389E9023349D902B3C9F902931690
:1022A000390036CA37190040FD8636D0930D09042F
:1022B00093D7F9413ED2F336048093F6860836DC94
:1022C00001000100930770052380FD00930680FA4A
:1022D0002380DD00010001008346390593F6860F57
:1022E000A309D9048346390593E61600A309D90446
:1022F00023800D00E256F3A6068001000100130CB6
:1023000080FA116DF336048093F6860836DE0100FC
:102310000100930770052380FD0023808D010100DB
:10232000010083463905216693E60602A309D90414
:1023300083560905B3E6A6012318D9048356090577
:10234000D18E2318D90423800D00F256F3A60680FF
:10235000010001008346390593F60602638A0618D8
:1023600003463905218A6DDE0818EF001004733624
:10237000048013768608B2C20100010023809D000C
:1023800023808D0101000100B717004003C6370507
:102390001376F60DA389C70403C637051366060234
:1023A000A389C704835609052166B3E6A60123184D
:1023B000D90483560905D18E2318D90423800D0032
:1023C0009646F3A60680010001008346390593F680
:1023D00006026386061483463905A18AEDFE97003E
:1023E0000020E78040CBAA8636D497000020E78003
:1023F00080CAA256E30AD5FE835609054255B3E6C4
:10240000A6012318D904C12783463905A18AEDDE28
:10241000035609058346290582473376CA00B30669
:10242000DA0293D5F641B296B388F640E24733B864
:10243000C6002E983308F840A247B3B616013308F9
:10244000D84063C70701631DF800924763FA17017C
:10245000C247634DF80E63950701B24763E8F80E73
:10246000894663E7660FF2469315180013D3F80107
:102470005E8613951800B365B30042D646D4EF606C
:1024800081353258050B137BFB0F63470001631244
:102490000838A258638F083613081500B336A80011
:1024A000B69513D6F5013298B336C800AE961358D8
:1024B0001800FE06B3E6060173360480137686081C
:1024C000B2C60100010023809D0023808D01010020
:1024D00001000356C902B296C206C1822316D90270
:1024E00023800D00B646F3A606800100010019BD49
:1024F000F336048093F68608B6C0010001002380FD
:102500009D0023808D01010001008346390593E67B
:102510000602A309D90423800D00864605BDF336C3
:10252000048093F68608B6C40100010023809D0054
:1025300023808D01010001008346390593E60602E0
:10254000A309D90423800D00A646A5BDE30D0BF019
:10255000F336048093F68608B6C80100010093069E
:1025600080FA23809D002380DD0001000100834666
:10257000390593F5FC0F93F6860FA309D90483461A
:102580003905CD8EA309D90423800D00C646F3A6D4
:10259000068001000100130580FA03463905930601
:1025A00039051D8A631496297336048013768608CC
:1025B000B2CC01000100130680FA23809D00238025
:1025C000CD000100010003C606001376F60D23803E
:1025D000C60003C60600136606022380C6008356A3
:1025E00009051166D18E2318D90483560905216681
:1025F000D18E2318D90423800D00E646F3A6068069
:1026000001000100130680FA8346390593F606029D
:102610006388062483463905130C3905A18AFDDA3F
:1026200008186123F336048093F68608B6D00100BB
:102630000100930680FA23809D002380DD000100C5
:10264000010083460C00116693F6F60D2300DC00B2
:1026500083460C0093E606022300DC00835609053E
:10266000D18E2318D904835609052166D18E2318EB
:10267000D90423800D008656F3A6068001000100D0
:10268000130680FA8346390593F606026385062011
:1026900083463905A18AEDFE97000020E780A09FC0
:1026A0002A8C97000020E780009FE30C85FF83566B
:1026B000090511664255D18E2318D9042923834672
:1026C000390513063905A18AFDDAF336048093F63D
:1026D0008608B6D401000100930680FA23809D008D
:1026E0002380DD00010001008346060093F6F60D0D
:1026F0002300D60023800D00A656F3A60680010015
:1027000001008356090503462905D247B376DA004E
:102710003306CA021305800C9355F6413696330DE5
:10272000F6408257333CD6002E9C3336A601330C3C
:10273000FC40330CCC403308850392564E86B335AB
:10274000A5033305A503C295EF60E1086346800148
:10275000631E0C16630C0D16130615003335A60008
:102760002E959356F5013696B335D600AA959396D5
:10277000F50105828585D18E6346B000639D051AFB
:10278000638B061A0356C90215823305D600333609
:10279000C500B2956348B000639105241306F00F9D
:1027A000637DA622894663F3561593078008F3B725
:1027B000078093F78708BED6010001003717004055
:1027C000930770052300F704930780FA2300F704AA
:1027D000010001008356C70289678117D58FC207A0
:1027E000C1832316F70223000704B657F3A7078017
:1027F00001000100FA506A54DA544A59BA592A5A67
:102800009A5A0A5BFA4B6A4CDA4C4A4DBA4D296126
:1028100082801308F5FF3335A800FD152E95135659
:10282000F5013298B336C800AA9651B1F336048048
:1028300093F68608B6CA0100010023809D0023801C
:10284000AD000100010083463905CD8EA309D904EE
:1028500023800D00D646F3A606800100010035BB9B
:10286000F336048093F68608B6CE0100010023807B
:102870009D002380CD00010001008346390593E6C9
:102880000602A309D90423800D00F646F3A60680AC
:102890000100010095BBF336048093F68608B6D29A
:1028A0000100010023809D002380CD000100010074
:1028B0008346390593E60602A309D90423800D0057
:1028C0009656F3A60680010001006DBB9306F5FF46
:1028D00033B5A600FD152E959355F501AE96B3B50B
:1028E000B600AA951396F501858269B5F336048082
:1028F00093F68608B6D801000100930680FA23807B
:102900009D002380DD00010001008356C902056699
:10291000011693F6F60FD18EC206C1822316D90294
:1029200023800D00C656F3A6068001000100850A2B
:1029300093FAFA0F49B233E6B60045C20356C9020C
:102940003305D0403338A000B305B040B38505410E
:1029500015826345B000D1E16371A608894663F032
:10296000560593078008F3B7078093F78708BEDA08
:1029700001000100B7170040130770052380E7042A
:10298000130780FA2380E7040100010003D7C70280
:102990007D8B2396E70223800704D65781BDF3364B
:1029A000048093F68608B6DC01000100930680FAE5
:1029B00023809D002380DD00010001008356C902B1
:1029C0000566011693F6F60FD18EC206C182231654
:1029D000D90223800D00E656B9B793078008F3B7F4
:1029E000078093F78708BEDE01000100371700401B
:1029F000930770052300F704930780FA2300F70478
:102A0000010001000356C70293975600B297C20710
:102A1000C1832316F70223000704F657C1BB914771
:102A200063EEB70217870100130787AB8A05BA95D3
:102A30009C41BA978287B717004003A7470B1345FD
:102A4000F5FF698F23AAE70A03A7070B698F23A85D
:102A5000E70A03A7070A798D23A0A70A8280B71780
:102A6000004083A6470B1347F5FFF98E23AAD70A28
:102A700083A6070B558D23A8A70A83A6070A758F7F
:102A800023A0E70A8280B717004003A7470B498FAE
:102A900023AAE70A03A7070B1345F5FF45BFB7179E
:102AA000004083A6470B1347F5FF758F23AAE70A5B
:102AB00003A7070A598D4DB7B717004003A7470B67
:102AC000498FEDB7914763EEB702178701001307EF
:102AD00067A28A05BA959C41BA978287B7170040CA
:102AE00003A7470D1345F5FF698F23AAE70C03A73A
:102AF000070D698F23A8E70C03A7070C798D23A086
:102B0000A70C8280B717004083A6470D1347F5FF37
:102B1000F98E23AAD70C83A6070D558D23A8A70CE1
:102B200083A6070C758F23A0E70C8280B71700409F
:102B300003A7470D498F23AAE70C03A7070D1345E9
:102B4000F5FF45BFB717004083A6470D1347F5FFB4
:102B5000758F23AAE70C03A7070C598D4DB7B7173C
:102B6000004003A7470D498FEDB7B71700408847CE
:102B7000420541819377050491EB9377F501375531
:102B8000E801130505803345F50282809377050C33
:102B9000130700046397E7009377F50137459C1C02
:102BA000CDB72165130505D0828037E700E01C43CF
:102BB0005443A183E206D58F1CC1FD572320F7188B
:102BC0002322F718828013178500B7E700E023A0BF
:102BD000E710618123A2A7108280B7F700E0884741
:102BE000CC478280814737370040A14663C4C70085
:102BF000328582800345B740E38EA6FE3385F5001B
:102C00000345050085072304A740CDB7970700209B
:102C10009387476A9C43173700201307A7563E95B2
:102C2000636EE500174700201307C79D6368A70080
:102C3000170700202320A7683E858280FD57EDBF3F
:102C4000411122C406C62A840D372947B307E5027D
:102C5000B2408D83B3D7870222449507B3D7E702EA
:102C600037370040C207C1832316F7004101828035
:102C7000716541111305052006C6D937B7370040E5
:102C8000130770F82381E7000D47A381E7001307BE
:102C90000004A380E70005472387E700B240410115
:102CA000828037370040834727001A0593F7F703E0
:102CB000C98F93F7F70F2301F7008280B7370040E1
:102CC00003C7170019C9D98DA380B70003C7070030
:102CD000136787002380E700828093C5F5FFF98D95
:102CE000A380B7008280B73700402147B736004045
:102CF00091E1828003C6B700E30CC7FE05050346D9
:102D0000F5FFFD15C2052384C600C181D5B7411169
:102D100022C406C62A84913D2947B307E502B24082
:102D20008D83B3D7870222449507B3D7E70237379D
:102D30000040C207C1832316F740410182807165BC
:102D400041111305052006C6D937B73700401307D0
:102D500070F82381E7400D47A381E7401307000483
:102D6000A380E74005472387E740B24041018280C6
:102D7000CC41411106C6328503C6150083C5050046
:102D800022064D8E42068D654186138875A2630C1E
:102D90000611634BC804138845A26300060D634AFD
:102DA000C800938535A26301B60823900600294622
:102DB0004DA0138855A26305060D938565A2E31601
:102DC000B6FE8D451D4663E6E5081146198E63F390
:102DD000C7003E86B7E704002390C600FC479795DE
:102DE0000100938525339DA0138895A263030611E6
:102DF000634E060D1388A5A263000613938505A5EF
:102E0000E315B6FA99451D4663E5E504198E63F3AB
:102E1000C7003E86B7E704002390C600FC4797052D
:102E200000209385A5491DA09D451D4663E3E5024D
:102E30002146198E63F3C7003E86B7E70400FC47BE
:102E40002390C600970500209385C54ABA958297BE
:102E50000146B240328541018280AD451D46E3EA1C
:102E6000E5FE3146198E63F3C7003E86B7E70400DE
:102E70002390C600FC47977501009385A56AF9B7B2
:102E8000B1451D46E3E7E5FC3546198E63F3C700FF
:102E90003E86B7E704002390C600FC479775010003
:102EA0009385456965B78D451D46E3E4E5FA11460E
:102EB000198E63F3C7003E86B7E704002390C6006F
:102EC000FC47979501009385A52549B78D451D467B
:102ED000E3E1E5F81146198E63F3C7003E86B7E7D4
:102EE00004002390C600FC479795010093850525B3
:102EF000B1BFA5451D46E3EEE5F42946198E63F3FF
:102F0000C7003E86B7E704002390C600FC479775CC
:102F10000100938565601DBFB5451D46E3EBE5F2F5
:102F20003946198E63F3C7003E86B7E70400239045
:102F3000C600FC47977501009385055D01BFB7E7A3
:102F4000040003A3071397060020938626D9414661
:102F5000A54517050020130565CF02832D4559EFC0
:102F600003C5050009476317E50803A8450041119B
:102F700006C6034718003285034608002207416849
:102F8000518F930828FE6308170363E9E8000518CA
:102F9000630307052390060029451DA8130648FE74
:102FA000630BC7021518E31707FF15463E87637BBF
:102FB000F602154705A83E8691C30546B7E704000B
:102FC000FC472390C6004206CC45418282970145CA
:102FD000B240410182801306700F3E876374F60091
:102FE0001307700FB7E704002390E600FC471316A1
:102FF0000701D9BF23900600054582808280416782
:1030000079176304E504411122C406C685472A8462
:10301000639FF500B7E7040022852244B24003A372
:103020008713970500209385A52D410102838947C9
:103030006399F500B7E7040083A7070B85458297DE
:1030400071D9B2402244410182808280797122D4B8
:1030500052CC2E842A8A977501009385E54F177507
:1030600001001305255106D63AC626D24AD0B684A9
:1030700032894ECEEF507141A685177501001305B8
:103080006550EF5091402945EF50714483478400CB
:1030900093F70702E1E78349040089470545324772
:1030A0006396F908544083C7160083C60600A2073A
:1030B000D58FC166138616FE638CC7028D16638F8B
:1030C000D7068D669386269029456391D706B7E784
:1030D0000400A285225403A34714B250F249A686E5
:1030E0004A86925402595285624A85474561028355
:1030F0002D450DEF9307700F354563E99702B7E74C
:103100000400FC4748441306700FCA858297814922
:10311000970700209387871F9C43014581CB9C43E1
:1031200091C74E852686CA8582970145B2502254A2
:1031300092540259F249624A456182802D457DF7D9
:103140009307700F3545E3E397FEB7E70400FC47AC
:1031500048441306700FCA8582975DBF2145F9B7B1
:10316000411122C437E404008327841326C2AA84B1
:10317000416506C697050020938585187D158297C1
:103180008327C40A170500001305A5E785888297E1
:1031900095C0032304132244B240924497060020B2
:1031A000938686C54146C545170500201305C5B35E
:1031B00041010283B2402244924401454101828090
:1031C00019C59707002023A3A71401458280454510
:1031D00082801147636AA70A977601009386863634
:1031E0000A0536951841411106C63697AE87B28555
:1031F00002871307700F6145639DE700B7E704007E
:10320000FC471306700F170500201305E51682977B
:103210000145B2404101828005476145E39BE7FEDD
:10322000B7E70400FC470546170500201305050D08
:10323000F9BF1307700F6145E39DE7FCB7E7040092
:10324000FC471306700F1705002013056522C1B750
:103250001307700F6145E39EE7FAB7E70400FC47E8
:103260001306700F17050020130505304DB71547DD
:103270006145E390E7FAB7E70400FC4715461705F8
:1032800000201305250861B709458280411126C237
:10329000B7E4040083A7C41322C44AC006C62E8420
:1032A000970500209385C5052A898297058905C55C
:1032B00097070020938747A383D7A70BA28503A373
:1032C000440D2310F4002244B24092444A8502493E
:1032D000014641010283B2402244924402494945D9
:1032E000410182809707002023840702970700206E
:1032F00023A20702B717004003A7070CB706C0FFB9
:10330000FD16758F23A0E70C03A7070DB706400035
:10331000558F23A8E70C03A7070C3D9B23A0E70CC0
:1033200003A7070D1367070123A8E70C8280B717CF
:10333000004003A5470C83A7470C5981134515008E
:10334000C18B058999E3136525009707002083C782
:1033500027FC6380A70297070020238BA7FA11C9D7
:1033600097070020938707FB03A30700630303006D
:103370000283828011456FE0DFE0411193962500C2
:10338000AA852D4506C697F0FF1FE780C017B240FB
:10339000014541018280011122CC06CE3714004044
:1033A00026CA4AC84EC652C483447405034AB405AB
:1033B0008349840503499405EFE09FB78347A4053B
:1033C00093F4F40F137AFA0F93E71700230DF40424
:1033D00093F9F90F1379F90FB717004003C7A70541
:1033E000058B6DFF03D5C705A38D4705238C3705D6
:1033F000A38C2705A38B9704F2406244D244424930
:10340000B249224A0561828041119397050122C485
:1034100006C626C2C1872E8463DC0700B7E4040019
:10342000FC54829719C1BC5482972165218D3DA01F
:1034300093F7150013C5150095E393F7250085C78D
:10344000FD35B7E70400BC4F1306000A8945170590
:1034500000200345A5EC829713452400B240224486
:103460009244410182809397250163D50702B7E416
:10347000040083A7C41E8297F53DBC4C37F60200BA
:10348000130606E0896517050020034525E98297A4
:10349000096569BF939715010145E3D107FC1775CD
:1034A00001001305E514EF501113B7E70400BC4FFA
:1034B00013060064916517050020034525E68297F1
:1034C0001165ADB72D71232A9110FD74E98C232C61
:1034D000811023282111232631112A84AE893289B3
:1034E000930600100A86A6852D45232E111097F00D
:1034F000FF1FE780400113154401B7E70400FC47B4
:1035000051810A0513962900CA850A958297A685D6
:1035100085660146254597F0FF1FE780C0FE0A86B5
:10352000A68593060010294597F0FF1FE780A0FDB0
:103530008320C11103248111832441110329011126
:103540008329C11015618280B7F7070003C70701FF
:10355000411106C622C426C24AC0A547631AF70015
:103560009537B2402244924402490145410182808C
:1035700013942500AA843289A286AA85014625458E
:1035800097F0FF1FE78020F8A2864A86A685294586
:1035900097F0FF1FE78020F7E9B71D71A2CC37E451
:1035A00004005C5C485886CE4946977501009385B7
:1035B000A5FF829701E91775010013052500EF505B
:1035C000910101A0B7F600E0795798CAFD57DCCA0F
:1035D0000567B7E700E023A0E7101306F00290C2EA
:1035E00023A0E71801000100370700201847130641
:1035F000000481459706002023A0E6D24157A38A04
:10360000E7403C440808829797170020938787DE9D
:103610003EC8856713870760231AE1001D673ACC0F
:1036200037070105130707103ACE9387B7D313075F
:10363000B00F2310E1022312F102054797F7FFFFB5
:103640009387E7592301E1023ED8170700001307CB
:1036500007D397070000938747D4B7F50700BAC28E
:103660003EDC17070000130767EE970700009387FB
:10367000A7D081463000E1051945BAC43EDE97F077
:10368000FF1FE78040E818088147994630003E96C2
:103690000346060085070507A30BC700E398D7FE7E
:1036A000C24791C70357410185676373F70001A0C3
:1036B000B7E7040083A7470A08088297AA8501C9CB
:1036C000177501001305C5F0EF50215C01A0F6400D
:1036D000664425618280411126C2B7E4040083A7B5
:1036E000040806C622C417050000130525D28297D8
:1036F00017040020130484C22300A4003128DD36FF
:1037000003450400224403A38405B24092441306F7
:103710000032896541010283797106D622D41307EC
:103720008008F337078093F787083EC20100010045
:10373000B7170040930570052380B704130680FA7D
:103740002380C7040100010083C6F70293F6A60F89
:10375000A387D702238007049246F3A606800100C0
:10376000010073370780137787083AC4010001000E
:103770002380B7042380C7040100010003C7F702B8
:1037800013672700A387E70223800704A247F3A754
:103790000780010001000545EFE0CFFCE13E014755
:1037A00081468147054685451305407EEFE07F80D1
:1037B00037E404003C446800514681458297B707CE
:1037C000C0A83EC8B787E803938707D03ECA97F7DB
:1037D000FF1F9387C7BD3EC67C5868008297B250D2
:1037E00022544561828041119775010093850550EF
:1037F00017750100130505D806C6EF500149177566
:10380000010013052569EF504148B24029454101A7
:103810006F50E14B4111977501009385654E177507
:103820000100130525D506C6EF5021461775010086
:1038300013050565EF506145B240294541016F50C0
:103840000149411122C406C6834705002A849DC34D
:10385000977501009385855017750100130585D173
:10386000EF50A1424C40177501001305E576EF506B
:10387000C1411DA058411DE7977501009385054E74
:1038800017750100130505CFEF5021401775010092
:1038900013050576EF50613F2244B24029454101AE
:1038A0006F50E142A1679386D7036311D7029775E2
:1038B00001009385A54A177501001305A5CBEF50AC
:1038C000C13C177501001305A573E9B7ED0797759E
:1038D00001009385A548177501001305A5C9631953
:1038E000F700EF50813A177501001305A5725DB717
:1038F000EF50A1394C40177501001305A57385BF22
:103900004111977501009385E54017750100130576
:1039100065C606C6EF506137B240294541016F5078
:10392000013B797122D426D24AD02E842A8981453E
:10393000B2844800714606D6EFE02FC397F7FF1F09
:103940009387076BDC4783D70700231421012313D8
:10395000F100EF2090019547A305F1009307401F68
:103960003EC6FD572305A100230AF100EF203012C7
:103970002686A2854800EF203002B250225492548D
:10398000025945618280970700202392079C970780
:103990000020238D079AB7E70400BC47411106C6F3
:1039A000414681451385413D8297EF101067EF1026
:1039B00090440145EF30201403C7C1259307F00A56
:1039C000631BF7009307F00889451385C125239EE3
:1039D000F124EF30A03EEF30804E814537050400E2
:1039E0009707002023A0079697070020239A0794A3
:1039F000970700202387079497070020239F0792AB
:103A000097070020239A079297070020239907928F
:103A100097070020239A0792EF20A0360145EF3048
:103A2000A040977501009385653117750100130556
:103A300065B4EF508125177501001305E565EF505A
:103A4000C124B240294541016F506128411122C46F
:103A500006C626C293F715002E84638D070C814697
:103A600017F6FF1F13064656854517050020035518
:103A7000658CEF80500905C5977501009385C52CAD
:103A800017750100130505AFEF50212017750100D0
:103A9000130545CEEF50611F2945EF50412397751F
:103AA00001009385652A177501001305A5ACEF5039
:103AB000C11D17750100130525CDEF50011D2945C6
:103AC000EF50E12017F5FF1F130585525C450547B0
:103AD0002390E700EFF08019977501009385C526C4
:103AE00017750100130505A9EF50211A177501007C
:103AF0001305C5CAEF5061192945EF50411D9307C1
:103B000010F8238EF1249707002083D76782A38EB5
:103B1000F1241385C125A1839145238FF124A38F1F
:103B20000124EF30A02913451400B24022449244EE
:103B30004101828093F72500D1CB1707002003575E
:103B4000278051C397F6FF1F9386C67F94429777CD
:103B500001009387675617F6FF1F0346867E81454F
:103B60001385413DEF407007AA8431CD9775010060
:103B700093854524177501001305C59FEF50E1108B
:103B8000A685177501001305E5C2EF500110294500
:103B9000EF50E11397F7FF1F2394077A930710F86C
:103BA000238EF12497F7FF1F83D78778A38EF12404
:103BB000A183238FF12491458D471385C125A38FC0
:103BC000F124EF30A01F1345240085B793F745007B
:103BD000B1CF977501009385E51D17750100130599
:103BE0006599EF50810A17750100130565BEEF5006
:103BF000C1092945EF50A10D930720F8238EF12428
:103C000097F7FF1F83D76773A38EF124A183238FB8
:103C1000F1248547A38FF124EF2060671385C12528
:103C20009145EF30A0191345440001B793F7850083
:103C30008DCF977501009385E51717750100130562
:103C40006593EF508104177501001305A5B9EF5076
:103C5000C1032945EF50A10797F7FF1F2392076E75
:103C6000EF40900413458400C9B593F70501A5C33F
:103C7000854517F5FF1F0355456CEF00514E9775AD
:103C8000010093852513177501001305A58EEF40DC
:103C9000D17F17750100130525B6EF40117F294527
:103CA000EF50E102930730F8238EF12497F7FF1FBE
:103CB00083D7A768A38EF1241385C125A1838D45E1
:103CC000238FF124EF30800F13450401B9BD93F722
:103CD0000502B5C3977501009385C50D17750100E1
:103CE00013054589EF40717A17750100130505B377
:103CF000EF40B1792945EF40917D930740F8238E3D
:103D0000F12497F7FF1F83D72763A38EF124A183A4
:103D1000238FF1248547A38FF12497F7FF1F239D5D
:103D20000760EF20C0561385C1259145EF3000098B
:103D300013450402DDBB93F70504CDC79775010059
:103D400093854507177501001305C582EF40F17390
:103D500017750100130505AEEF4031732945EF409B
:103D6000117783C7C1251307700A6388E704130717
:103D7000800A6386E7061307600A6397E7029307E2
:103D800060F8238EF12497F7FF1F83D7475BA38E3C
:103D9000F124A183238FF1248547A383F126B14524
:103DA0001385C125EF308001EF20604E13450404D8
:103DB00097F7FF1F239507588DBB930770F8238E45
:103DC000F12497F7FF1F83D78757A38EF124A18390
:103DD000238FF1248547A380F1269945D1B7930716
:103DE00080F8F1BF93F705080145E38007D4977584
:103DF0000100938525FC176501001305A577EF40A9
:103E0000D16817750100130565A4EF4011682945B5
:103E1000EF40F16B9307A0F8238EF12497F7FF1F73
:103E200083D78752A38EF124A183238FF124854762
:103E3000A38FF12497F7FF1F23980750EF20204509
:103E40001385C1259145EF20707713450408F1B91A
:103E5000411122C497750100938585F12A84176565
:103E600001001305257106C6EF4031624C401775FD
:103E700001001305E513EF4051612945EF4031651D
:103E8000034704009307F00F6319F70297750100C9
:103E9000938505EE176501001305C56DEF40F15ED2
:103EA0004C40177501001305A511EF40115E224427
:103EB000B240294541016F409161B2402244410125
:103EC000828085CD411122C4176501001305856AE2
:103ED0002E84977501009385A5E406C6EF40F15A3C
:103EE000A285177501001305E518EF40115A224409
:103EF000B240294541016F40915D8280411122C449
:103F000026C22E84AA8497750100938525E2176541
:103F100001001305256606C6EF40315717750100ED
:103F200013050516EF4071562945EF40515A977514
:103F300001009385A5DF97F7FF1F239D973E176527
:103F4000010013052563854497F7FF1F2392873EE1
:103F500097F7FF1F239F973C97F7FF1F2399873EF3
:103F6000EF40B15297F5FF1F83D5653E17750100ED
:103F700013058511EF4071512945EF40515597F7D1
:103F8000FF1F2385973CEF1000672285EF20B03696
:103F90000545EF20706997F7FF1F93876705DC479A
:103FA00003D70700C167FD176312F7022244B7E782
:103FB0000400B240924403A3870517F5FF1F034591
:103FC00065361306000A854541010283B24022444A
:103FD000924441018280011122CC37E404005C5CF0
:103FE00006CE26CA3546977501009385E5EB177511
:103FF000010013052578829701E917650100130573
:10400000E55BEF40515D01A097F7FF1F9387476580
:104010003EC4B7F507008567938707C0814617F64A
:10402000FF1F13066630E10519453EC697E0FF1FE6
:10403000E780604D7C44194697F5FF1F9385C52E98
:10404000138581368297340017F6FF1F1306C62D9D
:10405000977501009385C52F177501001305C530AD
:10406000EF402010AA8415C997750100938585D368
:104070001765010013050550EF403141A6851775FE
:104080000100130565E3EF4051402945EF403144FD
:10409000F2406244D24405618280EFA00027177588
:1040A0000100130565D8EF30602BEF704015EF006D
:1040B000D13317F5FF1F130565F0EF00B120177519
:1040C0000100130565D7EF001134AA84EF30100604
:1040D000EFC02059EF207153EF403022EF30506590
:1040E000EFE01036977501009385C5CB1765010089
:1040F0001305454889C8EF405139A6851775010059
:104100001305C5DD49B7EF40513817750100130598
:1041100025DFEF4091372945EF40713BEFE0B018C4
:10412000EFB0E0426305050E854537050400EF104A
:104130005045977501009385E5C617650100130585
:104140006543EF409134177501001305E5DCEF403E
:10415000D1332945EF40B13797F7FF1F938787D9B0
:1041600083D7070017F7FF1F2313F71E854717F79D
:10417000FF1F230DF71CEF104065EF10C04717F528
:10418000FF1F0355C51CEF20101797F7FF1F83C7AC
:10419000D71BB9EFA303010083274417130671004F
:1041A000854513055030829797750100938585BF2B
:1041B000176501001305053CEF40312D177501000F
:1041C0001305C5D7EF40712C2945EF405130977545
:1041D0000100938525BD176501001305A539EF4042
:1041E000D12A17750100130565DBEF40112A71BD57
:1041F00097750100938505BB176501001305853789
:10420000EF40B128177501001305C5D665BF977536
:104210000100938525B9176501001305A535EF4009
:10422000D12617750100130525E7EF401126294512
:10423000EF40F1290145EF20303F51BF411122C429
:1042400037E404008327041A06C68297EF20701310
:104250008327040817F5FFFF1305857F829797F7DB
:10426000FF1F2381A70C17F5FF1F130565D8EF204B
:10427000E02E2244B2404101B9BB411122C4914613
:104280002A84138601349D652D4506C697E0FF1FDD
:10429000E7806027B7F7070003C70701A547631347
:1042A000F70001A09306001001469D65254597E0A3
:1042B000FF1FE7804025238081342244B24091468D
:1042C000138601349D652945410117E3FF1F6700EF
:1042D0008323B7E704001171FC47CED79389C1252A
:1042E000A2DDCAD986DFA6DB2E8432892E86AA8576
:1042F0004E85829783C70900130780029387E707DB
:1043000093F7F70F636AF774176701001307872E97
:104310008A07BA979C43BA9782878D4797750100A1
:10432000938585AA176501001305C524630BF40066
:10433000EF40B115176501001305C567EF40F11493
:10434000FDA2EF4091141765010013052568EF40A9
:10435000D1132945EF40B117930720F811469385F3
:10436000C1254A85238EF124A38F0124EFF06FDB52
:104370002A840DC597750100938505A51765010071
:104380001305451FEF407110A28517650100130545
:10439000A567EF40910F2945EF4071139775010014
:1043A000938585A2176501001305C51CEF40F10D2B
:1043B0001765010013058566EF40310D2945EF4073
:1043C00011114165930730FA05469385C1257D1586
:1043D000238EF124EFF0EFD42A840DC597750100E8
:1043E0009385859E176501001305C518EF40F109F7
:1043F000A2851765010013052561EF4011092945C4
:10440000EF40F10CB7E70400BC4F0566130606C881
:10441000A14517F5FF1F0345E5F08297FE506E5446
:10442000DE544E59BE591161828091476301F402F6
:10443000977501009385459917650100130585134C
:10444000EF40B1041765010013058560C5BDB7E7EE
:104450000400FC4F914517F5FF1F0345A5EC82971B
:104460009775010093854596176501001305851022
:10447000EF40B101176501001305455FEF40F10002
:104480002945EF40D104EF1090609145E1A28547A6
:104490006301F40297750100938505931765010088
:1044A0001305450DEF40617E176501001305855D1D
:1044B00071B597F7FF1F239227E9B7E70400056658
:1044C000BC4F130606C8C145A9B78D476301F40266
:1044D000977501009385458F1765010013058509C0
:1044E000EF40A17A176501001305855B81BD930735
:1044F00040F811469385C1254A85238EF124A38F68
:104500000124EFF00FC22A84E30A05F09775010039
:104510009385858B176501001305C505EF40E1768E
:10452000A285176501001305254EEF400176294548
:10453000EF40E179E5B59147E31CF4F8B7E70400F3
:10454000FC4F9305000217F5FF1F0345A5DD829779
:10455000977501009385458717650100130585014F
:10456000EF40A172176501001305055501BF89478A
:1045700063E1870297750100938505851765010042
:10458000130545FFEF4061701765010013050554E1
:1045900075B383C4E12583C7D12597750100938541
:1045A000A582A204176501001305C5FCDD8CEF4050
:1045B000C16DA2851765010013058552EF40E16CBE
:1045C000C2042945EF40A170C1849305D4FF93969E
:1045D0000401C1824A8693F5F50F1385F125EF108A
:1045E000C07DE35D90E2930750F8238EF12483C7EA
:1045F000390022869385C12585074A85A38FF1243A
:10460000EFF02FB22A84E30B05E097650100938554
:10461000A57B176501001305E5F5EF400167A2854D
:1046200017750100130505A409B7894763E18702DF
:10463000976501009385457917650100130585F39A
:10464000EF40A164176501001305454BC5B9EF1094
:104650001044A2851385C125EF204076C1B38D4754
:104660006301F402976501009385057617650100E3
:10467000130545F0EF406161176501001305C54959
:1046800075B9B76602000146B7750200054597E0A7
:10469000FF1FE78040E7930760F8238EF124A38F84
:1046A00001249307002623A0F126E57793870721AD
:1046B0002392F1263146A383A1269385C1254A85FD
:1046C00023830126EFF0EFA52A84E30905D497653B
:1046D00001009385656F176501001305A5E9EF409B
:1046E000C15AA28517650100130585443DBDB14738
:1046F0006301F402976501009385056D176501005C
:10470000130545E7EF40615817650100130505449F
:1047100035B1B7E70400FC4F9305000417F5FF1F00
:10472000034545C08297EF109036B14525B79147B4
:1047300063E18702976501009385056917650100AC
:10474000130545E3EF406154176501001305C541AA
:10475000F5B683C4012683C7F125A204DD8C8E043F
:10476000B77702006D14BE942286A68517650100F6
:104770001305C540EF406151B7E70400FC472286AE
:10478000938511262800829793160401C182300078
:10479000A685094597E0FF1FE780E0D62A8419C562
:1047A000176501001305453FEF40E162930770F87C
:1047B00019469385C1254A85238EF124A38081263D
:1047C000EFF02F962A84E30B05C4976501009385CB
:1047D000A55F176501001305E5D9EF40014BA285E0
:1047E000176501001305453C89B399476301F4102F
:1047F000976501009385455D17650100130585D711
:10480000EF40A148176501001305853B05BE9147A0
:1048100063E18702976501009385055B17650100D9
:10482000130545D5EF406146176501001305C53AEC
:1048300031B683C4012683C7F125A204DD8C8E0422
:10484000B77702006D14BE942286A6851765010015
:104850001305C539EF406143B7E70400FC472286E2
:10486000938511262800829793160401C182300097
:10487000A6850D4597E0FF1FE780E0C82A8419C58B
:104880001765010013054538EF40E154930780F8A0
:1048900019469385C1254A85238EF124A38081265C
:1048A000EFF02F882A84E30B05B697650100938506
:1048B000A551176501001305E5CBEF40013DA28529
:1048C00017650100130585358DB199476301F40221
:1048D000976501009385454F17650100130585C94C
:1048E000EF40A13A176501001305C53481BCB7E755
:1048F0000400FC4F9305000417F5FF1F034585A234
:104900008297EF10D0189945B1B38D476301F40237
:10491000976501009385454B17650100130585C513
:10492000EF40A136176501001305453201BC17653C
:1049300001001305A532EF40014A1305C01297E0AC
:10494000FF1FE780409F0145EFE02FA60D45EFF0E8
:10495000DF92294597E0FF1FE780E09D97E0FF1F6A
:10496000E780008F65BC99476301F40297650100F9
:1049700093858545176501001305C5BFEF40E130FC
:10498000176501001305452E55BA03C7112683C7C5
:10499000012622075D8F9166BA96C2061166C18212
:1049A0001306F6EF8D476363D60297E7FF1F9387E1
:1049B00027649C4B03C6F1259386C70039C603D6EE
:1049C00007005DCA8907E39CD7FE89471307A0F853
:1049D00011469385C1254A85238EE124A38FF124B6
:1049E000EFE03FF42A84E30B05A29765010093856D
:1049F000A53D176501001305E5B7EF400129A28524
:104A000017650100130585270DB603D6070063025D
:104A1000E60A8907E39BF6FE8D474DBF9147630287
:104A2000F402976501009385253A17650100130587
:104A300065B4EF408125176501001305A5256FF0CA
:104A4000FF8FB7E70400FC4F9305000817F5FF1F21
:104A50000345458D829705BC976501009385C53652
:104A600017650100130505B1EF402122176501000C
:104A70001305C5236FF09F8C2390E70017E5FF1FF8
:104A800013050557EFE02020976501009385C53396
:104A900017650100130505AEEF40211F17650100E2
:104AA0001305C521EF40611E2945EF404122814792
:104AB00031BF2390070017E5FF1F13056553EFE093
:104AC000801C97650100938525301765010013054B
:104AD00065AAEF40811B176501001305A51FD9B713
:104AE000411122C406C6834705002A849DC39765E9
:104AF000010093852529176501001305A5A7EF403F
:104B0000C1184C40176501001305055CEF40E11723
:104B100075A05841B707CF009387777D6313F706D9
:104B2000976501009385052617650100130585A487
:104B3000EF40A1151C448356E4008355C40003C60E
:104B40000700176501001305A559EF400114294519
:104B5000EF40E1170357E40097E7FF1F83D7277F54
:104B60006307F7008355C4000844EFE0CF9703566E
:104B7000E4008355C40008442244B24041016FF070
:104B80004FF5B707CC009387777D631FF7029765D2
:104B900001009385251F176501001305A59DEF40B2
:104BA000C10E1C448356E4008355C40003C60700AD
:104BB000176501001305C552EF40210D2244B24094
:104BC000294541016F40A110B707CE009387777D3B
:104BD0006302F702976501009385C51A1765010006
:104BE00013054599EF40610A4C4017650100130514
:104BF000654429BFB2402244410182805171CAD12B
:104C000037E904008327C904A2D52E8686D7A6D308
:104C10002E84AA851385C125829783C7C1251307D2
:104C2000700A638DE70C636CF7001307600A6382F8
:104C3000E704BE502E549E540E596D6182801307B6
:104C4000800A6382E7121307900AE394E7FE8D4718
:104C5000630BF416976501009385C518176501006D
:104C600013054591EF406102176501001305C5ADBD
:104C700015A08D476306F40297650100938585169C
:104C8000176501001305058FEF402100176501002E
:104C90001305C5A4EF30717F2945EF40410351BF93
:104CA000854717650100130525A517E7FF1F230793
:104CB000F768EF404112B7750200B766020001467F
:104CC000054597E0FF1FE7800084930760F8238E77
:104CD000F124A38F01249307002623A0F126E57772
:104CE000938707212392F126B14523830126A383CD
:104CF000A1261385C125EF20600C25BF914763E1F4
:104D00008702976501009385E50D1765010013057E
:104D10006586EF309177176501001305E59F9DBF0C
:104D200083C4012683C7F125A204DD8C8327C9042F
:104D30006D14228693851126280082978E0493167F
:104D40000401B7750200C1823000A695094597D0CD
:104D5000FF1FE780407B930770F8238EF12499456D
:104D6000A380A12679B7914763E187029765010087
:104D700093854507175501001305C57FEF30F17086
:104D8000176501001305C59A31B783C4012683C78F
:104D9000F125A204DD8C8327C9046D142286938536
:104DA0001126280082978E0493160401B77502001D
:104DB000C1823000A6950D4597D0FF1FE780A074F3
:104DC000930780F859BF1765010013052599EF4037
:104DD00081001305C01297D0FF1FE780C055014521
:104DE000EFD0BFDC0D45EFF04FC9294597D0FF1F2D
:104DF000E780605497D0FF1FE78080451DBDB7E76F
:104E000004004111FC4726C29384C1252E8606C6A4
:104E100022C44AC02E842A89AA852685829797654E
:104E200001009385E5FD175501001305A574EF30CA
:104E3000D16583C5C125176501001305A5A2EF3013
:104E4000D1642945EF30B16883C704004147938797
:104E5000070693F7F70F6365F74817670100130715
:104E6000A7838A07BA979C43BA9782879D476303B3
:104E7000F402976501009385A5F817550100130505
:104E8000656FEF309160176501001305259EEF30C7
:104E9000D15FD1A283C7D125ADCF83D7012603D758
:104EA000E125C207D98F17E7FF1F232DF74883C7D6
:104EB0006400976501009385A5F41755010013055B
:104EC000656B17E7FF1F230EF746EF30115C97E77E
:104ED000FF1F938727478C4317E6FF1F034666464D
:104EE000176501001305459AEF30315A2945EF3017
:104EF000115EA38E01242244B240924402499307DA
:104F000000F8238EF1249D451385C12541016F10C2
:104F1000F06AEF300065239FA124935705012A848E
:104F20002380F126935785010145A380F126EF30B8
:104F300000642381A12697650100938565EC1755D0
:104F4000010013052563EF30515403C62126A285C5
:104F5000176501001305C59441BFCD476301F402F5
:104F6000976501009385C5E9175501001305856014
:104F7000EF30B151176501001305059409BF37E4FF
:104F800004007C4441469385D1251385413D829799
:104F90001385413DEF00C07CB92D83C7E12603C7CF
:104FA000D126A20703238405D98F17E7FF1F2319F2
:104FB000F7381306000A89452244B2409244024958
:104FC00017E5FF1F03450536410102838D47630145
:104FD000F402976501009385A5E2175501001305BA
:104FE0006559EF30914A176501001305A59C45B539
:104FF00003C4E12583C7D12597650100938545E06A
:105000002204175501001305E5565D8CEF30F1477A
:10501000A285176501001305A58BEF3011472945BF
:10502000EF30F14A0D469385C1252285EFE07F8F51
:10503000AA8415C997650100938585DC1755010081
:1050400013054553EF307144A6851765010013051C
:105050006589EF3091432244B24092440249294588
:1050600041016F30D14697E7FF1F2398872CB7E7A0
:105070000400116603A38705130606E891452DBFBA
:105080008D476301F40297650100938565D7175535
:1050900001001305254EEF30513F17650100130540
:1050A00025A0F5B303C4E12583C7D1259765010089
:1050B000938505D52204175501001305A54B5D8C7A
:1050C000EF30B13CA285176501001305E582EF3092
:1050D000D13B2945EF30B13F0D469385C12522854F
:1050E000EFE03F84AA840DC197650100938545D107
:1050F0001755010013050548EF303139A6851765AE
:1051000001001305A580B1B797E7FF1F23968722FB
:10511000B7E70400116603A38705130606E89305A5
:10512000000259BD894763E18702976501009385B5
:1051300025CD175501001305E543EF3011351765EF
:1051400001001305A598A1B383C4E12583C7D12528
:10515000976501009385C5CAA20417550100130580
:105160006541DD8CEF307132A685175501001305BE
:10517000657BEF3091312945EF307135228693857B
:10518000C1252685EFE0EFF92A84630A05169765A5
:1051900001009385E5C6175501001305A53DEF30C5
:1051A000D12EA28517550100130505795DB58547F8
:1051B00063F78714834519002244B24092440249A0
:1051C000B335B00097E7FF1F238AB71617550100C4
:1051D0001305C57741016F30512BA2852244B2409F
:1051E00092444A85024941016FF05FA199476301EA
:1051F000F402976501009385A5C0175501001305BA
:105200006537EF309128176501001305E5A541B119
:1052100003C4E12583C7D12597650100938545BE69
:105220002204175501001305E5345D8CEF30F1259C
:10523000A285175501001305E572EF3011252945A8
:10524000EF30F12819469385C1252285EFE06FEDF7
:10525000AA840DC197650100938585BA1755010091
:1052600013054531EF307122A6851755010013054E
:105270006570C5B397E7FF1F2398870CB7E7040055
:10528000116603A38705130606E8930500082DB3EE
:105290008547976501009385A5B61755010013054D
:1052A000652D6309F400EF30511E175501001305F9
:1052B000A56DF1BEEF30711D175501001305456E48
:1052C000EF30B11C2945EF3091202244B240924486
:1052D000024997E7FF1F2395070641016F30C01C65
:1052E000976501009385C5B1175501001305852801
:1052F000EF30B119176501001305459B49BEB24057
:1053000022449244024941018280411106C622C4CE
:10531000EFE02FE19377F50F95CB2A849765010095
:10532000938585AF175501001305C524EF30F1159E
:105330009375F40F176501001305C5D2EF30F11412
:105340002244B240294541016F307118B2402244D5
:105350004101828001114EC6B28917E6FF1F035634
:10536000E6F726CA4AC806CE22CCAA842E891D2377
:1053700097E7FF1F83C787FDA9CB03C4440083C7FA
:105380003400176501001305E5D922045D8CEF3068
:10539000D10F4A86A68522858D3F638F090297E744
:1053A000FF1F83C787FA8DCB6308090297E7FF1FAA
:1053B00083C7C7F895E36244F240B249CA8526859F
:1053C0004249D24405616F10701F17650100130533
:1053D000E5D5EF305120D1B7F2406244D244424982
:1053E000B2490561828083475500834545001765B2
:1053F00001001305E5D1A207DD8D6F301109176596
:1054000001001305E5CF6F30111D8D4763F2B70A18
:10541000011126CA06CE22CC0344350097E4FF1FB3
:1054200083C4B4F297650100938505D1B33780003A
:1054300017E7FF1FA30BF7F009C4976501009385D9
:1054400065D017650100130565D0EF30110497E7AB
:10545000FF1F83C797EF638397001D2C97E7FF1FFC
:1054600083C7B7EE9DC385472306F100B7E7040065
:1054700083A747177000854513055030829717653D
:1054800001001305A5CDEF3011159967938757EEED
:105490002316F100680085479145A3078100230783
:1054A000F100EF10B011F2406244D24405618280F5
:1054B0008280894763F2B708011122CC06CE26CA42
:1054C0008344250085472A846398F404914763F058
:1054D000B704034545008347340022055D8D97E7F7
:1054E000FF1F239DA7DE35219967938767EE23145D
:1054F000F1008347340023059100A305F1008347A1
:105500004400954528002306F100EF10300BF240CF
:105510006244D24405618280FDF89967938767EE03
:105520002314F10097E7FF1F83D747DBA305F100A2
:1055300023050100A183F1B782800111996722CC74
:10554000D51717E4FF1F130464E02314F100834709
:10555000040026CA97E4FF1F938464DF2305F1004B
:1055600083D7040028009545A305F100A18306CE4A
:105570002306F100EF10900403D6040083450400D5
:1055800017650100130505BFEF302170F24062443A
:10559000D244056182809D677971D9172316F10085
:1055A00097E7FF1F83C787DA06D62307F1009DCB55
:1055B000B7E70400FC4741469385413D1305F100E0
:1055C00082976800CD45EF10607F97E5FF1F83C588
:1055D000E5D7176501001305E5BCEF30016BB2504C
:1055E00045618280B7E70400BC4741468145130509
:1055F000F1008297F9B7B76702036971938757AAD9
:105600003EC4930710502316F10097E7FF1F9387BE
:10561000E7D383C7070023248112A30701002307D0
:10562000F10097E7FF1F938787D283D7070037E4FE
:105630000400232611122318F10097E7FF1F938718
:10564000E7C983D70700414648082319F1007C4485
:105650009385413D8297F1452800ED2A2312A1024E
:105660007C442C002810794682973C441305610441
:105670001306900D8145829730109305700F0145F8
:10568000EFD03FB58320C11203248112556182807F
:10569000B7C7A55A01119387C7333EC497E7FF1FC9
:1056A00083C7B7CA3EC6B7F7070003C7070106CED0
:1056B00022CCA5476313F70001A01164930504F001
:1056C000930600100146254597D0FF1FE780A0E311
:1056D0003000930504F0A146294597D0FF1FE780CD
:1056E00080E297E5FF1F83C555C6176501001305C6
:1056F00025BCEF308159F24062440561828001117E
:105700009165A1463000938505F02D4506CE97D0D2
:10571000FF1FE78040DF2247B7C7A55A9387C733EB
:105720006312F702B245176501001305A5ABB33547
:10573000B00097E7FF1FA38AB7C0EF300155F240D2
:105740000561828085478545176501001305C5AB56
:1057500017E7FF1FA30BF7BEEF302153153FC5B767
:10576000B7C7A55A79719387F7353EC6B7E70400E6
:10577000FC47AA8506D622D4414608088297B7F787
:10578000070003C70701A5476313F70001A01164D1
:10579000930504E8930600100146254597D0FF1FA6
:1057A000E78060D67000930504E8D146294597D07C
:1057B000FF1FE78040D517650100130525B3EF30C3
:1057C0008161B25022544561828079719165D146E0
:1057D0007000938505E82D4506D697D0FF1FE7801A
:1057E00080D23247B7C7A55A9387F73517650100AE
:1057F000130585A9631EF700B7E70400FC4713856E
:10580000413D41460C088297176501001305C5A567
:10581000EF30615CB25045618280B7F7070003C783
:105820000701A5476313F70001A091654111930695
:1058300000100146938505E8254506C697D0FF1F51
:10584000E78060CCB240176501001305E597410180
:105850006F306158C16769768146FD170506139759
:10586000060141836364B7003E8582803307D5001B
:1058700003470700B98F214713F817008583630595
:105880000800B18FC207C1837D171377F70F6DF73B
:105890008506F1B725CD25478546637AB7064111C0
:1058A00022C406C626C20347150083460500316898
:1058B0002207558F931687002183558F4207418316
:1058C0001308C8552A848546631C0703034725002F
:1058D00011486377E80213085700639305039304A4
:1058E0003700A301C50021822302C500A6859D378C
:1058F000B30794002380A7002181A380A7008146DD
:10590000B2402244924436854101828085463685E4
:105910008280B7C7A55A01119387E7343EC42AC6CF
:10592000B7F7070003C7070106CE22CC26CAA54752
:105930006313F70001A091642A84938504EE930613
:1059400000100146254597D0FF1FE780C0BB3000FF
:10595000A146938504EE294597D0FF1FE780A0BAA2
:10596000A285176501001305A596EF300132EFF00F
:105970009FC8F2406244D244056182800111916562
:10598000A1463000938505EE2D4506CE97D0FF1F2A
:10599000E78060B72247B7C7A55A9387E7346314F7
:1059A000F702B245176501001305058897E7FF1F49
:1059B0002396B792C205C181EF30212DEFF0BFC30E
:1059C000F24005618280D147D1451765010013057A
:1059D000A58717E7FF1F2313F790EF30012B17E57B
:1059E000FF1F0355A58F3537E1BF011126CA06CE2B
:1059F00022CC93F71500AE848DCBAD6737170040EE
:105A00009387A7AA1CC3B7E70400BC4F130600196D
:105A1000854517E5FF1F0345458C829713C5140084
:105A2000F2406244D2440561828093F7250063838B
:105A30000712976501009385658F2D464800EF306A
:105A4000611997E5FF1F83C57590854793C42400AE
:105A500063E1B70489CD97E7FF1F83C7078F85C32D
:105A60008545170500201305E5F8EF10203513953F
:105A7000040197E7FF1FA38B078C418155B7416550
:105A80000546970500209385E5F67D15EFF0FF8725
:105A9000F9BF170400200344E4F59707002083C7EB
:105AA00077F522045D8CAD679387B7556306F408DC
:105AB00063E68702A9679387A7556306F40897E70B
:105AC000FF1F83C787888DE741652E867D15970563
:105AD0000020938525F2EFF05F83B9A0B16793872B
:105AE000C755630EF400B5679387D755E319F4FCE7
:105AF00017050020130505F0EF10402C35A00546D2
:105B000017050020130505EFEFF0DF8497E7FF1F6F
:105B100083C7C78391EB4800EF302134931505010B
:105B2000C1814800EFD02F9CA285175501001305B5
:105B3000E57DEF30811525BF17050020130585EBA6
:105B4000EFF07F8AD5B7170500201305A5EAEFF01F
:105B50001F8BD9BF93F745000145E38307EC175529
:105B600001001305E57BEF300127EF10003713C567
:105B700044007DB5411122C437E404005C5C06C6D4
:105B800035469755010093852532176501001305A9
:105B900065BE829701E9175501001305E579EF30DD
:105BA000812301A08327041C82972A840545EF8066
:105BB0002075EF10C168EF100147EF70B029228502
:105BC000B2402244410182801567B7170040130795
:105BD000575598C3D8439D66558FD8C3D843FD7693
:105BE000758FD8C3D8431367F70FD8C3356713072A
:105BF000C7CC98C3828041111305800406C622C415
:105C000026C24AC097C0FF1FE780604A85457D5580
:105C1000EFC0FFE085457D55EFC0DFEA3714004057
:105C20008327840A8D451305002093E7072023244A
:105C3000F40AEFC0DFDEB7E40400EFD04F90C8589D
:105C40001309840C1304C40CEF30E118176501002C
:105C5000130545B2EF3021188327C4FF8545414520
:105C600093E70708232EF4FEEFC0DFE58D4513050B
:105C70000008EFC03FE5EFC0BFFF0145EFD06F82E6
:105C800085450545894717D7FF1F2303F76CEFD0DC
:105C9000EF8237070004B7E700E023A0E710EFD05A
:105CA000DF8FEFD05FA3F935EFF07FA5EFF01FCDC9
:105CB000EFE0CFD88D450D65EFC0DFE01705002080
:105CC000130545E385671CC589672320250140C16D
:105CD0002326250100C95CC983A7841E829783A758
:105CE000040817050000130585D0829797D7FF1F7A
:105CF0002385A75EBC4C1306006485458297E93571
:105D000097C0FF1FE780C06D01458280B7F707008D
:105D100003C70701A547AE866316F70093974501B1
:105D200091C301A0AA850146254517C3FF1F67003F
:105D3000837D4111B2862E86AA852D4506C697C061
:105D4000FF1FE780407CB2400145410182809307FC
:105D5000000463E6C7021D71A2CC2A84080886CE1F
:105D600032C6EF203167B2461008A285294597C098
:105D7000FF1FE7804079F6406644256182803955EF
:105D80008280411126C2AE848D4522C406C62A8473
:105D9000EFC05FD3B717004099C803A5C70C418D6A
:105DA00023A6A70CB240224492444101828003A55D
:105DB000870C418D23A4A70CF5B783470500034743
:105DC0001500A207D98FC2076177C1871307272063
:105DD0006397E70083452500370504005DB782809F
:105DE00097D7FF1F9387075718429C4383D64500D8
:105DF0000345070083C5C700035646006396A50008
:105E000083D5E700638DD502011106CE2386A70056
:105E10002397D700B705CF00DC4B9385757D050729
:105E20007D162EC2230001003AC42316C100231799
:105E3000D10099C30A858297F240056182808280F1
:105E4000DC4DDC4B81CFB7E70400904503A3870509
:105E5000914517D5FF1F03452550028382806D7140
:105E60003C083EC6B707E500232291103EC8AA842D
:105E70003C083285232611103ECA2324811023209A
:105E800021112E89EF2090672A8497550100938570
:105E9000E552174501001305E56DEF20115FA2855E
:105EA0001755010013058561EF20315E2945EF206C
:105EB0001162B705CB009385757D6800EF10A04394
:105EC000A2856800EF203059014781467000CA85DD
:105ED0002685EF10C06215C52A8497550100938569
:105EE000E54D174501001305E568EF20115AA2851D
:105EF000175501001305455DEF2031592945EF2065
:105F0000115D8320C11003248110832441100329D3
:105F100001105161828097D7FF1F9387A7431842D2
:105F20009C43797122D406D60348070083C8070131
:105F30002A8483D64500035546006396080183D81A
:105F40002701638DD8022388070105072399D7000D
:105F50003708CC00DC4B1308787D3ACC1307F5FFEB
:105F600042CA23080100231EE100231FD10099C764
:105F7000080832C62EC482973246A2452285C5350E
:105F8000B2502254456182806D713C083EC0B70713
:105F9000E5003EC23C083EC4232611102324811094
:105FA0002322911023170100231801002319010057
:105FB000231A0100231B010097D7FF1F83D7470730
:105FC00099E3C167FD172316F10097D7FF1F83D709
:105FD000470691EB97D7FF1F9387C7379C439C4396
:105FE000DC4783D7070017D4FF1F13046404584C01
:105FF0002317F10083574400484B2318F10005EDA7
:106000009755010093858542174501001305855674
:10601000EF20B1471755010013058542EF20F146E7
:106020002945EF20D14A8320C11003248110832405
:1060300041105161828097D7FF1F83C7D7FF89EB3B
:10604000B7E70400BC5782975C4C23AA0700E1BF66
:10605000FD1797D6FF1FA380F6FE0356070183475F
:1060600004014C470A85230BF100EF20F03C97D741
:10607000FF1F9387272E9C430147814688430A864A
:106080006C00EF10C047AA841DC997550100938585
:10609000E539174501001305E54DEF20113FA685B1
:1060A000175501001305853AEF20313E2945EF20B1
:1060B0001142584CB7E70400BC57484B69B797D713
:1060C000FF1F83C757F7F5D7B7E70400BC4F10444D
:1060D000854517D5FF1F034525288297A9B75C4E34
:1060E000DC4BA9CBA1C9411122C4174501001305FE
:1060F00065482E84975501009385853106C6EF20AB
:10610000D138A2851755010013058536EF20F137E8
:106110002945EF20D13BB7E704002244B24003A356
:10612000870517D5FF1F0345252313064006914514
:10613000410102838280411122C417D4FF1F13043E
:1061400024ED1C4C06C689C7DC4399C34C48829792
:10615000584CB7E70400BC57484B82975C4CB240A0
:10616000224423AA07004101828017D7FF1F13078B
:106170000717834707009306F00B850793F7F70F80
:1061800063E9F60097D6FF1F238BF614034507003B
:106190008280930700F8FDB7835745006386070E9A
:1061A00001114AC817D9FF1F130989E852C4032AED
:1061B000C90106CE22CC03274A0126CA4EC656C2C2
:1061C000F15721EF1307D00DFD576368C704B7E9F6
:1061D000040083A709072A8413058600420541812C
:1061E000B284AE8A8297232AAA000325C9015C499A
:1061F0009DEF975501009385A51F174501001305D5
:106200006537EF209128175501001305A52EEF20C3
:10621000D1272945EF20B12BDD57F2406244D2440B
:106220004249B249224A924A3E850561828093875B
:106230004400B705CF002319F5009385757D31051E
:10624000EF10600B0325C901834564003105EF2081
:1062500090200325C9012686D6853105EF20D01D63
:106260007146A2854A85EF20F116504419CA83A7CA
:106270008905854517D5FF1F0345050E8297814780
:1062800069BFEFF07FD0E5BFFD573E8582804111A9
:1062900026C297D4FF1F9384A4D9D84C22C437E4D4
:1062A00004003C54484B06C68297DC4C0323C405CB
:1062B0002244B240924423AA070017D5FF1F03458A
:1062C000A509854541010283411126C297D4FF1FCC
:1062D000938444089C4006C622C44AC0C9CBDC4310
:1062E000D9C75CC12300B5002A8497550100938566
:1062F000650B174501001305E527EF201119294506
:10630000EF20F11C9C4023A4070023A2070097D78D
:10631000FF1F9387E7CFDC4FDC4B81C72955EFF098
:106320009FE197D7FF1F9387A7D0DC4FDC4B91C32A
:10633000B93F37E904008327C905894517D5FF1FF1
:106340000345850182978327C905914517D5FF1F0E
:106350000345850082979C4003A34701630903001E
:1063600022852244B2409244024941010283B24054
:10637000224492440249410182800111328506CEB5
:1063800022CC26CA2E84EF207017AA8497550100CC
:1063900093858504174501001305C51DEF20F10EF7
:1063A000030784000356640083554400A6861755EE
:1063B00001001305E50DEF20510D2945EF203111A6
:1063C00097D7FF1F83C727C5639897000145EFF054
:1063D0009FD681450A85CD3DF2406244D244056195
:1063E00082806D71232481102326111023229110A5
:1063F00093F745002E84638507123C083EC0B7071B
:10640000E5003EC23C083EC42317010023180100EA
:1064100023190100231A0100231B010097D7FF1F36
:1064200083D707BF99E3C167FD172316F10097D7FC
:10643000FF1F83D707BE91EB97D7FF1F938787F185
:106440009C439C43DC4783D7070017D7FF1F1307E4
:1064500027BC2317F100544F835747002318F1003E
:10646000DC4A95EF97550100938545FB17450100E0
:1064700013054510EF20710117550100130545FC68
:10648000EF20B1002945EF209104134544008320FB
:10649000C11003248110832441105161828097D759
:1064A000FF1F83C757B72555ADCBFD1717D6FF1F65
:1064B000A303F6B603D6060183470701CC460A8537
:1064C000230BF100EF20407797D7FF1F938787E8D2
:1064D0009C4317D7FF1F1307A7B397660100938646
:1064E000A6C888430A866C00EF106001AA8451DDBB
:1064F00097550100938585F217450100130585071F
:10650000EF20A178A68517550100130525F4EF208B
:10651000C1772945EF20A17B2685EFF0DFC1B5B714
:1065200093F725009DC3B7E70400BC47414681456A
:10653000280882972555EFF01FC028089305F00F13
:10654000EFF09FD81345240099B793F71500014544
:106550009DDFEFF07FA31345140015BF5C4D411183
:1065600006C688C317D7FF1F2326F7DEB7E7040048
:1065700083A70708170500001305E5E68297B240D8
:1065800097D7FF1F238AA7DC0145410182800111B3
:106590009307700F2316F10006CE97D7FF1F83C70E
:1065A00077DC8DE7B7E7040083A7870D17D6FF1FB9
:1065B000034646D36C0017D5FF1F0355E5DA8297D3
:1065C0003335A00097D7FF1FA38EA7D8F2400561EF
:1065D000828041119397050122C406C626C2C18755
:1065E0002E8463D40702B7E40400FC5417D5FF1FC0
:1065F000034545CF829719C1BC5482972165218DEF
:10660000B240224492444101828093F715008DC725
:10661000B7E7040083A7471A17D6FF1F130646A340
:1066200097F5FF1F9385055217D5FF1F034585CBAF
:10663000829713451400E9B793F7250099CFB7E780
:106640000400BC4F13060064894517D5FF1F03459E
:1066500065C982971345240065B793F785009DC7E8
:10666000B7E7040003A8871A1307401F97D7FF1F37
:1066700083C747C7814613064006994517D5FF1FB4
:10668000035585CE0298134584009DBF93F74500BE
:106690000145BDD7B7E4040083A7041817D5FF1F31
:1066A000035585CC8297BC4C13060064914517D5E1
:1066B000FF1F034525C382971345440091B797D721
:1066C000FF1F83D767CA6396A70217D7FF1F231E32
:1066D000B7C817D7FF1F231BC7C817D7FF1F23181B
:1066E000D7C82E8617550100130585F6BE856F2085
:1066F000C15917550100130525F76F20C16D0357C8
:106700004500011106CE22CC97D7FF1F83D7C7C5FE
:1067100017550100130545F56310F706C167F91712
:1067200017D7FF1F2322F7C437E4040097D7FF1FB2
:1067300023AE07C27C4C894517D5FF1F034585BA98
:1067400082977C4C914517D5FF1F0345A5B98297C9
:1067500097D7FF1F83C777BF95C78547A307F1006A
:10676000832744171306F10085451305503082979F
:10677000175501001305C5E4EF20E165F2406244BE
:106780000561828097D7FF1F83C747BC175501005B
:106790001305C5E7F5F38547A307F10083274417E1
:1067A0001306F100854513055030829717550100F7
:1067B000130545E3D1B77D15954763E0A71A175731
:1067C00001001307A7DC0A053A951C41011122CCF0
:1067D00006CE26CABA972E84828717550100130564
:1067E00025E9EF20415F0DA203C725009947631DEE
:1067F000F7002E85EFF0BFF08345640017550100C8
:10680000130505E8EF20614897D7FF1F238F07B2D4
:1068100017550100130585E8E9B703C7250095471B
:106820006317F702C16717D7FF1F0357E7B3F917BD
:1068300003D5A5006307F702B7E7040083A7C717CE
:10684000829717550100130565E6EF20C15885476B
:1068500017D7FF1F230BF7AE17550100130585E768
:1068600049B797D7FF1F2391A7B083D7E500B7E4B7
:106870000400096617D7FF1F2319F7AE83D7050158
:106880001306069017D5FF1F0345C5A517D7FF1F91
:10689000231EF7AC83D72501A14517D7FF1F231867
:1068A000F7ACBC4C8297BC4C13060064914517D5DD
:1068B000FF1F034525A382970356E4008355A400D8
:1068C000175501001305C5DFEF20213C49B71755C7
:1068D00001001305E5E031B783C525009147639AB0
:1068E000F502854717550100130505E1A307F100DF
:1068F000EF20614EB7E7040083A747171306F100A6
:106900008545130550308297F2406244D2440561B8
:1069100082809947639EF5002285EFF05FDE834514
:106920006400175501001305A5D5EF200136E9BF16
:106930009547639FF5008347140017550100130521
:10694000A5DBE39007EA175501001305A5DC51BD4F
:1069500017550100130585DCC9BF82806D712324A2
:1069600081102326111023229110328401CD8947F2
:106970006306F5028320C110032481108324411093
:106980005161828017550100130505DAAE84EF20AE
:106990008144A2852685EFE08FC6E9BFB7E70400F2
:1069A000FC4728008297175501001305A5D8EF2052
:1069B00081428347810039C01307000B638EE700D3
:1069C0001387A7051377F70F8D4663E9E602A285C3
:1069D0002800EFE0AFA279BF8547E3FD87F8834544
:1069E000910017450100130565F6B335B00097D740
:1069F000FF1F2385B794EF204129ADBF03479100C6
:106A0000A207D98F35671307D755638DE7066366ED
:106A1000F7022D671307B7556381E7063167130740
:106A2000C7556386E70429671307A7556392E702F2
:106A3000A2852800EFE0BF9C35BF39679306E76564
:106A40006383D70663E9F6001307E7556388E70415
:106A5000A285280089B73D679306F755638AD70456
:106A60001307F766E396E7FEEFE0FFB221B70146B2
:106A7000A2852800EFE01F8EF5BDA2852800EFE07B
:106A80009F96CDBD8947E3F787EE9305E4FFC205E6
:106A9000C1811305A100EFC00FA5E9BDA2852800A3
:106AA000EFE0BF96C1BDA2852800EFE09FA0D9B559
:106AB000EFE0BFA8C1B5411122C417C4FF1F1304E2
:106AC000E45AAA86175601001306C6AD2285C145B1
:106AD00006C6EF2041310357440097C7FF1F938735
:106AE000E7592393E700035764002394E700B2407B
:106AF000224441018280011106CE22CC6D3F37E451
:106B000004008327841417C6FF1F13062656D54595
:106B100001458297832784179305F10013055030B0
:106B200082978347F100A1C7A30701008327441779
:106B30001306F100854513055030829783274417CB
:106B400017C6FF1F13068653CD4513057030829775
:106B50008547A307F100832744171306F1008545F5
:106B6000130550308297F24062440561828083278A
:106B7000441717C6FF1F13066650CD451305703026
:106B8000D5B7130101DE232C812037E404008327CD
:106B90000408232E1120232A912023282121232693
:106BA000312117050000130505A3829717C9FF1FA0
:106BB00013094973994785442300A9002318F1005C
:106BC00097550100938505A79307400617450100D7
:106BD0001305459A2314F1102304910097C9FF1F50
:106BE0009389E976EF20610A83D5090017550100E2
:106BF0001305059CEF2061092945EF20410D03D5C0
:106C00000900EFF05FEB832744173000854513053B
:106C1000503082978327441717C6FF1F1306064676
:106C2000CD451305703082978327441717C6FF1F81
:106C30001306C642B5451305603082978327441773
:106C400010088945130510318297832744173002B5
:106C50008945130520318297832744159305000544
:106C60000D458297832744159305000511458297AA
:106C7000A301910023029100230491002324011019
:106C800023080100832784163002914513057040C4
:106C9000829783278416130631008545130500402B
:106CA00082978327841650008545130510408297EC
:106CB0008327841610088545130520408297832773
:106CC00084163000854513055040829783270415AC
:106CD0007D558297832744137D5582977D55EFC05C
:106CE0002FC88327440C8297EFC06FA58327841495
:106CF00017C6FF1F13068637D5450145829789477A
:106D00001306700F814508082302F100EFB0EF85EC
:106D10008D471306700F814528022308F100EFB05C
:106D2000CF8491472304F11097C7FF1F9387075C17
:106D3000984383C747003AC42306F100EFE0BF8BB6
:106D4000500085450545EFC0CFC810089305700F6A
:106D50000945EFC00FC830029305700F0D45EFC015
:106D60004FC7300095451145EFC0AFC6C16717C783
:106D7000FF1F1307675FF9171CC32322070017C5FE
:106D8000FF1F1305E555EFC0AFC38327C41D17C50B
:106D9000FF1F1305A55C82973C4803450900854504
:106DA00082978320C1210324812183244121032947
:106DB00001218329C1201301012282800111C167B1
:106DC00026CA06CEAA8422CC17C5FF1F0355C55973
:106DD000F9176306F50437E40400832784122E862E
:106DE0002315B10001478146ED4582977C44035647
:106DF000A1002AC6A68582972C0017C5FF1F035540
:106E0000A556EFC0AFC801CD175501001305858306
:106E1000EF10717C8327C412ED4528008297F24061
:106E20006244D24405618280011106CE22CC2DC974
:106E3000854717C7FF1FA308F72297C7FF1F2385A2
:106E4000072237E40400832784179305F100130514
:106E5000503082978347F100A9CBA3070100832715
:106E600044171306F1008545130550308297832798
:106E7000441717C6FF1F1306661EB545130560307D
:106E800082978547A307F100832744171306F10073
:106E90008545130550308297F24062440561828037
:106EA00097C7FF1FA381071C49BF8327441717C635
:106EB000FF1F1306A61AB54513056030E9BFC16769
:106EC00017C5FF1F0355454AF9176307F500B7E7D4
:106ED000040003A3C7170283828001118547A3071B
:106EE000010017C7FF1F230FF746B7E7040083A76A
:106EF000471706CE1306F1008545130550308297DB
:106F0000F24005618280EFA2BFE12A8408452E8904
:106F1000B28909C900C1970500009385C574610550
:106F2000EF00810181447D5AEF10C00963C3A404BE
:106F30008144EF10200A63C6A40497F7FF1F9387CC
:106F400027C19C43DC47B307F94091872302F40033
:106F5000638109048327C900B307F4409587A3021E
:106F6000F4001C4C89C79C4799C3228582976FA067
:106F70007FDE5C44139714008504BA972390470181
:106F800065B71C48139714008504BA97239007002F
:106F90004DB7832789000547B307F4409587A302BF
:106FA000F40083570400638EE7028DC309476384AE
:106FB000E7040D47E397E7FA97570100938747CA1D
:106FC0001CCC975701009387A7CA11A897570100B7
:106FD000938787901CCC975701009387E7905CC8F4
:106FE00049B7974701009387277C1CCC974701003E
:106FF0009387877CEDB797570100938727CB1CCCED
:1070000097570100938787CBD9BF85E1EFA2FFD2C5
:10701000004618448347940075839D8B6315F700E1
:10702000EF00501C48C46FA09FD38280EFA25FCFB7
:1070300013893500C16442094111AA890144F11440
:1070400013590901054A2EC6EF00D077B2456346B1
:10705000A400014541016FA0FFCF83A709001317CA
:107060001400BA9783D707006388B700639497002A
:1070700063742A010504C1BF0545E9BFEFA27FC9BA
:10708000AA892E89328BB6843A8ABE8AEF80204C38
:1070900055C12685EF1030368D4763E5A7007D5535
:1070A0006FA0BFCA83DB4400EF00D0772A84EF00D3
:1070B000B0789307740031443305850263C5A70295
:1070C000EF005076EF0010762A84EF00F0769307F9
:1070D000740031443305850263CDA702EF0090743C
:1070E0009307450019A8EF00307533058502130793
:1070F000F0179307C017E357A7FC2D55E3C277FBA2
:1071000063000B02D6865286A6854A85EFE010639F
:1071100041BFEF007072330585029307C5FFF1BFD1
:10712000832749001385C90083D52700EFF01FF09E
:1071300071F9B5B76955ADB797F7FF1F239CA7A0A5
:1071400097F7FF1F9387C7A0904381470C463307EB
:10715000F500420741836393B70082805446139839
:1071600047008507C2962390E600D5B797F7FF1F23
:107170009387079E9C4303C58700828017F5FF1FF6
:107180000355459D8280EFA25FBBC1671387D7FF80
:107190006307E5026368A700F117630EF500014578
:1071A0006FA0FFBB1387E7FF630EE500FD171D8D82
:1071B00013351500F5B7EF40003D7D15D5BFEF4005
:1071C000801AE5BFEF40E018CDBFEFA21FB7411115
:1071D000AA8401442EC6EF00F05FB2456346A400C6
:1071E000014541016FA0BFB79C48131514003E959F
:1071F00083570500E387B7FE0504E9BF0348550040
:10720000814693F7F60F63E5070181473E8582804B
:10721000584593975600BA9703D727006316B700CF
:1072200003D70700E304C7FE8506E1BF8346450098
:1072300001479377F70F63E4D700814711A81C45F6
:10724000131657000507B29703D60700E313B6FEDF
:107250003E858280EFA2DFAC93170501C18797FAC4
:10726000FF1F938AEA8E6355F00883A70A00C04780
:107270009C4703570400198D420541816366F50060
:10728000014422856FA01FAD12052A94DDBFDC47A3
:1072900013944900014A3E94834744006341FA0233
:1072A000014A834754006347FA028509C20993D90A
:1072B000090183A70A009847E3EBE9FCD1B71C4416
:1072C00013195A00A6853E994A85EFF01FF011ED7B
:1072D000050AD9B75C4413195A00A6853E994A8518
:1072E000EFF0BFEE19E1050A6DBFE30009FC51BFE5
:1072F000AA8481497DBFEFA25FA41C452A8481E74F
:107300009307C5001CC51C44231204001CC093072E
:10731000F00F63E9B70093F5F50F2285EF10B01376
:107320006FA0FFA393940501C167C18063F7F500C7
:10733000A6852285EF10D015E5B7C18193F5F50F2D
:107340002285EF105011A6852285EF101012C9BFBB
:1073500097E7FF1F9387C77F884382801C4599C7A3
:1073600097E7FF1F23A6A77E014582807D55828077
:1073700097E7FF1F9387C77D98438347450048479A
:1073800092073E958280EFA25F9B617100451C18B9
:107390003EC6B70780013EC81C183ECA835744004A
:1073A00002CE02D002CC231EF100834784002A893A
:1073B00002D22301F1023C083ED402D6EFF05FFB7B
:1073C000835705002316F102EF30706B2307A102EB
:1073D0005C4003556400F18313F717008347F10203
:1073E00052055181F99BD98FA307F102EFE0702676
:1073F00039C5AA8403550500EF80401683D70400E1
:107400002AD26800231CF10083D72400231DF10039
:107410001C4803D647008C43EF1010028347B4008A
:10742000CA86174601001306A6318117A305F4008A
:107430006C004810EFE090305D616FA05F922155C5
:10744000E5BF1C45B1CF03C5A700894613576500AA
:10745000630BD7028D46630ED70285466300D702C1
:10746000130740063305E50203C7B700418B15CB70
:1074700083C7B700BD8B3355F54082801375F50384
:107480001307803EC5B709671375F5031307077126
:10749000D1BF372709001375F5031307077CD9B748
:1074A00001458280EFA27F8903A985006305090455
:1074B0008347B900AE8493F7070E91CF0345990037
:1074C000930520030D810505B305B50288446105C8
:1074D000EFF0B0320DA02E85EFF0BFF62A8401CD7B
:1074E00011238325C900B307B54063F887002E94A4
:1074F000B305A440E1FD6FA09F868545C1BFEFA203
:10750000DF832A8403D50500011132C636C43AC28E
:107510002EC002CA02CC02CEEF80400482452ACAA5
:1075200022852ECCEFF0DFE403570500231EE10097
:10753000EF30F054A24632469247230FA10036871F
:107540004C08B28622850146EFF05FB305616FA05B
:107550001F81EFA28FFE61711C183EC6B707800124
:107560003EC81C183ECA3C0800453ED4AA8402CC42
:1075700002CE02D002D202D6EFF09FDF8357050081
:1075800035592316F102EF30904F2307A10209C4A9
:107590008357440091E721594A855D616FA02FFC14
:1075A0000355640052055181EFE0B00A2A8965D580
:1075B0008347B40093F7070E89C713058401EFF0E2
:1075C000502583574400231EF10083478400230184
:1075D000F1025C4003550900D98313F7070883477C
:1075E0001102231CA10093F7F707D98FA300F10222
:1075F00083572900231DF1005C40F18313F7170026
:107600008347F102F99BD98FA307F102EF70107540
:107610002AD251D1834794006800139757008347BB
:10762000B400FD8BD98FA305F4001C4803D6470096
:107630008C43EF106060A6871747010013074710BF
:10764000740005464C102685EFF05FA32A8929D5E2
:107650008347B400A685FD8BA305F400EFF09FE4FB
:1076600025BFEFA28FED832485FE2A844111268554
:10767000EFF03FDD834734FF93F7070E9DC32AC623
:107680002685EFF05FD019C9834734FFB245FD8BE3
:10769000A309F4FE81C52285EFF0301641016FA0E9
:1076A0000FEC6DDD8327C4FF2685829765F983473C
:1076B00034FF93F7070E81C72285EFF0901503255D
:1076C00084FEEFF01FE9D9BFEFA22FE49C414111E6
:1076D0002A8903C7070089472E8493566700638C65
:1076E000F6020D466382C6049307F0076302F702B1
:1076F0002E85EF10A060AA848149C16B130C49004C
:1077000097E7FF1F9387C7449C43984763ECE902C0
:1077100041016FA04FE303D745008547E3FAE7FE39
:107720002E85EF108061C1BF03D74500E3F2E7FE6D
:107730002E85EF10A05CAA842285EF10805DC20424
:10774000C98C5DBFDC470355A900139A49003E9AD6
:1077500093170501C187635DF00083570A006395A5
:10776000A70263E574038327CA00034D5A001DA0D6
:10777000A1672167A98F1307F7EFE374F7FE6395FD
:107780000900EFF05FA071FD85099DBF83278A0086
:10779000034D4A00835DA90003576900216A138BDA
:1077A000C7003AC6814A33CA4D01631E5D0197E79F
:1077B000FF1F9387673A9C43E1DBA286628681457F
:1077C00026858297D1B7A1679387F7EF930C4BFF7C
:1077D00063F04703B2455A85EFF05F8519CD032763
:1077E0008B00104719CA10436380C4023107D5BF0C
:1077F000EE856685EFF07F9D71FD93861A0093FA02
:10780000F60F130B0B0255B7835644005C43E3EDB0
:10781000F6F622853AC6EF10603DA1679387D7043C
:107820002A8A035D4400324763E897008347D90002
:1078300093E707F8A306F9001C4766852286E285D0
:107840008297C1670844FD17337AFA00529508C041
:107850002312A40115BF97E7FF1F9387672F984353
:10786000814715C31447814763FFD50093974500AF
:107870004C47BE9519C903C7550081476375E6009B
:10788000DC451606B2973E85828003C745008147D6
:10789000E37BE6FE16069C45F5B7EFA26FC8AA8902
:1078A0002E8A814497EAFF1F938A8A2A83A70A00B7
:1078B000984763E4E4006FA0EFC9DC4713944400E9
:1078C00001493E9413BB140083474400634BF90005
:1078D000014913BB140083475400634FF90085042A
:1078E000F1B70844931759005287DA860146A285FA
:1078F0003E9582990509C9BF48449317590052879C
:10790000DA860546A2853E9582990509E9B7EFA278
:10791000CFC2814517F5FFFF1305255F97E7FF1FCE
:10792000239A0722EFF07FF76FA06FC397E7FF1F3F
:10793000938707229C4381CFEFA22FC0814517F583
:10794000FFFF1305855CEFF05FF56FA04FC18280EC
:10795000EFA20FBD37E404008327841241112315E1
:10796000E100AE893289368A3A8681460147ED4583
:10797000AA8482972AC621C50356A100D285EF109A
:1079800061258327C413CE8526858297058915C571
:107990008327440D2314210101462C00268582975C
:1079A0002A8401C9B7E7040083A7C712ED45280060
:1079B0008297228541016FA0EFB94944E5B765542C
:1079C000CDBF5C41FD175CC18280EFA20FB7B7E766
:1079D0000400FC5F829795473305F50281450D81D0
:1079E0006FA0EFB7EFA26FB5B7E70400FC5F829717
:1079F00095473305F5020D816FA06FB6EFA2EFB387
:107A0000B7E7040083A7870B0355050082976FA093
:107A10000FB5EFA28FB2035505003287AE8617B6B9
:107A2000FF1F0356C66B97E5FF1F93852513EFF0E5
:107A30003FF26FA0CFB2EFA24FB0B7E7040083A729
:107A4000C71782976FA0AFB1EFA22FAFB7E70400BF
:107A500083A7871397E5FF1F9385451082970145FC
:107A60006FA0EFAFEFA26FADB7E7040083A7C71F0A
:107A7000814517B5FF1F0355856282976FA02FAE12
:107A8000EFA2AFABB7E7040083A7871397E5FF1F0B
:107A90009385C50D829701456FA06FACEFA2EFA94A
:107AA000B7E7040083A7C71F814517B5FF1F03551C
:107AB000056582976FA0AFAAEFA22FA82E85EF6071
:107AC0000055EF60900D6FA08FA9EFA20FA7EF6098
:107AD000D0176FA0CFA85C49E1175CC95CC583577C
:107AE0002501A1072319F50083570501A1072318D4
:107AF000F5008280F1473305F50297E7FF1F938772
:107B0000E7089C433E9582808D476317F60603D7AE
:107B10004600854763F2E706EFA22FA2368536843A
:107B20002E89EF10A01D39C183574400931405011D
:107B3000C18063ED97022285EF10401CFD142312D3
:107B400094009307A002630EF5009307B00263014F
:107B5000F50293079002631BF5002285EFC0B07E0B
:107B600031A00146CA852285EF80000F6FA02F9FAC
:107B70002285EF001059DDBF828097E6FF1F9386B4
:107B800026019C42014599CF9843D44217E6FF1F36
:107B90002320E6006396D70097E6FF1F23ACE6FE9E
:107BA0001385C7FE8280EFA24F99E9267144330501
:107BB00085029145EF70606201E565556FA02F9ACF
:107BC00097E7FF1F23A2A7FC752633058502914581
:107BD000EF70A0607DD197E7FF1F23A9A7FA592E68
:107BE00097E7FF1F239CA7F8712697E7FF1F2398AD
:107BF000A7F8974701009387E7B917E7FF1F2323EB
:107C0000F7F897070000938747ED17E7FF1F232931
:107C1000F7F6014565B7EFA24F92AA8517E5FF1F5A
:107C20001305C5F5EF1060216FA06F93EFA2EF90E1
:107C3000EFF07FFEEF10E02197E7FF1F938747F5F6
:107C40009C4381CF1387C7FE09CB83D5C7FF17E5B8
:107C5000FF1F130565F4EFF0403A6FA04F90EFA2BD
:107C6000CF8DEFF09FF119C9834785002A8493F7E0
:107C7000070499E70355E500EFF05FFB6FA02F8E37
:107C80008347C5009304450117E9FF1F130949F015
:107C900085E3832709005CC997E7FF1F23AA97EEB6
:107CA00083274900E1FF97E7FF1F23A597EEF9B768
:107CB000FD172306F5006105EF60E07E8307840071
:107CC00063CB07048347840093E707F82304F40099
:107CD000B7E704009C5F82974205A947418133754D
:107CE000F5028347840093F707FCC98F2304F4004F
:107CF0008347D4003E951C402318A40089CF9843A5
:107D000019CB8347C4005040814585073305F502F0
:107D1000420541810297832709005CC897E7FF1F4E
:107D200023A897E68327490089E797E7FF1F23A346
:107D300097E68347C400B9D38355040117E5FF1FB5
:107D4000130585E5EFF0602B15BFEF921FFF97E756
:107D5000FF1F9387A7099C4701448583858B81EF8B
:107D6000AE84B2853A86EF1020142A8409C5EF103C
:107D7000200B829408CC22856F907FFEEF925FFAF1
:107D800041112E8932C6AA89712C32471306050289
:107D9000CA8697050000938525D617E5FF1F1305B2
:107DA000E5DDEFF09FFA2A8429CD9304C50065260E
:107DB0001946AA852685EF00306885452685EF009F
:107DC0001065174501001305A59A4E9583450500DA
:107DD0002685EF0050685C4831468145A1075CC8A4
:107DE0005CC483572401E1172319F400835704016D
:107DF000E1172318F4001C4C3E85EF901FF7A304F5
:107E00002501228541016F90FFF4EF921FF341118C
:107E1000AA842EC632C4EF100003004DB24522469C
:107E2000834784000CC050C093F7F70393E707041F
:107E30002304F400231804002685EF00707E834796
:107E40009400A9462317A40013D73700050733076A
:107E5000D7029D8B85072306F400A306E40083C7A1
:107E60000401D8488507230FF7FE17E7FF1F130704
:107E700027D25843232A0400930744011DEB17E738
:107E8000FF1F2329F7D017E7FF1F2323F7D017E49D
:107E9000FF1F130464D02285EFF0A00B1C44858BD8
:107EA0005D8D09E581452285EFF0201541016F9038
:107EB0001FEB1CC317E7FF1F232EF7CCC9BFEF92A0
:107EC000DFE797050000938565C40145EFF0DFBE4D
:107ED00001456F90DFE8EF925FE6EFF01FBF6F9014
:107EE0001FE88347C500A1E7EF923FE52A840355C9
:107EF000E500EFF05FD215C98347840093F7F7FBE5
:107F00002304F4001C4091C7DC4381C74C40014569
:107F10008297EFF09FC617E5FF1F1305E5C7EFF047
:107F2000400F0355E400EFF07FD06F905FE3828055
:107F3000EF92BFE097E7FF1F938787C59705000083
:107F4000938525D217E5FF1F130505C523A007005C
:107F500023A20700EFE0507E6F907FE01C4D91CB95
:107F6000DC4381CBEF927FDD8345070082976F90E2
:107F70001FDF828097E7FF1F938747C49C4303C599
:107F80000700828097E7FF1F938747C39C4303C581
:107F90001700828097E7FF1F938747C29C4303C562
:107FA0002700828097E7FF1F938747C19C4303C543
:107FB0004700828097E7FF1F938747C09C4303C514
:107FC0003700828097E7FF1F938747BF9C4303C515
:107FD0005700828097E7FF1F938747BE9C4303C5E6
:107FE0006700828097E7FF1F938747BD9C4303C5C7
:107FF0007700828097E7FF1F938747BC9C4303C5A8
:108000008700828097E7FF1F938747BB9C4303C588
:108010009700828097E7FF1F938747BA9C4303C569
:10802000A700828097E7FF1F938747B99C4303C54A
:10803000B70011E11D45828097E7FF1F938707B8BE
:108040009C4303C5C700828097E7FF1F938707B74C
:108050009C4303C5D700828097E7FF1F938707B62D
:108060009C4303C5E700828097E7FF1F938707B50E
:108070009C4303D50701828097E7FF1F938707B4CE
:108080009C4303C52701828097E7FF1F938707B3AF
:108090009C4303D54701828097E7FF1F938707B270
:1080A0009C4303D56701828097E7FF1F938707B141
:1080B0009C4303D58701828097E7FF1F938707B012
:1080C0009C4303C5A701828097E7FF1F938707AFF3
:1080D0009C4303C5B701828097E7FF1F938707AED4
:1080E0009C4303C5C701828097E7FF1F938707ADB5
:1080F0009C4303C5D701828097E7FF1F938707AC96
:108100009C438857828097E7FF1F938727AB9C4348
:1081100003D5C702828097E7FF1F938727AA9C4356
:1081200003D5E70219E11305800C828097E7FF1F52
:108130009387C7A89C4303C50703828097E7FF1F67
:108140009387C7A79C43C85B828097E7FF1F9387ED
:1081500067A68843828097E7FF1F9387E7A5884338
:10816000828019E17D558280F5DE984265DFFDD978
:1081700017E7FF1F130787C71847AA877155058B95
:108180006319072203C507001547E37DA7FC03C752
:1081900037001305F0057D171377F70FE364E5FC4F
:1081A00003C35700E30003FC83C86700E38C08FAAD
:1081B00003C77700494579171377F70FE364E5FAAA
:1081C00003C7A70011481305F7FF1375F50FE36BFD
:1081D000A8F803CE97000D481305FEFF1375F50FA1
:1081E000E362A8F803C8B7006309080065181378AC
:1081F000F80F1305600DE36705F703C5C70079485D
:1082000079151375F50FE36FA8F403C8D7000D4572
:108210007D181378F80FE36705F503D80701930E6F
:1082200040175118420813580801E3ED0EF303C834
:10823000E7007D181378F80FE36605F303C82701FC
:108240007D181378F80FE36F05F103C88700C54E5A
:1082500075181378F80FE3E70EF103D86701856E00
:10826000938EBEE06D18420813580801E3EC0EEF40
:1082700003D847016D18420813580801E3E40EEFD4
:1082800003D887017918420813580801E36C05EDFB
:1082900003C8A7017D181378F80FE36505ED03C542
:1082A000B7011D487D151375F50FE36DA8EA03C5E9
:1082B000D701714879151375F50FE365A8EA03D561
:1082C000E7011308E00F7D1542054181E36CA8E842
:1082D00003C50702494879151375F50FE364A8E84B
:1082E000C85301C937C834005915130858BFE36B88
:1082F000A8E603A8870237C53400130555BF5918EF
:10830000E36205E717E5FF1F2328C58A03C60501B9
:1083100017E5FF1F2324F58A0545E375C5E403D857
:108320002501D04933760603E31E06E203C6150194
:10833000E30A06E217E6FF1F232EB68683C5270051
:1083400001466387A50003C61700F1453306B60250
:1083500083C707039305C00272971A071307C7055F
:1083600016031A9796084697B387B70241553E976A
:10837000329742074183636EE802EF921F9C368575
:10838000EF60D06FEFD0B0212A84EF80B01D2A9427
:10839000EFC090252A94EF7040072A94EFF0BF8039
:1083A0002A94EF2050632A94EF50406622956F90F4
:1083B0001F9B8280EF927F984111A307A100EF805D
:1083C000801E9305F10017050000130565B9EFF055
:1083D000CFCC014541016F909F98EF929F9317E496
:1083E000FF1F1304A4A00328840079599368180080
:1083F00097E4FF1F23A014A113781800631E080040
:10840000BA84BE89368B328A2E89AA8AEFE01FD6BB
:108410007D15269509E531594A856F901F93EFE048
:10842000FFD47D152695A167E357F5FE97E7FF1F5B
:108430009387C7D298433E8C814B11C70145EFC04B
:10844000B03E933B15004A85DA865686D285EF709A
:1084500070372A8911CD1C44F99B17E7FF1F232B86
:10846000F79883270C00CDDBE3880BFA82976DB772
:10847000268597E7FF1F23AD0796EFE0FFCB414628
:10848000CE8517E5FF1F1305E59FEF00A174EFA050
:1084900070080325040BEFA0700A0545EFA07010CB
:1084A0000545EFF03FF18DBF97E7FF1F93870794D6
:1084B0009C47858BD5C7EF925F8817E5FF1F130593
:1084C000A59A97E7FF1F23A3079297E7FF1F23A112
:1084D000079297E7FF1F23AF0790EFE09033EF403D
:1084E000C002EFE0F00AEFE0700F97E7FF1F9387FD
:1084F000678E9C4381C70545EF60B03397D7FF1F58
:10850000938707779C4389C741657D15EF50A06B22
:10851000EFC0703AEFA0F00097E7FF1F938707A224
:108520009C431397170163540700EFC0A04597E7DA
:10853000FF1F23A9079497E7FF1F23A7079497E737
:10854000FF1F23A5079497E7FF1F23A30794EFF0CE
:108550009F984923EFF0AFBBEFC080676F903F80DB
:10856000828097E7FF1F9387678888438280EF9216
:10857000CFFCEF60B07EEF7080006F904FFEEF9207
:108580002FFA2A849304140201112E85B289A6853C
:10859000214636C63A89EF0081611DE1B2463808AE
:1085A0002686CE8513059404EF40604321462C08AF
:1085B0004A85EF00C15F1335150005616F908FF993
:1085C0000145E5BFEF926FF79305450617D5FF1FED
:1085D0001305055FEFE070226F906FF8EF92EFF5F3
:1085E00041112EC6EFF00FC0B24588C141016F9016
:1085F0000FF7EF92EFF2AA842E84EF605078AA89E9
:1086000085452285892D83C7E4011389940899E360
:1086100013890403CE8522853D2D21469305190239
:108620002285192D97D7FF1F9387477C8C4322857E
:10863000EF00E0682146938584022285F52B6F9038
:108640006FF1EF920FED3971EFC0E04E93054006E8
:1086500045EDEF60D06F630E051097D7FF1F83C7FE
:10866000E75713B7170097D6FF1F2389E656014433
:1086700089CFC16417D9FF1F130949779309400EA9
:10868000FD14EFF03F986348A408EFF0AFB54169DF
:10869000B7290900096AFD7A2A8B81447D199389DB
:1086A000F97B130A0A71938A8AC7EFF0BF9563D5E5
:1086B000A4041304400EB387840217D7FF1F1307C7
:1086C000E7720324070B3E948357C401638627098E
:1086D00018403307EB4063EAE9008347440085070D
:1086E000B3874703D6976369F70601468145094575
:1086F000EFF0CFE8AA8B29E1EF20105A8547631FDE
:10870000F50489659385057117D5FF1F1305454B42
:10871000EFE0B00EA1A8B30734030327090BBA9703
:1087200003D7C7016308970003C75700A382070058
:108730002382E7000504B1B79305C5002285EFF059
:108740005FEB5E852286973501009385A503EFF0E8
:10875000CFEB5E85EF00E06F850481BF97D7FF1FE9
:108760009387C7689C478D83858BC1FF21616F907C
:10877000CFDD01468545094502D002D202D402D69A
:10878000EFF0CFDFAA847DD1EFC0203A1389C40077
:108790002A8481454A85C1210C4041464A85692980
:1087A00083294400638809084E8502D802DA02DC76
:1087B00002DEEF00816A2ACE141005462C08081844
:1087C0004ECCEF4060191375F50F2DE583558400ED
:1087D00093E525004A856D2911460C104A85A92983
:1087E000014697350100938565FA2685EFF0EFE1A4
:1087F0002685EF0000665C40B5DB014685450D45EA
:10880000EFF0CFD7AA843DD148401389C400EF00D0
:10881000C1642AC64A85C5263246636AC5004C40F3
:108820004A851929014681452685EFF00FDE268508
:108830000D252DBF8355840071BFEF920FD097D7C0
:10884000FF1F9387A75A9C4719CD93E7870017D539
:10885000FF1F1305E53617D7FF1F232DF758EFE04D
:1088600060786F90CFCFDD9B17D7FF1F2324F75879
:10887000EF2090427DF517D5FF1F13056534EFE01B
:108880004079C5B7EF92EFC84169AA892E8AB28AAA
:10889000368BBA8B814417DCFF1F130C2C55930CBD
:1088A000400E7D19EFF00FF663C4A40001442DA023
:1088B0003384940383270C0B3E948357C401638055
:1088C00027055A87D6865286CE8513050403EFF016
:1088D0001FCB11C523800B0022856F900FC78347E4
:1088E000F40191CF5A87D6865286CE851305940817
:1088F000EFF0FFC809C585472380FB00F1BF850461
:1089000055B783574500638D0716EF926FC101116C
:108910002A84ED2619C58547630AF50405616F9021
:108920006FC3EFC040217DF9835744004947ED9B59
:10893000E396E7FEC14522854524AA842285F52ECB
:108940000357440002CE91472A896317F700228516
:1089500039293C082ACC3ECEEFC0201D5C55DDDF16
:1089600074084A86A685054582974DBF0357440083
:10897000D147E3F5E7FA032A0400C169014997DA10
:10898000FF1F938AAA46130B400EFD19EFF08FE7E5
:108990006344A90C2285032A04008D26A1452A8957
:1089A00022851D2CAA842285D92614402A86AA89CC
:1089B00078082685CA85EFF0FFECAA8425D103C785
:1089C000F40189476315F7008347C101A1DB5546D0
:1089D000D28513856400EF00E11F0145EF60103878
:1089E00001C583D7C401B1EB97D7FF1F9387074019
:1089F0009C4793551900858913D73700058B11CBF8
:108A00008983858B6397B70001452EC6EFF0FFE29F
:108A1000B2454E85EF60703C0346C1012A849375D0
:108A200019002685EF70703131C92685EF607037E7
:108A3000268511C00145EF60D061EF20F025854704
:108A4000E31EF5EC83C754001307F00FE388E7EC4F
:108A50008507A382F400D9B5B304690383A70A0B81
:108A6000BE9483D7C401638937015546D2851385E7
:108A70006400EF00C11371D1050909BF5DDC5DBF62
:108A80008280EF92EFA9EF60902C11CDC164014478
:108A900017D9FF1F130989359309400EFD14EFF014
:108AA0006FD6634AA40017D5FF1F13056511EFE0C9
:108AB00060536F902FAA330534038327090B3E952B
:108AC0008357C5016386970023120500EF60702D60
:108AD0000504F1B797D7FF1F938747319C478D83D4
:108AE000858B99EBEF926FA517D5FF1F1305450DE9
:108AF000EFE020526F90AFA68280EF920FA497050F
:108B00000000938545B417D5FF1F1305650BEFE0F3
:108B1000A0426F90CFA4EF924FA28841B7E7040024
:108B2000BC5B050542054181829709C58547230045
:108B3000F50005056F90AFA283C7F5FF2E85850769
:108B4000A38FF5FE828083C7F5FFFD1793F7F70F1C
:108B5000A38FF5FE99EBEF924F9EB7E70400BC5749
:108B60001385F5FF82976F908F9F82801C4103577A
:108B700045008D8FBA951CC12312B5003E858280B9
:108B800093D78500A2051441DD8D835745001387D7
:108B9000E6FF18C189072312F50013D6850041119D
:108BA000238FB6FEA38FC6FE410182801841930732
:108BB000F7FF1CC18357450085072312F500A30F5B
:108BC000B7FE8280835745008D8F2312F5001C412C
:108BD000BE950CC12E858280AA8703D74700084125
:108BE0000D8FAA952392E7008CC382801841084517
:108BF0003305A740828083574500035765001D8FCA
:108C00001C4108453385A7403305A7408280EF9279
:108C1000CF9241112EC62A84EFF0FFFDB245637357
:108C2000B50001A0835744000840BE952312B4004C
:108C30003E9541016F90AF92EF922F9041112E849B
:108C4000B28532C6EFF0BFFC3246A285EFF09078D5
:108C500041016F90CF90EF924F8E2E848545EFF0BB
:108C60001FFB230085006F908F8FEF920F8D4111B6
:108C70002317B1008945EFF09FF98347E1002300F6
:108C8000F5008347F100A300F50041016F902F8D9F
:108C9000EF92AF8A93D78500A2054111DD8D23178E
:108CA000B1008945EFF0BFF68347E1002300F500EE
:108CB0008347F100A300F50041016F904F8AEF92C6
:108CC000CF871397850193D78501C166938606F0F8
:108CD000D98F13D78500758FD98FA2053707FF006D
:108CE000F98D4111DD8D2EC69145EFF05FF26C00DC
:108CF0001146EFF0306E41016F906F86EF92EF8377
:108D00001C41854503C40700EFF0DFEB22856F901F
:108D10000F85EF928F821C414111894503C70700DF
:108D200083C717002307E100A307F100EFF09FE9D5
:108D30000355E10041016F908F82EF920F801C413B
:108D40004111894503C7070083C717002307E100C6
:108D5000A307F100EFF01FE78357E100410113D5AE
:108D60008700A2075D8D420541816F805FFFEF8222
:108D7000DFFC0C4141112A8411466800EFF0906538
:108D800091452285EFF01FE4B247C166938606F055
:108D90001397870113D58701598D13D78700758FD6
:108DA000598DA2073707FF00F98F5D8D41016F8054
:108DB0001FFB1C45BE950CC18280AE87944391E693
:108DC000584101EF0CC15CC1828003C75700136793
:108DD0001700A382E700B687D5B70CC3EDB7AA8703
:108DE000084119CD1841D44398C36313D500D8C3A3
:108DF0002A87034657009376160081E62320070052
:108E00008280944381CA8C4203A847008CC3639339
:108E10000601CCC3799A14C3A302C7003687D1BF19
:108E20001C45DC471D8DB777DBB6938777DB09855B
:108E30003305F502420541818280F147B385F50291
:108E400048452E9582808347450085072302F5001B
:108E50008280EF829FEE2A8419E06F805FF0834763
:108E60004400E5DFFD1793F7F70F2302F400F5F751
:108E70001C4403D7270005072391E700DC4399C36F
:108E8000228582974C4889CD83475400898B99E786
:108E90001C4422859C479C439C478297232A0400BC
:108EA0000040232004004DBFEF823FE98357250097
:108EB00041112EC691E70144228541016F803FEAAE
:108EC000035705008147F146E307F7FEB385D70254
:108ED000404585072E948345440008C4F5F5B24704
:108EE000AA8481E7232A040009A81C456C00228576
:108EF0009C439C43829748C85DDD85472312F4005C
:108F0000B24723200400231804002319F4005C480E
:108F10005CC483D72400FD172391F40071BFEF8256
:108F2000DFE197D7FF1F9387A7CB88432326050050
:108F3000232405004105EFE0C00D6F805FE2EF8262
:108F4000DFDF17D4FF1F1304A4C91C40411189CFD0
:108F50009C472300B5002AC65CC1EFF05FFC1C40B3
:108F6000DC4399C33245829741016F805FDF03473D
:108F700045001DEB584DAA877D550DCBEF82FFDBD9
:108F80001CC3DC4797D6FF1F23ACE6C4F15613057C
:108F900007012390D7009705000093858501EFD046
:108FA000B07901456F80BFDB7D5582808280EF8282
:108FB000DFD80111614681452800EF801FDB97D77C
:108FC000FF1F9387E7C19C4328009305F00FDC4700
:108FD0003EC6EFF0DFF605616F807FD897D7FF1FA1
:108FE000938707C09C43D847A1679387C702631242
:108FF000F70A397106DE22DC26DA80004AD84ED61E
:1090000052D456D23285B284EFF05FCFAA8926853A
:10901000EFF03FD02318A4FC2685EFF09FCF231953
:10902000A4FC2685EFF0FFCE83D744000A8A231ADA
:10903000A4FC858393F7F70F230EF4FC8607BD0786
:1090400093F7073F3301F1408A8A01498347C4FD02
:109050006365F902CE85130584FC232C54FDEFF0E3
:109060001FEE5281130104FCF2506254D254425953
:10907000B259225A925A216182802685EFF07FC927
:1090800093171900D69705092390A7001379F90FB4
:1090900075BF828097D7FF1F938787B49C43D847BB
:1090A000A1679387A7026310F70A397106DE22DCF5
:1090B00026DA80004AD84ED652D456D23285B284AF
:1090C000EFF0DFC3AA892685EFF0BFC4FD57231850
:1090D000A4FC26852319F4FCEFF0BFC383D744001A
:1090E0000A8A231AA4FC858393F7F70F230EF4FC56
:1090F0008607BD0793F7073F3301F1408A8A01498C
:109100008347C4FD6365F902CE85130584FC232CD7
:1091100054FDEFF0DFE25281130104FCF25062547F
:10912000D2544259B259225A925A216182802685DC
:10913000EFF03FBE93171900D69705092390A700BB
:109140001379F90F75BF828097D7FF1F938747A9BF
:109150009C43D847A16789076318F708397106DE71
:1091600022DC26DA80004AD84ED652D456D2328536
:109170003289EFF0BFB8AA894A85EFF09FB98357CB
:1091800049000A8A2318A4FC858393F7F70F230C60
:10919000F4FC8607BD0793F7073F3301F1408A8A45
:1091A0008144834784FD63E5F402CE85130584FC86
:1091B000232A54FDEFF0BFD85281130104FCF25072
:1091C0006254D2544259B259225A925A2161828031
:1091D0004A85EFF01FB493971400D6978504239027
:1091E000A70093F4F40F75BF828097D7FF1F938772
:1091F000279F9C43D847A1679387E7046312F70A28
:10920000397106DE22DC26DA80004AD84ED652D4E6
:1092100056D23285B284EFF07FAEAA892685EFF070
:109220005FAF2318A4FC2685EFF0BFAE231AA4FC81
:109230002685EFF01FAE83D744000A8A2319A4FCC9
:10924000858393F7F70F230EF4FC8607BD0793F78A
:10925000073F3301F1408A8A01498347C4FD6365B2
:10926000F902CE85130584FC232C54FDEFF03FCD8D
:109270005281130104FCF2506254D2544259B25943
:10928000225A925A216182802685EFF09FA8931777
:109290001900D69705092390A7001379F90F75BF18
:1092A000828097D7FF1F9387A7939C43D847A167D6
:1092B0009387C7046310F70A397106DE22DC26DAC9
:1092C00080004AD84ED652D456D23285B284EFF0BE
:1092D000FFA2AA892685EFF0DFA3FD572318A4FC7F
:1092E0002685231AF4FCEFF0DFA283D744000A8A14
:1092F0002319A4FC858393F7F70F230EF4FC86074C
:10930000BD0793F7073F3301F1408A8A014983473C
:10931000C4FD6365F902CE85130584FC232C54FD3E
:10932000EFF0FFC15281130104FCF2506254D25499
:109330004259B259225A925A216182802685EFF011
:109340005F9D93171900D69705092390A7001379FD
:10935000F90F75BF828097D7FF1F938767889C435B
:10936000D847A167DD07631BF702EF821F9D797164
:1093700032853284EFF09F982AC62285EFF07F99DC
:109380002311A1022285EFF07F97B2452300A102AD
:109390002808EFF0DFBA45616F807F9C828097D705
:1093A000FF1F9387E7839C43D847A1679387870470
:1093B000631BF702EF827F98797132853284EFF078
:1093C000FF932AC62285EFF0DF942311A1022285A4
:1093D000EFF0DF92B2452300A1022808EFF03FB67C
:1093E00045616F80DF97828097C7FF1F9387477F14
:1093F0009C43D847A1679387A704631CF700EF82BB
:10940000DF93011128008145EFF07FB305616F8084
:109410001F95828097C7FF1F9387877C9C43D847FF
:10942000A167938757026311F702EF821F91011121
:109430003285EFF0BF8C2308A10081452800EFF0B2
:109440001FB005616F80BF91828097C7FF1F938710
:1094500027799C43D847A1679387E702631FF702E8
:10946000EF82BF8D011132853284EFF09F8AAA848A
:109470002285EFF01F8A854719E52285EFF01F88C6
:109480004205B337A00028008145231891003ECA49
:10949000EFF0FFAA05616F809F8C828097C7FF1F46
:1094A000938707749C43D8479947631FF704EF825B
:1094B000DF88797132853284EFF05F842AC6228595
:1094C000EFF03F852310A1022285EFF03F832301B7
:1094D000A1022285EFF09F82A301A1022285EFF075
:1094E000FF812302A1022285EFF05F812313A102F5
:1094F0002285EFF0BF80B2452314A1022808EFF0C7
:109500001FA445616F80BF85828097C7FF1F938727
:10951000276D9C43D847A1679387C703631FF70450
:10952000EF82BF81797132853284EFF02FFD2AC638
:109530002285EFF00FFE2310A1022285EFF06FFDD0
:109540002311A1022285EFF06FFB2302A1022285E5
:10955000EFF0CFFAA302A1022285EFF02FFA230346
:10956000A1022285EFF08FF9B245A303A1022808DA
:10957000EFF0FF9C45616F808FFE8280EF82EFFBF2
:1095800001112A84EFF08FF7AA842285EFF06FF89B
:109590002285EFF00FF8035744008D4763F5E7008D
:1095A0002285EFF00FF72285EFF0AFF62800A685B1
:1095B000EFF0FF9805616F808FFA97C7FF1F9387C1
:1095C00027629C43D847A167FD076319F700EF8224
:1095D000CFF63285EFF09FFA6F806FF8828097C7E1
:1095E000FF1F9387E75F9C43D847A167E507631197
:1095F000F706EF828FF4797132853284EFF00FF045
:109600002AC62285EFF0EFF02285EFF08FF02310CD
:10961000A1022285EFF0EFEF520551812311A10243
:10962000228523020102EFF06FEDA302A102228541
:10963000EFF0CFEC2303A1022285EFF02FECB2452F
:10964000A303A1022808EFF09F8F45616F802FF1DF
:10965000828097C7FF1F9387A7589C43D847A1676D
:109660009387E7036319F700EF822FED3285EFF060
:10967000FFF06F80CFEE828097C7FF1F938747561A
:109680009C43D847A167938747046314F702EF828E
:10969000CFEA797132853284EFF04FE62AC622850F
:1096A000EFF02FE7B2452808EFF07F8945616F8022
:1096B0000FEB828097C7FF1F938787529C43D84741
:1096C000A167938787026316F702EF820FE779712C
:1096D00032853284EFF08FE22AC62285EFF00FE266
:1096E000B2452300A1022808EFF07F8545616F8015
:1096F0000FE78280EF826FE40111EFF02FE0AA857F
:109700002800EFF0DF8305616F806FE597C7FF1FCB
:109710009387074D9C43D847A167D1076319F7008A
:10972000EF82AFE13285EFF0FFFC6F804FE3828084
:1097300097C7FF1F9387C74A9C43D847A167C507B0
:109740006319F700EF826FDF3285EFF0BFFA6F80A9
:109750000FE1828097C7FF1F938787489C43D847B4
:10976000A167B9076319F700EF822FDD3285EFF0AB
:109770007FF86F80CFDE828097C7FF1F93874746B1
:109780009C43D847A167AD076319F700EF82EFDA72
:109790003285EFF03FF66F808FDC828097C7FF1F26
:1097A000938707449C43D84789476310F702EF82A9
:1097B000CFD80111328532C8EFF04FD4AA852800E6
:1097C000EFF0EFF705616F808FD9828097C7FF1F99
:1097D000938707419C43D847A1678D076317F7021A
:1097E000EF82AFD5011132853284EFF02FD113060D
:1097F0006100AA844C002285EF20D00C2800A685A9
:10980000EFF0EFF305616F808FD5828097C7FF1F60
:109810009387473D9C4381CBDC4391C7EF82EFD1D7
:1098200082976F80CFD38280EF822FD179713C08ED
:10983000AE843ED2A165B7070A002A843ED4481000
:109840003C08DD053ED636C432C63AC2EFD0BFAAC8
:1098500012474810BA85EFF00FC032464810B28563
:10986000EFF0AFC0A2464810B685EFF0CFBE501063
:1098700001478146A6852285EFD07FC845616F806C
:109880000FCEEF828FCB01117C000329C501AE847E
:109890003ECAA165B70707002A843ECC48087C0071
:1098A000C5053ECEEFD03FA58345D9004808EFF06F
:1098B0008FBA500801478146A6852285EFD03FC464
:1098C00005616F80CFC9EF824FC783C7950093F7BB
:1098D000F707A384F500EFF0DFFA6F804FC8EF823F
:1098E000CFC579713C08AE843ED2A165B7070900A7
:1098F0002A843ED448103C08938545043ED632C69F
:1099000036C4EFD05F9FA2464810B685EFF0AFB4E3
:1099100032464810B285EFF04FB5501001478146EE
:10992000A6852285EFD0BFBD45616F804FC3EF8212
:10993000CFC083C7950041112A8493F7F707A3840A
:10994000F50032852EC6EFF0CFBC85672AC4637C54
:10995000F500EF50B0402246B24509E91147814673
:109960002285EFF07FEC41016F806FBF0147834696
:10997000F501FDB7EF82CFBA01113C003ECAB7072F
:109980000A003ECC3C003ECE83C79500AA893285B2
:1099900093F7F707A384F5002E84EFF08FB7856760
:1099A0006371F504A165AA84938585044808EFD006
:1099B0009F942685EF50903A2A891DE591454808E5
:1099C000EFF06FA9A6854808EFF02FAACA854808CE
:1099D000EFF06FA8014781465008A2854E85EFD071
:1099E0001FB205616F800FB781454808EFF0AFA641
:1099F00003490902C1BFEF82AFB279711C103ECAA0
:109A0000B7070F003ECC404D1C10AA84AE89480811
:109A1000994532C636893ECEEFD0FF8D3246480892
:109A2000B285EFF04FA363040902A5454808EFF0A3
:109A30000F9E2546CA85EFF0E01950080147814680
:109A4000CE852685EFD0BFAB45616F80AFB0835523
:109A5000C4024808EFF06FA10355E402814515C127
:109A600085478545630FF500C167FD179305F00F26
:109A70006309F5007D15EF5020749305150093F5EB
:109A8000F50F4808EFF02F9D834504034808EFF0D9
:109A90008F9C834514034808EFF0EF9B8355240304
:109AA0004808EFF08F9C835544034808EFF0EF9B84
:109AB00069B7EF828FA883C795008146014693F767
:109AC000F707A384F500EFF01FF36F804FA9EF8233
:109AD000CFA679713E841C103ECA2E89B7070F00AD
:109AE000A1653ECCFD051C10AA84480842C03AC2BC
:109AF0003ECE36C432C6EFD01F8032464808B2850B
:109B0000EFF06F95A2464808B685EFF00F96124722
:109B10004808BA85EFF06F95024863040802914542
:109B20004808EFF0CF8E1146A285EFF0A00A50084A
:109B300001478146CA852685EFD07F9C45616F80AD
:109B40000FA289454808EFF08F8C8347040023005B
:109B5000F50083471400A300F500D1BFEF824F9CAE
:109B600083C7950001112A8A93F7F707A384F500AC
:109B70003285AE8432C6EFF0CF9932462A893285DB
:109B8000EFF0CF978567637FF900AA894A85EF5088
:109B9000F01C2A8419E9114781464A86A685528518
:109BA000EFF09FC805616F80EF9A9387E9FF93F705
:109BB000F70F0547E368F7FE8347F50195E7894707
:109BC000E382F9FE8346F401528501474A86A68561
:109BD000EFF09FC5A167D90748083ECC230A0100D2
:109BE00002CEEFF0BFC27DBF639CE7008947639C54
:109BF000F90093071020231FF500EF50901AD9B7F2
:109C00000947E391E7FC8D47E39EF9FA2285EF507F
:109C1000D03B97C7FF1F9387E71B9C4399E797C7E4
:109C2000FF1F9387E7049C4389C703D50400EF60B7
:109C3000300C231F04002285C9B7EF820F90011159
:109C40003C003ECAB7070B003ECC3C003ECE83C76B
:109C500095002A89328593F7F707A384F500AE842F
:109C6000EFF02F8B93170501C187635EF004A165A8
:109C70002A849385E5024808EFD0EFE7A2854808DB
:109C8000EFE0BFFE97C7FF1F938787FE9C439DEFC2
:109C900001449375F40F4808EFE0FFFB93558440AF
:109CA00093F5F50F4808EFE01FFB9355044193F53A
:109CB000F50F4808EFE03FFA014781465008A685B6
:109CC0004A85EFD0DF8305616F806F8941658546E6
:109CD0000546A2857D15EF3070675DD95105EFD03F
:109CE0004027130440063344850265B7EF82EF84B2
:109CF0000111B70706003EC683C7950021642A8973
:109D000093F7F707A384F500AE8428009305A40415
:109D10000AC40AC8EFD02FDE300001478146A6856D
:109D20004A85EFD0CFFDEFE02FF8130494044808E4
:109D300022CC230A010002CEEFF05FAD05616F80F7
:109D40000F82EF72FFFDC1642A89014497C9FF1F8A
:109D50009389C909130A8002FD14EFE0AFAB634594
:109D6000A40001456F701FFFB307440303A7C90A8E
:109D7000BA9703D707006306970083D72700638449
:109D800027010504D9BF0545F1BFEF727FF92A8A83
:109D90002E8999C123A005008149814497CAFF1FDC
:109DA000938A8AE4614BEFE02FAD63C5A4004E8532
:109DB0006F705FFA3384640383A70A003E9483576D
:109DC000040099E763040900232089008504E1BFAA
:109DD0004146D28513054400EFE0705D65F9A28924
:109DE000F5B7EF72FFF339717C083ED4B7070A006C
:109DF0003ED67C083ED883C795002A8A328593F7E1
:109E0000F707A384F5002E8932C6EFE09FF085673F
:109E10006373F5063246AA843285EFE03FEE85474C
:109E2000AA8963EAA704A165938585042810EFD069
:109E30008FCC2685EF5080722A8429E19145281025
:109E4000EFE07FE1A6852810EFE03FE2CE85281005
:109E5000EFE07FE0014781463010CA855285EFD0A0
:109E60000FEAA1679387770448183EDC230A0102B2
:109E700002DEEFF0BF9921616F70DFED81452810A0
:109E8000EFE07FDDA6852810EFE03FDE97C7FF1FDC
:109E90009387872C9C4391C7228563870900EFB085
:109EA000600C8345040265B7EFB0200BDDBFEF7295
:109EB0003FE783C795004111AA8993F7F707A38469
:109EC000F5003285AE84328AEFE0BFE48567637BBC
:109ED000F5022A89EF5080682A84914621C1834780
:109EE000F50105476383E70291C70D47636EF702EB
:109EF000AD462DA09305050303250A004146EFE07A
:109F0000104B1DE141016F70FFE493059508032597
:109F10000A004146EFE0B049814679F94A86A685B4
:109F20004E85EFF0DF9BF9BF83250A0013059408E7
:109F3000EF60600119C1C146D5B797C7FF1F93876E
:109F400067E99C4399E797C7FF1F938767D29C43B4
:109F500089C72285EF60A05479FD8547A30FF400DF
:109F60002285EF80B05D2285EF50A0634E8581464B
:109F70004A86A685EFF0BF96A167938757044800ED
:109F80003EC42302010002C6EFF05F88A5BFEF7256
:109F90005FD883C795004111AA8993F7F707A38477
:109FA000F50032852E89B28AEFE0BFD685676370EF
:109FB000F50CAA84EF50805A2A841DE9416B014AAE
:109FC00097CBFF1F938B8BE2130C400E7D1B19A8C0
:109FD00033048A0383A70B0B3E948357C401638D1C
:109FE0006703050AEFE00F82E344AAFE954639A80D
:109FF0008357C501639297029305050303A50A00E1
:10A000004146EFE0D03A994611E181462686CA855D
:10A010004E85EFF0DF8CA1A883A50A001305040389
:10A02000EF507072C1467DF12285231E9400EF80AF
:10A03000F0502285EF50E05697C7FF1F9387C71156
:10A040009C438DCB230004022285EFA090614E85B6
:10A0500081462686CA85EFF09F88A167938707040B
:10A0600048003EC42302010002C6EFF02FFA41016E
:10A070006F70BFCD89472300F402D1BF397106DE6E
:10A0800022DC4AD8800052D456D25AD026DA4ED694
:10A090005ECE2E8A32892A8BEFD0DFF3060571055A
:10A0A00041998A8A3301A140232224FC231404FC11
:10A0B000EFD05FF283479A000605350593F7F7075F
:10A0C0002315A4FCA304FA004A85232624FCEFE010
:10A0D0005FC493170501C1876340F00256811301E5
:10A0E00004FCF2506254D2544259B259225A925A44
:10A0F000025BF24B21618280AA844A85EFE07FC136
:10A10000AA894A85EFE0FFC0A1659385C5022A8927
:10A11000130544FCEFD02F9E2685EFD0AF938545E5
:10A1200001C94A86CE85EFD06F8DAA8B15ED894582
:10A13000130544FCEFE03FB2A685130544FCEFE0B5
:10A14000DFB2CE85130544FCEFE03FB2CA851305AC
:10A1500044FCEFE09FB101478146130644FCD285E1
:10A160005A85EFD0CFB99DBF8145130544FCEFE080
:10A170009FAEA685130544FCEFE03FAFCE851305E7
:10A1800044FCEFE09FAECA85130544FCEFE0FFAD51
:10A190008144EFD03FE4E3D0A4FC83A70B011397E5
:10A1A0001400BA9783D5070089C5130544FCEFE076
:10A1B000DFAB8504F9BF797106D622D44AD00018E6
:10A1C0004ECE52CC56CA26D25AC8AE893289AA8AF5
:10A1D000EFD05FE00605690541990A8A3301A14085
:10A1E000232A24FC231C04FCEFD0DFDE83C7990064
:10A1F00006052D0593F7F707231DA4FCA384F9009A
:10A200004A85232E24FCEFE0DFB093170501C187B8
:10A21000634FF0005281130104FDB2502254925456
:10A220000259F249624AD24A424B45618280AA846D
:10A230004A85EFE01FAEA1659385A5022A89130523
:10A2400044FDEFD04F8B2685EFD0CF80854519C5D3
:10A25000CA85EFC0BFFD2A8B0DE98945130544FD72
:10A26000EFE07F9FA685130544FDEFE01FA0CA85A0
:10A27000130544FDEFE07F9F01478146130644FD2F
:10A28000CE855685EFD0AFA771B78145130544FD44
:10A29000EFE07F9CA685130544FDEFE01F9DCA8576
:10A2A000130544FDEFE07F9C8144EFD0BFD2E3D59E
:10A2B000A4FC83270B0113971400BA9783D50700DA
:10A2C00089C5130544FDEFE05F9A8504F9BFEF727D
:10A2D000DFA683474500404DD5E7FD574DC0834677
:10A2E00094000947636DD7080346B400854663E8C8
:10A2F000C6088306E40063C406085C45F95623904B
:10A30000D70097C7FF1F83C7678E99E3A304E400B4
:10A3100097C7FF1F9387C7959C4381E78947A3068B
:10A32000F40097C7FF1F938727E39C4381E7894782
:10A330002306F4009705000093854505AA841305BC
:10A340000401EFC0703FFD57231AF40281471CDC63
:10A35000014897C7FF1F23A7878897C7FF1F9387C9
:10A36000A788232E040304C08043EFD0FFD06146AA
:10A370003306C50281452285EF703F9F81473E85A8
:10A380006F70FF9DFD57E5BFEF723F9B2A84035519
:10A390004502EF50A01C09E5231E04006F703F9C8E
:10A3A0008357E401E5DF930504FF1715010013054A
:10A3B000A577EFB01063DDB7EF723F982E89A165E6
:10A3C00041119385E5032A8436C432C6BE843AC25D
:10A3D000EFC07FF212472285BA85EFE0DF87324671
:10A3E0002285B285EFE07F88A2462285B685EFE020
:10A3F000DF87630D090091452285EFE05F811146FB
:10A40000A685EFE0207D41016F707F95894522850B
:10A41000EFE0EFFF83C704002300F50083C71400BB
:10A42000A300F500CDB7EF725F9183C79500444D4F
:10A43000054793F7F707A384F5001C42411183C732
:10A440000700636DF7042E842A8985CC03C7D400E6
:10A450006309F70217C7FF1F13078781184301CF4E
:10A46000A386F400EF80902B83C7D40089E7416571
:10A470007D15EF30407583D72403918B99C3EFB0DE
:10A48000B0624A85A285EFF0CFBFA167C10748003F
:10A490003EC42302010002C6EFF04FB741016F70C6
:10A4A0001F8CEF729F8903D745008D47AA84411105
:10A4B0002E8432892E8563EDE700EFE09F85AA8523
:10A4C000230009002685EFC07FD641016F703F89C8
:10A4D000EFE03F842AC62285EFE0BF83B24585477F
:10A4E0002A862300F9002685EFC05FD1F9BF3971B4
:10A4F00006DE22DC26DA80004ED652D456D24AD866
:10A500005AD05ECEAE89B284AA8AEFD0BFAB060520
:10A510001305250241990A8A3301A140232224FC14
:10A52000231404FCEFD01FAA83C7990006054D052C
:10A5300093F7F7072315A4FCA384F90026852326A7
:10A5400024FCEFE00FFD93170501C1876340F00283
:10A550005281130104FCF2506254D2544259B25950
:10A56000225A925A025BF24B21618280AA8B03AB82
:10A570000400EFC03FCE35E983D74400014985444C
:10A58000F11793B71700A301F4FC834734FCA165CE
:10A59000BDC79385E504130544FCEFC0DFD5A68550
:10A5A000130544FCEFE02FEBDE85130544FCEFE0E0
:10A5B000CFEB834734FC114691E30946DA85130556
:10A5C00044FCEFE06FE7814463080900416B7D1BA9
:10A5D000EFD05F9F63C8A40201478146130644FC85
:10A5E000CE855685EFC0BFF1A5B7A685130634FC0E
:10A5F000EFF03FEB933415002A89860479B79385F1
:10A60000C50451BF8327C90013971400BA9783D597
:10A61000070063866501130544FCEFE00FE5850440
:10A6200045BFEF720FEF79711C103EC4B7070F00E2
:10A630003EC61C103EC883C79500AA8A328593F790
:10A64000F707A384F500AE893284EFE08FEC93170F
:10A650000501C1876350F0062A8A2285EFE06FEB7F
:10A660002A895285032B0400EFC0DFBE39E58357EA
:10A67000440081440544F11793B71700A303F10088
:10A6800083457100DA872287CA8652862800EFF058
:10A69000BFD2014781463000CE855685EFC03FE6E8
:10A6A000A1679387D70348083ECC230A810026CEB2
:10A6B000EFF0CF9545616F704FE9A28513067100E9
:10A6C000EFF03FDEAA84094445DD3544E30A55FB3B
:10A6D0004A85EFF00FE70D4445D50144EFD09F8E3A
:10A6E000634BA400C16B0144FD1BEFD0BF8D634ED3
:10A6F000A400154471B7DC4413171400BA9783D72C
:10A700000700638127030504D1BFD84493171400C1
:10A71000BA9703D70700631977012390270126858D
:10A72000EF80C0540144A9BF0504C1B7EF724FDFE9
:10A7300083C7950041112A8A93F7F707A384F50090
:10A7400032852E893284EFE0CFDC93170501C18773
:10A75000635BF004AA892285EFE0AFDB2311A1003F
:10A760004E85832A0400EFC0FFAE29E183574400E1
:10A7700085440144F11793B71700A300F100034883
:10A78000110003572100D6875285CE862686CA85BA
:10A79000EFF0EFB3A167F10748003EC42302910038
:10A7A00022C6EFF0AF8641016F70CFDAA2851306A3
:10A7B0001100EFF01FCF2A84894471D18357210003
:10A7C00011678544BA97C2071167C1831307F7EF72
:10A7D000E367F7FA97B7FF1F9387C75F9C4391C75B
:10A7E000854513052100EF40300E83552100228559
:10A7F0008144EFC09F9D41D5231005002285EF8045
:10A800008048B5BFEF72EFD083C7950041112A8B06
:10A8100093F7F707A384F50032852E8A3284EFE0A0
:10A820004FCF93170501C1876359F004AA8A228587
:10A83000EFE02FCE2A895685832B0400EFC09FA11D
:10A8400021E18357440081440544F11793B7170071
:10A85000A301F10003483100DE875A854A87D68676
:10A860002286D285EFF0AFA6A167ED0748003EC46F
:10A870002302810026C6EFE07FF941016F70EFCC23
:10A88000A28513063100EFF0DFC1AA84094479D113
:10A890009167CA97C2071167C1831307F7EF054491
:10A8A000E36AF7FACA85EFC05F92014445F5814932
:10A8B000EFD04FF263DBA900984893971900BA973D
:10A8C00003D7070015E723902701EFD0AFF0154419
:10A8D000E382A9F82685EF80003B97B7FF1F938797
:10A8E000674F9C430144BDD74A85EF4040769DB7F2
:10A8F00085097DBFEF72CFC279713E847C083EC866
:10A900002E8AB7071400A1653ECAE5057C08AA890E
:10A91000080836C4428932C6BA8AC6843ECCEFC023
:10A920009F9DCA850808EFE00FB332460808B2853C
:10A93000EFE0AFB3A246630E09029D450808EFE0C1
:10A940000FAD1D468145EF704FC263870A069145E2
:10A950000808EFE0CFAB1146A685EFE0A02710086E
:10A9600001478146D2854E85EFC07FB945616F7042
:10A970006FBEB6850808EFE04FAF1C400808D8430B
:10A980009355C701858912075183B205D98DEFE030
:10A99000CFAD1C40080883C58700EFE0CFAB1C405B
:10A9A000080883C5A700EFE00FAB1C40080883C56B
:10A9B0009700EFE04FAA51BF89450808EFE02FA5A7
:10A9C00083C704002300F50083C71400A300F5002B
:10A9D00079B7EF72EFB483C795004111AA8993F755
:10A9E000F707A384F5003285AE843284EFE06FB2BE
:10A9F00093170501C1876357F0042A89032A0400CD
:10AA0000EFC05F8519E9835744000548F11793B7F4
:10AA10001700A307F100814621A81306F100A285C3
:10AA2000EFF03FA81DC11C459DC383D647000148D8
:10AA30000347F10093078500D2884A86A6854E8594
:10AA4000EFF05FEB41016F70EFB00948E9B71D48C7
:10AA5000D9B7EF72EFAC65715C083EC4B7077B01F4
:10AA60003EC65C083EC883C795002A8A328593F7A4
:10AA7000F707A384F500AE89EFE04FA88357E10004
:10AA8000C5C389452800EFC01F8781452800EFE036
:10AA90008F9CEFC0FF8B97B7FF1F9387E76B9C439B
:10AAA00017B4FF1F03448414AA843334800099C36D
:10AAB0001364240097B7FF1F9387871B9C4399C398
:10AAC0001364440097B7FF1F9387C7309C4399C313
:10AAD0001364840083D5040028000149EFE0EF9857
:10AAE00083D524002800EFE04F9883D54400280048
:10AAF000EFE0AF97EFD00FC993150501C181280092
:10AB0000EFE0AF96A2852800EFE02F969C44636C9F
:10AB1000F900014781463000CE855285EFC03F9E47
:10AB200059616F702FA3DC441314490028003E9430
:10AB3000EFE06F8C83474400034754008907060702
:10AB4000BA978607E36EF5FC835524002800814AF6
:10AB5000EFE0AF91834544002800EFE0CF8F8345BD
:10AB600054002800EFE02F8F8347440063C9FA00A8
:10AB7000814A8347540063CFFA00050941BF1C4452
:10AB800013975A002800BA9783D50700850AEFE08B
:10AB9000CF8DD9BF032BC40093975A0028003E9B4A
:10ABA00083552B00850AEFE04F8C83550B0028005E
:10ABB000EFE0AF8B7DBFEF724F985C4993E71700D2
:10ABC0005CC9EF8020336F708F99EF720F972E84DE
:10ABD0008145EFF08F9B05C183570500FD172310BA
:10ABE000F50009C4835725002310F400EFF0BFFCE3
:10ABF00001456F70CF9631456DDC23100400D5BF41
:10AC0000EF720F9283C7950041112A8A93F7F707D5
:10AC1000A384F50032852E893284EFE08F8F93175D
:10AC20000501C187635EF004AA89C1452285EFD082
:10AC3000BFFA2A8B4E85832A0400EFC0AFE121E5DD
:10AC400083574400231101000544F11793B71700FF
:10AC5000A300F10081440348110003572100D68767
:10AC60005285CE862286CA85EFE07FE6A16793876C
:10AC7000170248003EC42302810026C6EFE01FB938
:10AC800041016F702F8D13061100A285EFF07F81B7
:10AC9000AA8409E523110100094475BF9305210029
:10ACA0005A85EFF09FF2835721002A84CDD797B7BA
:10ACB000FF1F938727129C4391C7854513052100E9
:10ACC000EF4080408355210026853144EFC0EFCF0F
:10ACD00059D1231005002685EF70F07A0144A5BFF5
:10ACE000EF72AF8541112E896C00AA8402C6EFF085
:10ACF000CF8909CD0357050005072310E500EFF0C4
:10AD00009FEB81473E8541016F706F8532479547C4
:10AD100075DBCA852685EF20D008C147E34405FED0
:10AD20003244854741462310F40083570900A68525
:10AD3000130544002311F400EFD0D0692285C1B778
:10AD4000EF621FFE83C795004111AA8A93F7F707A8
:10AD5000A384F5003285AE893284EFD09FFB931730
:10AD60000501C187635EF0042A8AC1452285EFD0C0
:10AD7000BFE6AA845285032B0400EFC0AFCD21E5C6
:10AD800083574400231101008544F11793B717003E
:10AD9000A300F10001440348110003572100DA87A2
:10ADA0005685D2862686CE85EFE07FD2A16793872F
:10ADB000070248003EC42302910022C6EFE01FA50F
:10ADC00041016F603FF9A28513061100EFF06FEDAE
:10ADD0002A8409E523110100894475BF268593055E
:10ADE0002100EFF0FFEFAA845DF583552100228555
:10ADF000EFC0AFBD4DF10149EFD0CF9D635DA9001C
:10AE0000184893171900BA9703D707001DE703578F
:10AE100021002390E700EFD0EF9B6302250397B753
:10AE2000FF1F938727FB9C4389C703552100EF40F1
:10AE300000222285EF703065B9BF050975BF9544C2
:10AE400099BF05C19307F00F630FF500C547630C69
:10AE5000F5009307F5FF05453315F50042054181DF
:10AE600082800145828041657D158280B9E1EF6273
:10AE7000DFEC034506033284EFF0BFFC9305803E10
:10AE8000B305B502C205C18191C90357E4028547E4
:10AE900063F6E70013050401EFC020168357E402B0
:10AEA00041677D176385E700FD172317F4026F6084
:10AEB0001FEB8280EF62FFE5004283C79500444D9F
:10AEC0000349140093F7F707A384F50083470400B0
:10AED000220911673369F900A167B347F9004111ED
:10AEE0002A8BAE8A63ECE70C834724001307C00E5D
:10AEF000B91793F7F70F6371F70E03473400C14793
:10AF000063ECE70C834744001307E00793C7070887
:10AF10006373F70A8349840083477400A209B3E985
:10AF2000F900856763F9F908034A64008347540010
:10AF30004E85220A336AFA00EF40406245C12396EB
:10AF40002403834B3400137AFA00239A34032388B2
:10AF500074032399440393890401631A090023A607
:10AF60000402239804024E85EFC0A00A1DA00349E5
:10AF700024004A85EFF0FFEC2397A40283474400A6
:10AF80004E85A388F402E3810BFEE30F09FCEFC0BA
:10AF90006005EF70907981460146D6855A85EFE0CD
:10AFA0009FA5A167938797033EC423020100480031
:10AFB00002C6EFE0BF8541016F603FD98544A2869C
:10AFC0002686D6855A85EFE01FA3A167938797034E
:10AFD0003EC423029100E1BFBD44D5B79144C5B73B
:10AFE000EF621FD401111C08404D3EC2B7070F008D
:10AFF0003EC41C083EC62A89AE89EFC01F9D585C1E
:10B000001C5C634CB70A6394E50063E8A70A3385C8
:10B01000A740B3B7A700B305B7401306803E8146EB
:10B020009D8DEFD0407B93140501C180A165938570
:10B03000C5034800EFC02FAC81454800EFD0BFC129
:10B04000835504044800EFD05FC2835524044800B0
:10B05000EFD0BFC1814599C8C167FD179305F00FB7
:10B060006386F4002685EF402015AA854800EFD0BE
:10B070009FBE03554404814511C9C167FD1793055F
:10B08000F00F6305F500EF402013AA854800EFD0CC
:10B090009FBC834564044800EFD0FFBB8345740424
:10B0A0004800EFD05FBB500001478146CE854A85FE
:10B0B000EFC0EFC405616F60FFC9814485BFEF62D7
:10B0C000DFC783C7950093F7F707A384F500EFF078
:10B0D0003FF16F60DFC8EF62BFC483C795004111C5
:10B0E000404D93F7F707A384F5002A8A3285B2848E
:10B0F000AE89EFD01FC22A8B2685EFD09FC12A8947
:10B100002685EFD0BFBF93170B0163CA0702E17713
:10B11000CA97C207C183116763E3E7029307091067
:10B12000C207C1831307B00F637BF70093170901B0
:10B13000C187AA8A6348F000C54763FA57014101F5
:10B140006F605FC1EFC08F83E31B25FFF5B7630618
:10B150000B0263040902814463870A02B7077F0078
:10B1600023106405231124057CC05685EFF07FCDA4
:10B170009304803EB304950239A0B7077F002320D3
:10B1800004047CC0814403552404EFB0101095CC16
:10B19000EFC0BF83269593D7F44133379500AE9720
:10B1A000BA9708DC5CDCCE855285EFF07FE399E04E
:10B1B00023220404A1679387B70348003EC42302F7
:10B1C000010002C6EFE08FE49DBF814701481CDC0F
:10B1D000232E0403C9BFEF625FB6EFC0FFE9E1476A
:10B1E0003305F5029145EF30507FE55711C597B70C
:10B1F000FF1F23ABA79E81473E856F605FB68547E3
:10B2000017B7FF1F2304F79E8280EF621FB397B723
:10B21000FF1F9387279D80432DC083570404639E9F
:10B22000A70483572404639AB7043689B284EFC015
:10B23000CFF95C5C63C3B7046395B7001C5C63EE35
:10B24000A7028347640463F3F400A6872303F4048E
:10B250008347740463F39700A687A303F40483571A
:10B26000440441677D176385E70085072312F404D2
:10B270003C4481C7CA85268582976F605FAE97B7C9
:10B28000FF1F938727969C43014599C303C58700F9
:10B290008280EF629FAA0111B70707003EC683C7ED
:10B2A0009500584D0AC493F7F7070AC8A384F50020
:10B2B0002A89AE8401CB1C4283C707002304F70010
:10B2C000EF70D0452164930554022800EFC0AF828F
:10B2D000EFF0FFFAAA852800EFD0FF973000014772
:10B2E0008146A6854A85EFC08FA113044402480811
:10B2F00022CC230A010002CEEFE04FD105616F603E
:10B300001FA6EF629FA301117C003ECAB70707008A
:10B310003ECC7C003ECE83C795002E84AA8493F752
:10B32000F707A384F500A165938555024808EFB09F
:10B330009FFCEFF0DFF4AA854808EFD0DF915008BA
:10B3400001478146A2852685EFC06F9B05616F602E
:10B350001FA197B7FF1F9387E7889C43094599C3AF
:10B3600003C59700828097B7FF1F9387A7879C43E9
:10B37000094599C303C5D700828097B7FF1F9387FC
:10B3800067869C43014599C303C5A7008280EF628D
:10B390003F990111B70708003EC683C79500404D8D
:10B3A0000AC493F7F7070AC8A384F5002A89AE8474
:10B3B00029C01442854703C7060063EEE7068347AA
:10B3C000940009468149638EC700B307F740A30480
:10B3D000E400B339F00083C716002305F400EF70D2
:10B3E000F03303572403058B09C763840900EFA0DA
:10B3F000B06B2164930584022800EFB0DFEFEFF01B
:10B400005FF5AA852800EFD01F85EFF01FF7AA850A
:10B410002800EFD05F84014781463000A6854A8529
:10B42000EFC0EF8D13047402480822CC230A0100F8
:10B4300002CEEFE0AFBD05616F60DF91EF62FF8F7D
:10B4400001117C003ECAB70708003ECC7C003ECE0E
:10B4500083C795002E84AA8493F7F707A384F50089
:10B46000A165938585024808EFB0FFE8EFF07FEE15
:10B47000AA854808EFD02FFEEFF03FF0AA854808D4
:10B48000EFD06FFD500801478146A2852685EFC0A9
:10B490000F8705616F60BF8C97A7FF1F9387877425
:10B4A0009C43014599C303C5B7008280EF62FF88C2
:10B4B0000111B70707003EC683C79500404D0AC477
:10B4C00093F7F7070AC8A384F5002A89AE8405C458
:10B4D0001C42054783C70700636AF7040347B400AB
:10B4E000630BF700A305F400EF7050238347B4000B
:10B4F000A9C3EFD00FD921649305B4002800EFB0A1
:10B500009FDFEFF07FF9AA852800EFD0CFF4014745
:10B5100081463000A6854A85EFB07FFE29044808A1
:10B5200022CC230A010002CEEFE04FAE05616F602E
:10B530001F83EFD02FDAC1B7EF623F8001117C008B
:10B540003ECAB70707003ECC7C003ECE83C79500BD
:10B550002E84AA8493F7F707A384F500A165AD05AF
:10B560004808EFB05FD9EFF03FF3AA854808EFD065
:10B570008FEE500801478146A2852685EFB03FF83F
:10B5800005616F60CFFD97A7FF1F9387A7659C4359
:10B59000094599C303C5C7008280EF620FFA011104
:10B5A0007C00AE843ECAA165B70707002A843ECC62
:10B5B000D1057C0048083ECEEFB0FFD3EFF0BFFCD2
:10B5C000AA854808EFD02FE9500801478146A68593
:10B5D0002285EFB0DFF205616F606FF8EF62EFF583
:10B5E00083C7950093F7F707A384F500EFF0FFFA00
:10B5F0006F60EFF6EF62CFF283C795000329C501B4
:10B60000411193F7F707A384F5001C4283C9070093
:10B61000854763EC370597B7FF1F9387E7B39C43D4
:10B620002E84AA8495C7EFF01FF689476302F502BE
:10B63000630009028347C900638C3701230639017F
:10B64000EF70D00D83572903898B99C3EFA0D045A4
:10B650002685A285EFF07FF4A167CD0748003EC4A0
:10B660002302010002C6EFE06F9A41016F608FEE86
:10B6700097A7FF1F938707579C431D4599C303C591
:10B68000E7008280EF626FEB0111B70707003EC64B
:10B6900083C79500584D0AC493F7F7070AC8A384D7
:10B6A000F5002A89AE8405C71C4283C7070093961C
:10B6B0008701E18663C8060485466385D70483460F
:10B6C000E7006386F6002307F700EF70300521647A
:10B6D0009305E4002800EFB01FC2EFF07FF9AA85C0
:10B6E0002800EFD04FD7014781463000A6854A8514
:10B6F000EFB0FFE03504480822CC230A010002CE57
:10B70000EFE0CF9005616F608FE5EF620FE301110D
:10B710007C003ECAB70707003ECC7C003ECE83C704
:10B7200095002E84AA8493F7F707A384F500A165FA
:10B73000B9054808EFB03FBCEFF09FF3AA85480871
:10B74000EFD06FD1500801478146A2852685EFB022
:10B750001FDB05616F60AFE0EF628FDCAA840144FC
:10B7600017A9FF1F13094948E149EFC0FF9063443F
:10B77000A400014519A833053403832709003E9529
:10B78000835725006395970011056F60AFDC0504B2
:10B79000E9BF032E850063040E1017A3FF1F1303D8
:10B7A000636303230300631503002943639A060EB2
:10B7B00003234E01631503001D436393070EEF62DD
:10B7C0004FD5C689428A3E89BA8AB684328BAE8BFF
:10B7D0002A84A1E903554E0009E501431A856F60EB
:10B7E000CFD6A167A98F116763F7E700EFF0DFF607
:10B7F0008145EFF08FBD0844B70700E05841F98F4D
:10B8000018455CC1B707001FF98F1CC55C4981C78B
:10B810006105EFB01000E38209FC2285EF70606ED5
:10B820006DBF3285EFA0E0620D434DD91C44116716
:10B8300003D54700A167A98F63F7E700EFF0DFF1B9
:10B840008145EFF08FB80323840093164B01D1821A
:10B850008347B300035663008588FD8BA305F3007F
:10B86000FD777D8E558EFD76FD16B204F18E832711
:10B870004301C58E231273012313D3002304530104
:10B8800023052301A3044301D9D72285EFB07FBB51
:10B89000AA850844B5DD6105EFB02076ADBF1D4334
:10B8A0001A858280EF62CFC70569AA84AE89328A81
:10B8B0000144FD5A7D19EFC0EFF06345A400014536
:10B8C0006F604FC9D84493171400BA9703D7070085
:10B8D000631B37032390570163050A002685EF7029
:10B8E000E0389C448DC383D76700B3F72701639C7E
:10B8F0003701D28801488147014781460146814589
:10B900002685EFF01FE905047DB7EF626FC17971FD
:10B910001C103EC4B7070F003EC61C103EC883C7AC
:10B920009500AA8A328593F7F707A384F5002E893C
:10B930003284EFD00FBE93170501C1876350F00624
:10B94000AA892285EFD0EFBC2A8A4E85032B0400FA
:10B95000EFB05F9039E58357440081440544F11707
:10B9600093B71700A303F10083457100DA8722879C
:10B97000D2864E862800EFE03FA401478146300082
:10B98000CA855685EFB0BFB7A1679387F70348080C
:10B990003ECC230A810026CEEFD05FE745616F6081
:10B9A0006FBBA28513067100EFE0BFAFAA84094404
:10B9B00045DD5285EFE0EFB80D445DD50546D285F3
:10B9C0002685EFF03FEE2A8445B7EF620FB7835527
:10B9D00007000346270041112A842E8532C62EC453
:10B9E000EFE02FB611C53246A2452285EFF09FEB5E
:10B9F00041016F60CFB6EF62CFB183C795004111AF
:10BA0000AA8A93F7F707A384F5003285AE893284BA
:10BA1000EFD02FB093170501C1876357F008C145D8
:10BA20002A8A2285EFD04F9B2A8D2285EFD06FAED8
:10BA30002A892285EFD08FAC930705F893F7F70F8B
:10BA40001307E007AA8B6371F7062285EFD00FABCF
:10BA50002A8C2285EFD08FAAAA8C5285032B040052
:10BA6000EFB04FFF29E583574400231101008144C3
:10BA7000F11793B71700A300F10005440347110025
:10BA800083562100938784005685DA88228852865F
:10BA9000CE85EFE03FE6A167E90748003EC42302F8
:10BAA000810026C6EFD09FD641016F600FAA130612
:10BAB0001100A285EFE0FF9EAA8409E52311010091
:10BAC00009446DBF930521006A85EFF06FA12A84B8
:10BAD00055F5835521009356C90013164901854831
:10BAE0006688E2875E87858A51822685EFF07FCA65
:10BAF0002A8469B7EF62EFA183C7950041112A8BB1
:10BB000093F7F707A384F5003285AE893284EFD02E
:10BB10004FA093170501C1876352F0082A8A228536
:10BB2000EFD02F9FAA8A2285EFD0AF9E2A89228547
:10BB3000EFD0CF9C930705F893F7F70F1307E007B3
:10BB40002A8C637DF7042285EFD04F9BAA8C228537
:10BB5000EFD0CF9A2A8D5285832B0400EFB08FEF60
:10BB600029E18357440085440144F11793B7170036
:10BB7000A301F10003473100930784005A85DE8852
:10BB80002688D6865286CE85EFE0DFD68D474800E0
:10BB90003EC42302910022C6EFD05FC741016F600F
:10BBA000CF9AA28513063100EFE0BF8F2A84894423
:10BBB00071D19356C9001316490185486A88E687F2
:10BBC0006287858A5182D685EFF0BFBCAA845DB7B3
:10BBD000EF620F952A8981440144617A916A17AB1B
:10BBE000FF1F130B2B1FEFC0EFBE63C5A400228500
:10BBF0006F604F968327090093991400CE9703D561
:10BC0000070033074501420741836362570311CDA3
:10BC100003270B0009C785453E85EF30E04A83279F
:10BC200009000504CE972390070085046DBFEFF04F
:10BC3000BFB2832709000504CE972390070075D56E
:10BC40008145EFE09FF8D5B7EF628F8D83C79500F0
:10BC500041112A8A93F7F707A384F50032852E89CC
:10BC60003284EFD00F8B93170501C1876354F00422
:10BC7000AA89832A0400EFB0EFDD21E18357440055
:10BC800085440144F11793B71700A301F10003485D
:10BC90003100D68752850147CE862686CA85EFD0E9
:10BCA0001FE3A167F50748003EC42302910022C6A6
:10BCB000EFD0DFB541016F60EF89A2851306310037
:10BCC000EFE02FFE2A84894479D197A7FF1F93873D
:10BCD00067109C4381CB0449EFC0CFAFAA8526856E
:10BCE000EF30803E13050401EFF09FEE2285EF60F8
:10BCF0009079814469BFEF62CF8183C7950041117C
:10BD0000AA8A93F7F707A384F5003285AE893284B7
:10BD100023110100EFC0FFFF93170501C187635C8A
:10BD2000F0042A8AC1452285EFC01FEBAA8B5285F9
:10BD3000032B0400EFB00FD231E183574400854458
:10BD40000144F11793B71700A300F1000348110055
:10BD500003572100DA875685D2862686CE85EFD016
:10BD60001FD7A1679387270248003EC42302910092
:10BD700022C6EFD0BFA941016F503FFDA285130637
:10BD80001100EFE00FF22A84894469D197A7FF1FC1
:10BD90009387470498433E8901CB0449EFC08FA3A2
:10BDA000AA852685EF30403213050401EFF05FE2EB
:10BDB000EFC04FA2954459D9930521005E85EFE06D
:10BDC0003FF2AA8441F51C480357210022852390A5
:10BDD000E700EF60506B83270900ADDB03552100BE
:10BDE000EF30E026A5B7EF52DFF283C7950041118F
:10BDF000AA8A93F7F707A384F5003285AE893284C7
:10BE0000EFC03FF193170501C1876359F0042A8AF7
:10BE10002285EFC01FF02A895285032B0400EFB062
:10BE20006FC321E18357440085440144F11793B760
:10BE30001700A301F10003483100DA8756854A87CD
:10BE4000D2862686CE85EFD09FC8A167F907480025
:10BE50003EC42302910022C6EFD05F9B41016F5088
:10BE6000DFEEA28513063100EFE0AFE32A848944B8
:10BE700079D19167CA97C2071167C1831307F7EF9A
:10BE80008544E36AF7FA97A7FF1F9387A7F49843BF
:10BE9000BE8B01CB0449EFC0EF93AA852685EF3016
:10BEA000A02213050401EFF0BFD2EFC0AF9295447A
:10BEB00059D11C482285814423902701EF60B05C52
:10BEC00083A70B00ADDB4A85EF306018ADB7EF52AA
:10BED000DFE62A844105B284EFF09FCF01C52285B9
:10BEE000EF60705A81460146A6852285EF70C00B2F
:10BEF0001C4C89C7DC4799C3228582976F503FE667
:10BF000097A7FF1F938707CE9C43014599C31385CD
:10BF10000701828097A7FF1F9387C7CC8843828041
:10BF2000EF52BFE19317C600DD8DC2054111C181FB
:10BF30002A8432C6EFC07FD33246228511829375A0
:10BF4000F60FEFC05FD141016F507FE1EF525FDD2F
:10BF500079713C083ED2B7070C003ED43C083ED66F
:10BF600083C79500AE842A8993F7F707A384F50069
:10BF7000A165938535044810EFB0EFB7C165FD1595
:10BF8000014417AAFF1F130A6AE6930A400EAE89FE
:10BF90002E8B2EC6EFC00F874205931704014181F7
:10BFA000C183B24563E3A702C167FD176385F5004E
:10BFB0004810EFC09FCB501001478146A6854A85A7
:10BFC000EFB0EFD345616F50FFD833075403832799
:10BFD0000A0BBA9703D6C701630836016388350197
:10BFE0004810EFF0FFF3DA85050465B7B285EDBFC1
:10BFF000EF523FD279717C083EC8B70711003ECAA4
:10C000007C083ECC83C79500AA89328593F7F70751
:10C01000A384F5002E89EFC0DFCF8567637EF5022C
:10C02000A165AA8489050808EFB0EFAC2685EF303A
:10C03000E052133415000A04A2850808EFC0BFC1FE
:10C04000A6850808EFC07FC235C0014781461008A9
:10C05000CA854E85EFB0AFCA45616F501FCFB30799
:10C0600054030327CA0ABA9703D70700631A970035
:10C0700003D62700638A65030808EFF07FEADE85B0
:10C0800005042EC6EFB01FF9420593170401418144
:10C09000C183B245E3E5A7FCC167FD17E387F5FA65
:10C0A0000808EFC09FBC55B7B285D9BFC165FD1563
:10C0B000014417AAFF1F130A6AD3930A80022E8B2A
:10C0C000AE8BC1B7EF527FC7184183471700834635
:10C0D0000700A207D58FD207D1832390F5008347AD
:10C0E0002700034717008D45A207D98F918323109E
:10C0F000F600EFC03FAD6F509FC6EF527FC2C164E4
:10C10000014417A9FF1F130969CE93098002FD148A
:10C11000EFB05FF06345A40001456F50BFC3330526
:10C1200034038327C90A3E9583570500E38797FEAA
:10C130000504F9BFEF52DFBE2A8AAE89B284B68AFF
:10C14000EF30C04109E591473E856F50BFC02A8955
:10C150004E85EF9010502A84638A0A048D476DD56E
:10C1600003570500C547E31147FF0347F90185461B
:10C17000AD47E31BD7FC8347450091CB4146A685DD
:10C180005D05EFC0D022814761D1AD4775BF13096E
:10C1900065012302E500CA852685EF10202D15CD07
:10C1A000A547E3830AFA2302040079BF11CD835720
:10C1B0000500E39A47F94146A6851905EFC0301FEF
:10C1C000814759D1994749B74E85EFF01FF32A842B
:10C1D00095473DD9130955007DBF4146A6852310DB
:10C1E00044012311340113051900EFC0B01E22854C
:10C1F000EF60B03C814789BFEF523FB479717C005A
:10C200003ECCB7070A003ECE7C003ED083C79500E7
:10C21000B2842E8493F7F707A384F5001306A100D8
:10C220002A892C002685EFF0FFE9A16528088D05F5
:10C23000EFB06F8C90408355A10003558100854677
:10C24000EFF05FEFAA84AA852808EFC0DFA00356AD
:10C25000A100835581002808EFF09FCC30080147EA
:10C260008146A2854A85EFB08FA9854748103ED404
:10C270002302910202D6EFD06FD945616F503FAED5
:10C28000EF52BFAB79717C003ECCB7070A003ECEBF
:10C290007C003ED083C79500B2842E8493F7F707C5
:10C2A000A384F5001306A1002A892C002685EFF04F
:10C2B0007FE1A16528088D05EFB0EF83904083559D
:10C2C000A100035581008146EFF0DFE6AA84AA852C
:10C2D0002808EFC05F980356A10083558100280805
:10C2E000EFF01FC4300801478146A2854A85EFB0B0
:10C2F0000FA148102302910202D402D6EFD00FD131
:10C3000045616F50DFA5EF525FA3EFF0BFE26F50C2
:10C310001FA597A7FF1F9387278D88438280EF5221
:10C32000DFA1835725004111AE842A842307B10081
:10C3300017F5FFFF1305A5696C002316F100EFB098
:10C34000CFD581C42285EF60B02DFD572310F400B6
:10C3500013062002814513055400EF501FA141012F
:10C360006F50FF9FEF52DF9B79717C003ECCB70787
:10C370000A003ECE7C003ED083C79500AA89AE84D9
:10C3800093F7F7073285A384F5001306A1002C006C
:10C39000EFF05FD3035581001144EF30201C15C12D
:10C3A0000355A1000144EF90D02A01CD03570500A9
:10C3B0008357810045446316F7008545EFF03FF64B
:10C3C00001442169930539002808EFA0DFF2A28516
:10C3D0002808EFC05F880356A10083558100280814
:10C3E000EFF01FB4300801478146A6854E85EFB0B7
:10C3F0000F9148104AD42302810202D6EFD00FC118
:10C4000045616F503F95EF52BF919797FF1F9387FC
:10C41000677D2A8488432E8915C1035745038357B6
:10C42000C401631DF70023260502231805024105F8
:10C43000EFA0303E63040900EF60302F814497A9DC
:10C44000FF1F9389A99A130A8002EFB0BFBC63CC87
:10C45000A40297A7FF1F9387A7819C4389C7035511
:10C46000C401EF104076630509002285EF60500398
:10C470001306400E81452285EF503F8FFD57231E46
:10C48000F4006F503F8D3385440383A7C90A3E955E
:10C49000035705008357C4016315F700CA85EFF001
:10C4A0001FE885045DB7EF52BF8783C79500411130
:10C4B000AA8993F7F707A384F5003285AE84EFC00D
:10C4C0005F8585676370F5042A89EF302009014490
:10C4D00011C983D704003144638627018545EFF0F5
:10C4E0009FF201444E85A2864A86A685EFD02FBFD3
:10C4F000A1679387170448003EC42302810002C647
:10C50000EFD0CFB041016F50FF84EF527F819797FA
:10C51000FF1F9387276D80431DCC0145EFA0E05698
:10C5200081470148C1641CDC232E0403232004043A
:10C5300017A9FF1F1309898B01449309400EFD14AD
:10C54000EFB05FAC634BA4008145170500001305F5
:10C550004598EFB08FB46F50EFFF33053403832756
:10C56000090B3E958357C501638597008545EFF01C
:10C570009FE90504F1B79357050113D78700A380FE
:10C58000F50093170501C183A1832380E500238172
:10C59000F500A381A5008280EF522FFA2300050049
:10C5A00083C71500A300F50083C725002301F5000C
:10C5B00083C73500A301F50083C745002302F500BA
:10C5C00083C75500A302F50083C765009305950056
:10C5D000A30305002303F500230405003285EFF0D3
:10C5E0009FF96F50CFF7EF52AFF34111E9541DC9D6
:10C5F00095C993F9C5FF2E842A89AA84338AA90094
:10C60000B7EA040063149A020D88854401CCB7E7A9
:10C6100004009C5F82972AC622866C00330539018C
:10C62000EFC0405B268541016F50CFF283A78A039C
:10C630009104829793170501C183A183A38EF4FE11
:10C6400093570501238FF4FEA183238EA4FEA38FAD
:10C65000F4FE4DBF63E0D502EF522FEEB2874111D9
:10C660003686BE8536C6EFC0E056B24641013685F5
:10C670006F50EFEE814636858280838705001387F1
:10C68000F5003D05FD8793F77708834607007D1584
:10C690008606B58FA300F5006307B7007D178347B3
:10C6A00017009D83DDB78280EF522FE9B7E70400C2
:10C6B00083A7070932872A863A85829713351500A2
:10C6C0006F50EFE901CD814799C9EF520FE741461D
:10C6D000EFC0405085473E856F506FE881473E85EB
:10C6E00082801DC5EF526FE5414681452A84EF5097
:10C6F000CFE74146814513050403EF500FE701479B
:10C70000C1672322040438C87CC805456F502FE553
:10C7100001458280814729CDA1CDEF520FE2B2843D
:10C720002E891306800581452A84EF500FE4CA85BF
:10C7300024C42685EFF01FF9414681452285EF503C
:10C74000CFE23044A2852285EFF01FF69304040166
:10C75000A2852685EFF07FF2A68513050402EFF08F
:10C76000DFF12285EFF0FFF785473E856F502FDF21
:10C770003E858280EF52CFDA4111E9541DC995C937
:10C7800093F9C5FF2E842A89AA84338AA900B7EABF
:10C790000400639444030D88814401CCB7E704008E
:10C7A0009C5F82972AC622866C0033053901EFC050
:10C7B0006042268541016F50EFD983A78A03910417
:10C7C000829793170501C183A183A38EF4FE93572B
:10C7D0000501238FF4FEA183238EA4FEA38FF4FE14
:10C7E0004DBF71CDEF52CFD3B28401E605456F50F6
:10C7F0006FD62A842E890145FDD93C487848B3E696
:10C80000E700F5D69386F7FFB3B7F6007D17032A46
:10C810004404BA9734C87CC8630F0A04C14913059D
:10C820000A03B38949412295637B3601B2862E867D
:10C83000A685EFF03FE27C40BE9464C045BFCE8643
:10C840002E86CE85EFF01FE1C114D2944E9923229B
:10C850000404A2879306040103C7070003C6070365
:10C860008507318FA38FE7FEE398F6FE3044A2855B
:10C870002285EFF07FE32699C1493306994063EAA8
:10C880009900ADD4A686A68513050403EFF09FDCBE
:10C890006DB78147B306F4003307F600034707007E
:10C8A00083C5060085072D8F2380E600E39437FFBC
:10C8B0003044A2852285EFF03FDFC1147DBF0145E2
:10C8C000828019C9EF526FC7130680058145EF506A
:10C8D000CFC905456F50AFC80145828081473DC92A
:10C8E000B5C9EF528FC5FC4141462E84AA8463939B
:10C8F000C70413860501A2878146C14503C7070007
:10C9000003C507038507298F3305D60003450500B6
:10C910008506298FA38FE7FEE392B6FE3044A285F9
:10C920002685EFF07FD82285EFF0BFF985473E8559
:10C930006F50EFC2138507031D8E81452295EF507E
:10C94000CFC27C40130700F813060402A297238885
:10C95000E70255B73E858280EF522FBE6D712E845F
:10C96000B284AA85901028003689EFF0BFDA19E961
:10C97000D55705A050400C402800EFF09FE66DD938
:10C98000FD142104E5F82C004A85EFF03FF58147BE
:10C9900065D13E8551616F508FBCEF520FBA411186
:10C9A0002EC432C62C000546EFF01FFB41016F502C
:10C9B0000FBBEF528FB801112A842EC602C802CADB
:10C9C00002CC02CEEFC06049B2462A86A285080892
:10C9D000EFF0BFFC1375F50F05616F504FB8EF52C4
:10C9E000CFB57971B2872A8421462308B100130597
:10C9F0001101BE853AC436C6EFC0C01DB2469305CC
:10CA000091013685EFF03FB72285141035460C08AA
:10CA1000EFF0BFF82A84224711E521460C103A8531
:10CA2000EFC0401B228545616F506FB3EF52EFB0EE
:10CA30007171AE84AA850A853284EFF0BFC801C93E
:10CA40000A86A6852285EFF03FC6814711E1C547DA
:10CA50003E854D616F50AFB0EF522FAB1D712A8AEA
:10CA6000B289BE8435468547130511012E8CB68ADE
:10CA70003A8BC28C468D2308F100EFC0A015101030
:10CA80000C085285231F0100EFF05FFA2A842DE97C
:10CA9000A147631BFD069307900591E0E5473546E6
:10CAA000E2851305110113990A012308F1001359B6
:10CAB0000901EFC020121357890093978A00D98F7C
:10CAC00090080C085285231FF100EFF03FF62A84EE
:10CAD00005E9A1E09387FA0091831379F9003EC636
:10CAE000631309004149668B8144C14B854DB247B0
:10CAF0006397970C6A868C0033855C01EFC0800DCC
:10CB0000228525616F502FA493079004C9F8A5478B
:10CB100079B7834701050947C14B2308F1008347D3
:10CB20001105A58FA308F10093872400814463EFCA
:10CB3000FB02014714083386E6008C08B386E40044
:10CB4000BA95DA9683C6060083C505000507AD8E43
:10CB50002300D600E390E7FE41476398E70490087E
:10CB60000C085285EFF09FEC35D535A8B3069B0035
:10CB7000BA871008B305F60090083E9603C5060074
:10CB80000346060085078506298E2380C500E392AB
:10CB900077FF998F90080C085285BE94EFF01FE93B
:10CBA0008947014749D52A84A1BF90083E9603468C
:10CBB00006001408BE962380C600850779BFB247D9
:10CBC0008504638B971281471808B306F70098080D
:10CBD0003E973386F90003470700034606008507A2
:10CBE000318F2380E600E39177FF90080C0852858F
:10CBF000EFF0DFE34DF93546E28513051101230817
:10CC0000B101EFB0307D1397040141839397840005
:10CC10002183D98F10180C085285231FF100EFF0E3
:10CC2000FFE051F1814710183387F9003E96034722
:10CC3000070003460600B306FB008507318F2380FB
:10CC4000E600E39277FF75A01808B306F70098088E
:10CC50003E973386F9000347070003460600850721
:10CC6000318F2380E600E3E127FFCA8763987709C5
:10CC700090080C085285EFF07FDB15F5814798008E
:10CC8000B306F700900818103E973E96034707003A
:10CC9000034606008507318F2380E600E39177FF86
:10CCA0003546E285130511012308B101EFB09072FA
:10CCB000139704014183939784002183D98F10181F
:10CCC0000C085285231FF100EFF05FD6E31D05EC41
:10CCD000814710183387F9003E9603470700034643
:10CCE0000600B306FB008507318F2380E600E3E2F0
:10CCF00027FFC109410BE5BB8147B5B79408BE9634
:10CD000083C6060018083E972300D7008507B9BFE1
:10CD1000638E062CEF427FFF59712A84BE89B28B45
:10CD200085473546130511022E8B468C4289BA8AF7
:10CD3000368A2300F102EFB0F06910180C1022853A
:10CD400023170102EFF09FCE631E0510A147631960
:10CD5000FC069307900563930900E5473546DA859D
:10CD60001305110293140A012300F102C180EFB0F0
:10CD7000706693178A0013D78400D98F90080C101F
:10CD800022852317F102EFF07FCA69ED6390090451
:10CD90009307FA00BD88918391E0C144C207C18323
:10CDA000DE8C814A3EC6414DB24763EAFA0C628688
:10CDB000B3854B018810EFB0905F4DC53D555DA028
:10CDC00093079004E39C09F8A54749BF83470105F1
:10CDD0000947C14C2300F10283471105B3C7F9008D
:10CDE000A300F10293872900814963EFFC02814689
:10CDF00018103306D7008C083387D900B69556979C
:10CE00000347070083C5050085062D8F2300E60034
:10CE1000E390D7FE4147639AE70490080C102285FF
:10CE2000EFF0DFC035D53DA8B3863A01BA871010C0
:10CE3000B305F60090083E9603C5060003460600BB
:10CE400085078506298E2380C500E39297FF3387E7
:10CE5000EC4090080C102285BA99EFF03FBD89474D
:10CE6000014741D565616F401FEE90083E9603462D
:10CE700006001410BE962380C600850769BFB2471E
:10CE8000850A93990A01939D8A0093D909016399B0
:10CE9000570D85473546DA85130511022300F10247
:10CEA00093D98900EFB01053B3ED3D0190000C1001
:10CEB00022852317B103EFF07FB74DF58147A6898F
:10CEC00063E6970626860C084A85EFB0B050814786
:10CED0001810B306F700100898083E973E960347CF
:10CEE0000700034606008507318F2380E600E3E153
:10CEF00097FE639DA90590080C102285EFF01FB3E3
:10CF000035F181479810B306F700900818183E973E
:10CF10003E9603470700034606008507318F2380AE
:10CF2000E600E391A7FF4109C10CBDBD18089000C0
:10CF3000B306F7003E963387FC000347070003461D
:10CF400006008507318F2380E60095BF98084E972D
:10CF5000034707001C10CE972380E700850951BFC7
:10CF600085473546DA85130511022300F10293D96E
:10CF70008900EFB03046B3ED3D0190000C102285E2
:10CF80002317B103EFF09FAAE31E05EC81471808B1
:10CF90009000B306F7003E963387FC000347070076
:10CFA000034606008507318F2380E600E391A7FF43
:10CFB00041460C084A85EFB0F04181471810B3068E
:10CFC000F700100898083E973E960347070003466F
:10CFD00006008507318F2380E600E391A7FF9008C4
:10CFE0000C102285EFF09FA41DDDADBD7D55828024
:10CFF000EF42BFD401112A842E8593055100328956
:10D0000002C002C202C402C693047400EFF0AFD69D
:10D010001D46A68513059100EFB0D03B10088A8508
:10D020004A85EFF0BFA019ED93071400180883C6D6
:10D0300007000346070085070507B18EA38FD7FEBB
:10D04000E397F4FE05616F409FD1EF427FCD2E84C0
:10D050008C414111AA89838715003289914463D399
:10D060000700A1449797FF1F9387070F9C43B1C305
:10D07000B5CE8D472310F10083C725004A852301D3
:10D08000F10083C73500A301F10083C745002302E7
:10D09000F10083C75500A302F10083C76500930523
:10D0A0009100A30301002303F10023040100EFF02A
:10D0B0008FCC0C404A860A85EFF00FCE032804007F
:10D0C00083564400A6881D0881470147E51642861D
:10D0D0008A854E85EFF05F982A8909E5A685228525
:10D0E000EFB0FFB24A8541016F40DFC64A860A852C
:10D0F000EFF08FCA7DBFEF42BFC22E848C41411139
:10D10000AA89838715003289914463D30700A1441B
:10D110009797FF1F938747049C43B1C3A5CE8D47C4
:10D120002310F10083C725004A852301F10083C73E
:10D130003500A301F10083C745002302F10083C736
:10D140005500A302F10083C7650093059100A30376
:10D1500001002303F10023040100EFF0CFC10C40D4
:10D160004A860A85EFF04FC3835644000328040023
:10D170008A85858EC2061D08C1822312D400A68826
:10D1800081470147E51642864E85EFF07FB84101A1
:10D190006F405FBC4A860A85EFF00FC0C9B7EF4207
:10D1A000DFB9B335B000011185052A891315F601E1
:10D1B000336515012308B1009305110136843AC681
:10D1C00032C03EC442C2EFF00FBBA24712484255E4
:10D1D00093D68700230BF1009305910193578800A4
:10D1E000A30AD100A30BF100230C0101EFF0AFB8AB
:10D1F0003247024603280400B337E0008356440058
:10D200009207914411C2A1444A85A68842860C081F
:10D21000EFF09F842A8909E5A6852285EFB03F9F1C
:10D220004A8505616F40BFB3EF429FAF01113EC613
:10D230008647B335B0008505AA891315F6015D8DC3
:10D240002308B1009305110136843A89B28442C49F
:10D2500046C2EFF04FB222489248164593578800D5
:10D26000A30AF1009305910193D78800230B0101D4
:10D27000A30BF100230C1101EFF0EFAF3247104088
:10D2800083564400B337E000920703280900914811
:10D2900091C0A1480C084E85EFF09FA7AA8411E524
:10D2A000835544004A85EFB09F96268505616F40FF
:10D2B0007FAAAA959307F00F17F700001307478A74
:10D2C0006317B50013C5F7FF1375F50F82800505C9
:10D2D0008346F5FFB58FBA9783C70700D5B70357C5
:10D2E000450014419307F00F17F600001306468718
:10D2F000369742074183139506014181631BE50080
:10D30000AD8FB29703C50700130515F3133515004C
:10D310008280850603C5F6FFA98FB29783C70700F1
:10D32000D9BFEF429FA1B28736842E86BA86AA85DE
:10D330003E85BA84EFF06FE6634B05002285EFB0BF
:10D34000D0312A86A686A2852685EFF00FE56F40AC
:10D350001FA1EF42FF9C5D712A8BAE8A17E500008A
:10D360001305857D2C00B284368ABA893E89EFF098
:10D370004FE42A8459E534104146DA852800EFF05D
:10D38000CFE12A843DED8547A303F100A6C29307B0
:10D3900071002408BEC4A68685470D462C182810A7
:10D3A00002DC02DED6C0BEC6EFF00FDB2A8431E914
:10D3B00083477102A6860D4693F7F7072300FA000C
:10D3C000C1473EDE2C188947281026DCA303F10054
:10D3D000EFF08FD82A8415E54146A6854E85EFB03B
:10D3E000607F8D47A6860D462C182810A303F100F8
:10D3F000EFF08FD62A8411E54146A6854A85EFB025
:10D40000607D228561616F40FF94EF421F9397D743
:10D4100000009387270C984383C7470079712A89B6
:10D42000AE8417E500001305A5710C083AC4230665
:10D43000F100EFF00FD82A8415E514104146CA8593
:10D440000808EFF08FD52A8411ED140815462C003A
:10D450000810EFF08FD42A8411E521462C08268588
:10D46000EFB04077228545616F407F8FEF42FF8CA0
:10D4700097D70000938707069C477971AA842E846A
:10D4800017E500001305456C0C083EC6EFF06FD29F
:10D490000DE514104146A6850808EFF00FD011EDF8
:10D4A000140811466C000810EFF02FCF19E58347E0
:10D4B000F10193F7F7032300F40045616F403F8AC1
:10D4C000EF42BF873688A14881470147E546EFF024
:10D4D000AFD86F40DF88EF425F863688A14881472A
:10D4E0000147E546EFF0DF826F407F87EF42FF8420
:10D4F00001112A842E850C0832C6EFF08FCB19E972
:10D50000324797E600009386A6621008C14522853F
:10D51000EFF03FE105616F409F84EF421F824111B0
:10D52000C1472EC032C48A8509463EC23EC6EFF0CE
:10D53000AFC241016F40BF82EF423F804111AE86D2
:10D5400013061009AA850A8502C002C202C402C6D7
:10D55000EFF0AFC441016F409F80EF420FFE328772
:10D5600097E600009386C65E2E8693050002EFF0D4
:10D570005FDB6F40CFFEEF424FFC7971C1472ACC91
:10D580002ED032D42C080D4628003ECE3ED23ED6B8
:10D5900002C402C602C802CAEFF00FBC45616F4068
:10D5A0000FFCEF428FF90111AA842E8417E50000C9
:10D5B0001305855A8A85EFF0CFBF05E5140841466B
:10D5C000A6850A85EFF06FBD09ED8347E1010347AA
:10D5D000F101A207D98FCA07C9836177D98F2310B8
:10D5E000F40005616F40AFF705C9EF420FF597876B
:10D5F000FF1F9387E76390439785FF1F938585639C
:10D600001785FF1F1305C55EEFB080091785FF1F43
:10D610001305055E6F40AFF41785FF1F1305455DC9
:10D6200082809DC5EF426FF19787FF1F9387476008
:10D63000944301112E840A869785FF1F9385855F89
:10D64000EFB0800A0A850294014505616F402FF111
:10D650007D558280EF426FEEEFB080149787FF1FF9
:10D6600023A8A75C17F5FFFF130525F8EF90D0401E
:10D670006F40EFEE1787FF1F1307C75D9317150065
:10D6800008433E95FD572310F5008280EF42EFEAF4
:10D690002A84084019E16F408FEC1C4158401CC09F
:10D6A0006313E5005CC08347550023200500F99B08
:10D6B000A302F500EFB0EFF9E9BFEF426FE69787FD
:10D6C000FF1F9387275B98432A8411CB834735003C
:10D6D00093F7070289C7035505008945029713058B
:10D6E0004401EF901013835504000355E400EF202C
:10D6F000701B485809C5EFB0CFF5232A0402130563
:10D700008403EFF0BFF88144B149EFA0FF9A63C5ED
:10D71000A402834734002320040493F727FCA301C9
:10D72000F4000048EFA05F9A13161500814522858A
:10D73000EF40AFE36F400FE2B387340303290403E4
:10D7400085043E994A85EFF07FF42304090075BFF4
:10D750008347350093F7070299E301458280835799
:10D76000E500E39CB7FEC167FD176316F6000545AB
:10D7700082800545B9A0EF424FDC93170601C187AF
:10D78000B2842A8401496359F002835705008DCB86
:10D7900001456367F600034584003E953325A600E6
:10D7A0001375F50F39A81C4813171900BA9783D7BA
:10D7B0000700E38097FC0509EFA01F91E345A9FE50
:10D7C00001456F40CFD9EF42AFD5AE89AA84EFA013
:10D7D0007F852A84EFD0BFAAAA8601471306840159
:10D7E00097050000938545E91785FF1F1305C5467A
:10D7F000EFA0AFD52A8921CD8C441304C500228522
:10D800009E0593F50508EFB00FC5CC4083877400E3
:10D81000E18163D1070493E505082285EFB0AFC32A
:10D820000D46938544002285EFB00FC183D50400D7
:10D830002285EFB0EFC583D524002285EFB04FC518
:10D8400003D6490083A509002285EFB0EFBE4A85C3
:10D850006F404FD093F5F507C9B7EF420FCE0111D6
:10D860002A84328532C6EFB06FB4EF903F91835770
:10D8700004001787FF1F130767573246231BF10069
:10D88000930700F8A30DF1001C471843231AA100C9
:10D890008983858BB307F740B28548083ECE231CA9
:10D8A0000100230D0100EFF01FF205616F402FCB47
:10D8B000EF420FC70041014529CC9304C4002685DF
:10D8C0003289AE89EFB08FB295452A8A2685035BEF
:10D8D0000401EFB02FAF2685EFB02FC68D45AA8A81
:10D8E0002685EFB02FAE2685EFB02FC55C48420AE3
:10D8F000135A0A01D2975CC42318640181476398C4
:10D900003A0146054D81330625419337160013F53C
:10D91000F70F6F402FC4EF42CFBF89692A8BAE8BC0
:10D92000328AB68A81440144314CFD19EFA0CFF808
:10D9300063C9A400EFA04FFB018D33B5AA006F406F
:10D94000CFC03389840383270B003E9963170A00F5
:10D950008347890085043E94D1BF03560A00DE85C3
:10D960004A8533F6C900EFF0BFF47DD10545C1BF4C
:10D97000EF42AFBC01112A847C000355E5003ECA8A
:10D98000B70707003ECC7C003ECEEF10303D2A8921
:10D9900085454808EFB0EFC199454808EFB02FA77B
:10D9A000AA844A85EF10B03D2380A4009787FF1F0B
:10D9B0009387C7439C434166130606F093968701FD
:10D9C00013D78701558F93D68700F18E558FA20705
:10D9D000B706FF00F58FD98F11462C001385140070
:10D9E0003EC4EFB0201F5008A38204008945228561
:10D9F000EFF0BFE609C9AA8513058403EFB0EFBBBA
:10DA00003C4085073CC005616F406FB5EF42EFB207
:10DA1000EFA08FED2A840504EFA00FEC3305A402DC
:10DA2000F14791453305F502EF10207B01E565557F
:10DA30006F40EFB29787FF1F23A6A722EFA0CFEA80
:10DA40002A840504EFA04FE93305A40289450605A1
:10DA5000EF10A07869DD9787FF1F23ADA71EEFA009
:10DA6000AFE82A840504EFA02FE73304A4029787C8
:10DA7000FF1F2393871EEFA02FE72A84EFA0CFE597
:10DA8000930714003385A7029787FF1F2397A71CCE
:10DA900097E70000938707D01787FF1F2322F71C03
:10DAA000014579B7EF42CFA7AA842E89014497890F
:10DAB000FF1F9389A933130A8006EFA0EFE16345A6
:10DAC000A40001456F400FA93305440383A7090251
:10DAD0004A86A6853E95EFF0BFC719E10504F1BF60
:10DAE0000545CDB7EF42EFA2AA8A2E8BB28B368CBA
:10DAF0003A8A814401448149978CFF1F938C0C2FF3
:10DB0000130D8006EFA04FDD63C7A40011E0854927
:10DB10004E856F408FA33389A40383A70C025E86D2
:10DB2000D6853E994A85EFF0BFC219CDEFA0CFDB75
:10DB30000544636B4501D2866286DA8513050903C5
:10DB4000EFF07FDD11C1854985046DBFEF424F9D28
:10DB5000C16441112A8901449789FF1F93890929CA
:10DB6000130A8006FD1436C632C42EC2EFA0CFD6EB
:10DB700092452246B2466346A400014541016F40EA
:10DB80006F9D3305440383A709023E9509C6834769
:10DB90003500C18B9DC791C68347350093F70702B7
:10DBA0008DC3630699008357E500639C27010357E3
:10DBB000050001CB63E7E50083478500BA97E3CF13
:10DBC000F5FA05044DB7EF42AF95C1642A890144C7
:10DBD0009789FF1F93898921130A8006FD14EFA0FE
:10DBE000AFCF6344A4006F40EF963305440383A78F
:10DBF00009023E958357E500638897006304990006
:10DC000063942701EFF07FAB0504D1BFEF42EF8FA4
:10DC100089692A8AAE8A328BB68B8144178CFF1FA2
:10DC2000130CCC1C930C8006314DFD19EFA0CFCA0C
:10DC300063C4A4006F402F913389940383270C029F
:10DC40008355CA015A863E994A85EFF07FB005CDCB
:10DC5000814D05A03384AD038327090303D60B0050
:10DC6000D68533F6C9003E942285EFF07FC419E5CE
:10DC7000850DEFA06FC4E3CFADFC31A02285EFF09E
:10DC8000FFA023040400850455B7EF428F88416943
:10DC9000AA8A014A178BFF1F130B4B157D19C14B25
:10DCA000054CEFA06FC36344AA006F400F8A93092D
:10DCB0008006B3073A0383290B02BE9983D7E90094
:10DCC000638C270163842A016398570103A48903A5
:10DCD00011E44E85EFF0DFC9050AE1B7835704016F
:10DCE000639977079304C4002685EFA03FF085452C
:10DCF0002A8D2685835C0401EFA0DFEC2685EFA04A
:10DD0000FFFF62056185635F05028D452685EFA0F3
:10DD10007FEB89452685EFA0FFEA89452685EFA0A0
:10DD20007FEA85452685EFA03FEB8347050009473D
:10DD300093F7F7076398E70099452685EFA0DFE999
:10DD4000A30285014848337D2D01231894016A956B
:10DD500048C40040B5BFEF325FFE37E404008327BC
:10DD6000041D82979787FF1F83C747F51755FF1F2D
:10DD70001305453EA300F5008327441C82978327A3
:10DD8000841C81461306F00F8145014582976F3050
:10DD90001FFD1787FF1F130767E218439785FF1FB3
:10DDA00083C5C5F19787FF1F9387C7EF8346870316
:10DDB000034697036397D5009787FF1F2380C7F01B
:10DDC000828083C587010347A7036317B60097873F
:10DDD000FF1F2385E7EE828003C687016317C70014
:10DDE0009787FF1F238CD7EC828083C68701130798
:10DDF00050026319D700930760021787FF1F230F94
:10DE0000F7EA828083C68701130660026315D60095
:10DE100093077002DDB783C7870155BF9787FF1F40
:10DE2000938747E8D44B09476385E608EF32FFF054
:10DE30001789FF1F130949E43E8483470900918B2A
:10DE40009DCFB7E4040083A7041D829783A7441CD9
:10DE50001785FF1F1305C5E2829783A7841C81469F
:10DE60001786FF1F0346C6E381450145829721C1FE
:10DE700083470900ED9B1787FF1F230FF7DE8347BA
:10DE8000040093F7F70F85C791471787FF1F2325D6
:10DE9000F7E2EFF05FECEFF0DFEFB7E70400BC4F25
:10DEA000414691451785FF1F034545E082976F3036
:10DEB0001FEB8280EF327FE88D4741116304F50448
:10DEC000C5476306F50285476310F5029787FF1F74
:10DED0002388A7DEB7E70400BC4B93050010178525
:10DEE000FF1F0345A5DC829741016F305FE785473F
:10DEF0001787FF1F2306F7DCB7E70400BC4B930529
:10DF00000020F1BF9787FF1F9387C7D9D44B1147D4
:10DF1000638DE600B7E7040083A7071D8297B7E784
:10DF20000400BC4B930500045DBF05491787FF1F24
:10DF3000232427D983C7070032C62E8493F7F70F0F
:10DF4000C5D7B7E4040083A7041D7D141374F40F30
:10DF50008297E37689FCB245994703C61500E3F042
:10DF6000C7FCFC4409061785FF1F1305A5D582973A
:10DF7000BC48930500081785FF1F034525D38297EA
:10DF800079BFEF329FDB1787FF1F1307A7D14047E9
:10DF9000184B1C409786FF1F23ACF6D06316E40095
:10DFA0001787FF1F2328F7D0130584FEEF907FF318
:10DFB000035564FFEF903FC6EFA0BFE96F303FDA33
:10DFC000EF32BFD79787FF1F9387C7CDD84BDC476A
:10DFD00099C3EFF01FFB85471787FF1F232EF7CC50
:10DFE0009787FF1F938787BD9C4393050002178582
:10DFF000FF1F0345A5CB83C787031787FF1F230F89
:10E00000F7CAB7E70400BC4B82976F305FD597879C
:10E01000FF1F23ABA7C88280EF329FD037E40400F4
:10E020007C4CA1451785FF1F034545C882977C4856
:10E03000A1451785FF1F034565C79784FF1F93847C
:10E0400064C68297DC4489E7EFF05FDD6F309FD0D4
:10E0500003D567FFEF903FBCAA897DD5D84891478B
:10E060006310F7027C4C91451785FF1F034505C4DB
:10E0700082977C4891451785FF1F034525C38297EA
:10E0800003A9490103D409018947B7E904001787A7
:10E09000FF1F2323F7C283A7091D2104420482978F
:10E0A00083C784011755FF1F1305C50A6119175748
:10E0B000FF1FA301F70A83A7491C41808297978716
:10E0C000FF1F238F07BE83A7C91C8146094693758E
:10E0D000F40F4A85829711E99787FF1F83C787CE80
:10E0E00089C79740FF1FE780A078B7E70400BC4FBF
:10E0F0002146A1451785FF1F034545BB8297B9B748
:10E10000EF32BFC393F7052001112E8481CBEFF0CE
:10E110003FEB1345042005616F307FC493F7051072
:10E12000A9CB9784FF1F9384E4B7DC48EFF07FC648
:10E130001787FF1F130787A8184383C78401034766
:10E1400087036316F700DC4499C3EFF09FE385472C
:10E150001787FF1F2322F7B6B7E70400BC4B9305D0
:10E1600000021785FF1F034565B48297134504100D
:10E170005DB793F70508ADC79787FF1F83C797B4AF
:10E18000E91719469785FF1F9385E5B31305D1005D
:10E1900093F4F70F1789FF1F0349C9B2EFA090232B
:10E1A00093970401C1831787FF1F130727B2231D0D
:10E1B000F100231CF1009787FF1F9387A7AE3ACE8B
:10E1C0003ACAD8432306010009CBDC4393158901E1
:10E1D00054080D46E185680082971345040825BF61
:10E1E00093F72500B1CF9787FF1F9387A7ABD84B35
:10E1F00089476306F7029787FF1F83C7E7A713F7CF
:10E20000270011EF918B99CFB7E70400BC4F13069D
:10E21000000A89451785FF1F034545A982971345C5
:10E220002400D5BD9787FF1F938747999C4383C7D9
:10E2300087031787FF1F2303F7A8EFF0FFDDC5B79C
:10E2400093F7050291C7EFF03FDD13450402E1B5F6
:10E2500093F7850091C7EFF0BFD61345840065BDE5
:10E2600093F7150091C7EFF07FBB1345140065B518
:10E2700093F7450091C7EFF07FBA1345440061BDA5
:10E2800093F7050485C39787FF1F83C7A7A181CB99
:10E29000EFF07FAC91471787FF1F232FF7A013459F
:10E2A000040495BD93F705010145E38607E69787CA
:10E2B000FF1F9387279FD84B91476310F7049787D9
:10E2C000FF1F9387679B9C4313D727008583D98FB4
:10E2D000858B91E7B7E7040083A7071D8297B7E70F
:10E2E0000400FC4F91451785FF1F0345259C82972D
:10E2F00085471787FF1F2321F79C1345040121BD84
:10E300009787FF1F2380A7AC8280EF321FA39787D8
:10E31000FF1F23AF07989787FF1F23AD07988547F7
:10E320001784FF1F130484891787FF1F2326F7987C
:10E330001C4083C787031787FF1F2301F798EF90BF
:10E34000FFDF39C19757FF1F23AAA7E01C4017051D
:10E350000000130525DB83C787031787FF1F230FE3
:10E36000F7941757FF1FA307F7DE9787FF1FA38BAD
:10E370000792B7E7040083A7070882979787FF1FD4
:10E380002386A7926F30BF9DB7C7898E938767EDAD
:10E390001757FF1F2324F7DC55BF1787FF1F0347BD
:10E3A0006790795555E39787FF1F9387A78F03C71A
:10E3B000170005079786FF1FA386E68E03C7170081
:10E3C0008D463377D7029786FF1FA38DE68C83C6D1
:10E3D00017001777FF1F1307677E184393F6F60F92
:10E3E000A9EA834787031787FF1F2309F78C85470F
:10E3F0001787FF1F2308F78A9787FF1F9387C78711
:10E400009C430145998BA9E3EF323F9337E4040025
:10E410007C48C1451785FF1F0345458982973C48C5
:10E4200085451785FF1F03456588829701456F3035
:10E430001F9383C7170085466395F60083479703AC
:10E440005DB78347A70345B782809787FF1F83C7C0
:10E450006785A1CBEF327F8E37E404009787FF1FDB
:10E46000238207847C4885451785FF1F0345058463
:10E4700082977C4C91451785FF1F03452583829722
:10E480007C4891451785FF1F0345458282973C488C
:10E49000C1451785FF1F03456581829701456F3090
:10E4A0001F8C79558280EF325F892A84035565FF7E
:10E4B000EF906FF69777FF1F9387C77ED847BE848C
:10E4C0001DEBEFA05F989C48232004008DEB97770D
:10E4D000FF1F23A1877E9777FF1F23AB877CB7E7BA
:10E4E0000400BC4B89451775FF1F0345257C8297A7
:10E4F00001456F30DF86630A87001843D1B780C3B8
:10E500009777FF1F23A8877AD9BF7955DDB7EF32F8
:10E51000DF829787FF1F9387278B88432326050079
:10E52000232405005105EF80D02E6F305F83EF323A
:10E53000DF801784FF1F130424891C40411189CFF9
:10E540009C472302B5002AC61CC1EFF05FFC1C40AB
:10E550009C4B99C33245829741016F305F80EF3207
:10E56000CFFD4111444D328532842EC6EFA00FF904
:10E570002AC42285EFA0EFF903A84400630C080029
:10E58000B245835744001840224683D54500AA86E9
:10E590002685029841016F308FFCEF320FFA404D13
:10E5A0001DC408C0970500009385E50213054401CA
:10E5B000EF8090189787FF1F938707819C43014541
:10E5C00089E79787FF1F23A187806F304FF97D551B
:10E5D000EDBFEF328FF6011168009305F00F02C610
:10E5E00002C802CA02CC02CEEFF07FF405616F30A0
:10E5F0000FF79777FF1F9387277D9C43D847A16725
:10E600009D076311F702EF324FF301113285EFA03E
:10E61000EFEE230AA10081456800EFF05FF105618C
:10E620006F30EFF382809777FF1F9387E7799C43E2
:10E63000D847A167938777036311F702EF32EFEFB3
:10E6400001113285EFA08FEB230AA10081456800FC
:10E65000EFF0FFED05616F308FF082809777FF1F3D
:10E66000938787769C43D8479547631CF702EF3220
:10E67000CFEC011132853284EFA04FE8230AA100CC
:10E680002285EFA00FE983574400231BA100814599
:10E690003ECC1C4068003ECEEFF07FE905616F3054
:10E6A0000FEC8280930785FF89CF8327C5FF91CB2D
:10E6B000DC4B81CBEF326FE8032585FF82976F300B
:10E6C0000FEA8280EF326FE72A843285EFA00FE3F2
:10E6D000BD4763EBA70018449377F5000345B700E7
:10E6E00041995D8DA305A7006F306FE7EF32EFE42E
:10E6F00001117C003ECAB70707003ECC7C003ECE2D
:10E700005C4D8DCF2A8413858700AE84EF80700422
:10E71000A1652A899D054808EF80FFBD9305803ECD
:10E72000B345B902480893F5F50FEFA0CFD20147E2
:10E7300081465008A6852285EF807FDC05616F3019
:10E740000FE2EF328FDFEFF07FFA6F304FE1EF3201
:10E75000CFDE01117C00AE843ECAA165B707070079
:10E760002A843ECC48087C00938575033ECEEF801A
:10E770009FB81C44480883C5B700BD89EFA0AFCD42
:10E78000500801478146A6852285EF805FD7056145
:10E790006F30EFDCEF326FDA2A84AE84EFF09FF255
:10E7A000A6852285EFF0BFFA6F306FDBEF32EFD82E
:10E7B000EFF0FFF96F30AFDAEF322FD80329C50140
:10E7C0004111630409022A843285B284EFA00FD379
:10E7D0002AC62685EFA0EFD3832749002A8691C752
:10E7E000DC4781C7B2452285829741016F302FD720
:10E7F000EF32AFD4444D81CC2A843285EFA06FD163
:10E80000DC40AA8589C79C4799C3228582976F30CF
:10E810000FD5EF32EFD0032AC501411163030A0679
:10E820002E89AA84954532853284EF80DFAC8545F8
:10E830002285EFA0CFBDAA89CA852285EFA0EFC2AD
:10E8400083274A009DC7DC438DC72285EFA0AFBA5E
:10E8500083274A00104083564400DC437115A30708
:10E86000A100B2961307F1004E86CA8526858297CD
:10E8700001C52380090031A08345F1002285EFA066
:10E880000FB941016F300FCDEF322FCB65711C08EE
:10E890003EC2B70780013EC41C0832893EC62A84A6
:10E8A000AE84EFF07FF14A85EFA0AFC68357A10099
:10E8B00089CFAA8550002285EFF0BFF50147814638
:10E8C0005000A6852285EF809FC359616F302FC904
:10E8D000EF320FC565711C088329C5013EC2B70719
:10E8E00080013EC41C082A84AE8432893EC6EFF003
:10E8F0003FF0638409024A85EFA0AFC18357A100AE
:10E90000AA8581CF50002285EFF0BFF001478146F4
:10E910005000A6852285EF809FBE59616F308FC35E
:10E92000EF32AFC165711C083EC2B70780013EC41B
:10E930002A841C0832853EC6AE84EFA08FBD835763
:10E94000A10089CFAA8550002285EFF09FEC0147F6
:10E9500081465000A6852285EF807FBA59616F30CD
:10E960000FC0EF328FBD444D91E88347450093B708
:10E970001700B307F0403E856F306FBE1845FD5756
:10E980007DDB97070000938707032A845CCB9705FC
:10E990000000938565D113858400EF80E05980C025
:10E9A00003474400814761FB1777FF1F23209742ED
:10E9B000D9B7EF32EFB68329C5014111032985008C
:10E9C0008147638B09080324090191452A8A22851E
:10E9D000EF807F9285452285EFA06FA38945AA8AA3
:10E9E0002285EFA0CFA2AA84EF809F9683A749003B
:10E9F0002A8B9DC79C438DC72285EFA0CF9F83A7FD
:10EA00004900A306A1001040835644009C4313070D
:10EA1000D100B296D6851306E1005285829709CDC2
:10EA200083570B002380F400A183A380F40023808C
:10EA30000A00A306010029A88357E100228523804C
:10EA4000F4008345D100A183A380F400EFA02F9CA4
:10EA50008347D100B337F0000347B900920701455F
:10EA60003D9BD98FA305F90041016F30AFAEEF3266
:10EA7000CFAC41111DE99777FF1F9387273580435E
:10EA800005C80440130984009DC55C4099C79C4B90
:10EA900089C726852EC68297B2459307803EB385E7
:10EAA000F5024A85EF80605521A0404DAA8479F88F
:10EAB00041016F30CFAA4A85EF80A0555C40EDDB65
:10EAC000DC4BFDD726858297E5B7EF320FA72A8466
:10EAD0003285EFA0AFA2AA852285EFF05FF96F30F3
:10EAE0000FA8EF328FA52A84AE84EFF01FFEA68513
:10EAF0002285EFF0BFBF6F308FA608413355B500B8
:10EB000005898280EF326FA31774FF1F1304042E50
:10EB10001C5C0111231701008D83858BA303F10079
:10EB20008327040B231801002319010003D7C70111
:10EB30003ECA3C002314E1007D572315E100035732
:10EB4000C4023ECC02CE2316E100EF802FE38357B0
:10EB5000E101231EA10093F707E093E71710231F9D
:10EB6000F1009777FF1F83C7072B85C30547014532
:10EB7000638AE7008347840393E727001777FF1F23
:10EB80002302F72A05616F308F9D814717D7000058
:10EB90001307471C85461306710085454808EF702A
:10EBA000E04B6DF183478403F59B1777FF1F230B21
:10EBB000F72685471777FF1F230FF724E1B7EF32BA
:10EBC000CF94977DFF1F938D6D2203A6CD063971DB
:10EBD0002A8981478144930600023357F600058B4A
:10EBE00001C7850493F4F40F8507E398D7FE83A744
:10EBF0000D0B231701022318010203D7C7013EDAC8
:10EC00003C102314E1027D572315E10203D7CD0206
:10EC10003EDC231901022316E10202DEEF800FD64B
:10EC20008357E103231EA102014593F707E093E711
:10EC30001710231FF1029777FF1F83C7C71DA9EF86
:10EC40009777FF1F83C7171E3EC69779FF1F9389CB
:10EC5000E9190144014D9D4A054B954B177CFF1F57
:10EC6000130C0C20977CFF1F938C0C1F03DAC90533
:10EC700063090A00EA85631459036685EFF0FFE72C
:10EC80001DC1050DA1478909E312FDFE2DE097770F
:10EC9000FF1F23A5071C014521616F30CF8A6285C4
:10ECA000EFF0BFE579DD3247B3878400E3F0E7FE9C
:10ECB0009C001306140006043E9413178A00935711
:10ECC0008A00D98FC207C183A30EF4FCA183230F4E
:10ECD000F4FC03A70D07B317AB01D98F1777FF1FFC
:10ECE000232EF71663047601328461BF15449777AB
:10ECF000FF1F83C72712138717009776FF1F238BE9
:10ED0000E61093161400230EF10017D70000130726
:10ED10006704814785067008CA854818EF7000347B
:10ED2000E34705F68347C10105451777FF1FA30396
:10ED3000F70E9777FF1F2380270FB9BFEF225FFEE3
:10ED40000111AA892E84EFD0EF9C2A899774FF1FA6
:10ED50009384C4096399090A9C5C414793F70703AC
:10ED60006393E70A1777FF1F0347370B894763EC65
:10ED7000E70883A7040B231701002318010003D71A
:10ED8000C7013ECA3C002314E1007D572315E10072
:10ED900003D7C4023ECC231901002316E10002CEA2
:10EDA000EF80CFBD231EA100EFC06FCD8357C101FF
:10EDB000230FA100914613D78700A207D98F2312F2
:10EDC000F1009777FF1F83D7070613D78700A207A5
:10EDD000D98F2313F10017D70000130727F78147B6
:10EDE000500095454808EF70602705889317240068
:10EDF00003C484036D985D8C9777FF1F238487027B
:10EE000005616F203FF5EF70B0781775FF1F130590
:10EE1000E501EF80002083A7040B9775FF1F83D5C2
:10EE2000A5FF03D5C701EF10E0279777FF1F83C722
:10EE300067FF93F60702014789E61777FF1F03571D
:10EE4000A7FD9776FF1F2391E6FE1777FF1F130795
:10EE5000A7F8184309CBC18B99C789451775FF1FC0
:10EE6000035585FB02979777FF1F23A707FA97772C
:10EE7000FF1F238207FA9777FF1F23AF07FC9777BF
:10EE8000FF1F23AD07FC9777FF1F23AB07FC83D73A
:10EE9000840393F7270C93E717001777FF1F2313BB
:10EEA000F7F883572903A18B99C3EF70E03F11C492
:10EEB0009777FF1F23AE07F4A1B78D471777FF1F82
:10EEC0002328F7F4EF902FA59305803EB305B502F4
:10EED0001775FF1F130585F5EF80201215B797777B
:10EEE000FF1F9387A7F0D85325C791C99777FF1FB6
:10EEF000238307F29777FF1F23A207F68280EF2272
:10EF0000DFE383C7F70241112EC685071777FF1F7E
:10EF1000A305F7F09777FF1F2399A7F09D47177771
:10EF2000FF1F2327F7EEEF900F9E2A84EF90AF9DEF
:10EF3000B24501E5EF902F9DAA85B305B440177542
:10EF4000FF1F1305A5EEEF80400B41016F203FE14D
:10EF500082809777FF1F938767E9D85331C7EF22E5
:10EF6000DFDD03C7F70205079776FF1FA387E6EAF1
:10EF700011CD8C5F0D470145898185899776FF1FEB
:10EF800023A8E6E8EFF09FDB6F207FDD8547930540
:10EF9000C0441775FF1F130565E91777FF1F232965
:10EFA000F7E6EF808005CDB78280EF221FD9177773
:10EFB000FF1F034747E68547631EF7009777FF1F4C
:10EFC0009387C7E283C7870393C787001777FF1F1D
:10EFD000230AF7E41775FF1F130545E5EF8060036B
:10EFE000EF807FEF99471777FF1F2323F7E297778B
:10EFF000FF1FA38407E29777FF1F238E07E0EF90A0
:10F00000AF8F930740063305F5029777FF1F23A7BD
:10F01000A7E06F20DFD49777FF1F83C7A7E0C18BDE
:10F0200099C7EF229FD1EFF0FFAD6F205FD36955F5
:10F0300082809777FF1F938767DBDC5381CBEF22BA
:10F04000DFCF8545EFF09FCF6F207FD1828017778C
:10F05000FF1F1307A7D901468146BA852148631EC1
:10F0600006019DCA2390A60083C7850393E7170076
:10F070001777FF1F2308F7DA05A08357C705631D1D
:10F08000F502F8598547B397C70093C7F7FFF98F83
:10F090001777FF1F2326F7DC9C5D9183858B85C73F
:10F0A0009777FF1F83C727D799EFEF221FC91D4509
:10F0B000EFF0FFB06F20BFCA81E699E39306C70562
:10F0C0000506090769BF8280EF22BFC48605AA84AE
:10F0D000B309B500977AFF1F938A0AD8054B977B2F
:10F0E000FF1F938BABD7214C639434039777FF1F9B
:10F0F0009387C7CF9C5F9183858B89CB9777FF1FC1
:10F1000083C767D181E72145EFF07FAB6F20FFC355
:10F1100003DA0400630B0A041779FF1F130909CDF2
:10F120000144CA8C8357C905639D4703A285568550
:10F13000EFF0BF9C11E5A2855E85EFF01F9C05C92D
:10F1400003A74C07B3178B00D98F1777FF1F23290D
:10F15000F7D083C78C0393E717001777FF1F2303AC
:10F16000F7CC05040909E31F84FB8904B5BF231EFE
:10F170000904C5BF1777FF1F0347E7C98547631A0F
:10F18000F700EF229FBBEFF05FE2EFF0BF976F2039
:10F190001FBD8280814785451306000293861700B4
:10F1A000B397F500E98F13F7F60F89E7B687E39772
:10F1B000C6FE01473A858280FD4785457D56B39658
:10F1C000F50013871700E98E1377F70F89E6FD170F
:10F1D000E397C7FE01473A85828089E901473A856E
:10F1E000828001473A8541016F207FB7EF22FFB44B
:10F1F00041112AC62E852EC4EFF0DFF9A2457D15F8
:10F200008547B397A700E39EF5FC32469377360017
:10F2100099C3719A11069777FF1F9387E7BC9443B0
:10F220003E871778FF1F130868BB89EA8327080009
:10F230009107F19B9776FF1F23A8F6BA0325880054
:10F240001843B307A700B3F7B702B387F540FD151E
:10F25000FD8D83274800AA95B306B600E3F3F6F8C0
:10F26000E371D5F82E979777FF1F23ADD7B63DDB17
:10F270003A858145EF207FAF2A87ADB71841977750
:10F28000FF1F9387A7B523A4070098C35841D8C38D
:10F290009777FF1F23AA07B48280EF227FA8AA8452
:10F2A00001441779FF1F130969B49309400EEF80D9
:10F2B0007FD56345A40001456F20DFA933053403E2
:10F2C0008327090B3E958357C501E38797FE050405
:10F2D000F9BFEF221FA49779FF1F938929B13E84BC
:10F2E000BA848347060003A7090041119D83058B5B
:10F2F0003D8F83C74401AE8A2A89F99BD98F238A1F
:10F30000F4001C44B685231204001CC02285328AF6
:10F3100036C6EF90DF8FB246D2853686EF90900BDF
:10F32000DC4883A509000840858B56869D8DEFD06B
:10F330003FCC61E918407D5583475700034767007C
:10F34000A207D98FC207C1872394F4006358F00A3B
:10F3500083C7440193F70703B5CBD04893771600D2
:10F3600003A609001D8E9777FF1F9387E7DE9C4356
:10F37000ADEB814641A003A70B0093172A00BA9773
:10F3800018409443834757008345670033F656017E
:10F39000A207CD8F6311F60283473700034647006B
:10F3A00003472700A207D18F4207D98FBD82B3F749
:10F3B0006701638AF604050AEF80DFC342059317ED
:10F3C0000A014181C183E3E8A7FA41BFA16A370B73
:10F3D0000200014A977BFF1F938B0BAFFD1A7D1B29
:10F3E000E1BF83C7440113070003854693F7070372
:10F3F000E391E7F8A2854A85EFD0FFCF41016F2066
:10F40000DF946155E5BF7955D5BFEF227F919774A1
:10F41000FF1F9384E4859C40D9EF9777FF1F938764
:10F42000679B9C436399070CEF80DFBE93078002C4
:10F430003305F5028945EFF05FDA41C99777FF1F81
:10F4400023ACA7A4EF801FBC9307400E3305F50241
:10F450009145EFF09FD835C99777FF1F23A0A7A448
:10F46000EF805FB201CDEF80FFB191450E05EFF067
:10F47000DFD621CD9777FF1F23A4A7A2EF801FCB54
:10F4800011CDEF80BFCAD9473305F5028945EFF0AA
:10F49000DFD405CD9777FF1F23AEA79EEF809FB5E2
:10F4A00091450A05EFF07FD30DC19777FF1F23AD7C
:10F4B000A7A0014521A8EF803FC29307800633052E
:10F4C000F5029145EFF07FD101E565556F209F88EA
:10F4D0009777FF1F23ACA7920144130A8006177980
:10F4E000FF1F1309A990B14AEF801FBF6364A402F4
:10F4F0009C40E38407F2EF803FBE9307A0043305EE
:10F50000F5028945EFF07FCD69D19777FF1F23A1E1
:10F51000A79C19BFEF805FBB89450605EFF0FFCBC5
:10F520004DD5B3094403032709024E9708CBEF805A
:10F53000BFB8330555039145EFF03FCA59D583272E
:10F54000090205041374F40FCE9788DB71BF977717
:10F55000FF1F9387A789884705898280C167FD17A8
:10F560006319F5009777FF1F9387478803A5070B5B
:10F570008280EF228FFCEFF05FD26F204FFE814739
:10F5800009C58347E501B337F0001777FF1F13075D
:10F59000E78518470983058B19C393E727003E8544
:10F5A0008280EF228FF92A84EFF07FFD8347E40108
:10F5B000AA851305940899E3130504039776FF1FA2
:10F5C0009386C6829442130615021307840213051C
:10F5D0009504EFD0CFC06F208FF8EF226FF49774AF
:10F5E000FF1F9384A48098442A892E840983058B65
:10F5F0009C4019C76314F5006380050E014401A205
:10F60000E3FEA7FE1387A702E36AA7FE850763FC54
:10F61000A70883A9440BEF80FF9613163500814598
:10F620004E85EF208FF49767FF1F23A1277D9767F3
:10F63000FF1F23AF077A49CC9C4493E74700176725
:10F64000FF1F2329F77A9777FF1F238D0780630F0A
:10F65000040C9767FF1F23AB277901440549EF800E
:10F660007F926341A40AEF80FF9493050006B3C51F
:10F67000A502B7F73600938707E81765FF1F130544
:10F68000A57E416901449309400E7D19B385F502B9
:10F69000EF70B016EF801F97634FA4080145EF305D
:10F6A00040700544A9A86398A7029DE583A9440B6F
:10F6B000EF805F8D1316350081454E85EF20EFEA10
:10F6C0009767FF1F23A427739767FF1F23A2077263
:10F6D0009C44ED9BADB785C51767FF1F034787782F
:10F6E0009307F005E3FCE7F021F8EF60F03C6DD103
:10F6F0009C4493E707021767FF1F232DF76E2285AF
:10F700006F204FE583A7440B131534003E958357B4
:10F71000050081CB8347250099C721468145EF200D
:10F72000CFE405042DBF23012501E5BF9767FF1F27
:10F7300023A0076C0DBF3305340383A7040B3E954C
:10F740008357C50163842701EFF0BFE5050499B72E
:10F75000EF22AFDEEF801F86130400063345A402BC
:10F760009764FF1F9384846883C784073E9513754D
:10F77000F50F9767FF1F2387A76E9307F00563E7D1
:10F78000A7020545EF30E061EF80DF823345A40238
:10F79000B7F53600938505E8B305B5021765FF1F79
:10F7A0001305856CEF7070056F206FDB9C44054579
:10F7B0008983858B81CBEF904F8888408145EFF01E
:10F7C000DFE1DDB7EF30E05DC5B7EF226FD51304A1
:10F7D00095082A8913069005A28513050503EF9065
:10F7E000603F1306900581452285EF200FD84A859A
:10F7F000EF30C0548144176AFF1F130A2A5F930A2F
:10F800008002EF803F8163C4A4006F20AFD43384B3
:10F8100054038327CA0A3E94035704008357C9013F
:10F820006317F702834744009DC39309640145466B
:10F83000CE8513055400EF90E039454681454E854D
:10F84000EF20AFD2228523020400EF300057850459
:10F850004DBFEF228FCE9767FF1F938767419C4371
:10F860002A8491C70DC50355C501EFE00FC29777F4
:10F87000FF1F9387678E9C4389CBEFB0DFD085470E
:10F880006315F5002285EF50C05D6F204FCD4165B7
:10F890007D15E1BFEF226FCA1764FF1F13040455E3
:10F8A0004440938714001767FF1F2323F754EF305A
:10F8B000605E1C448983858B9DE75840B7E7B000A4
:10F8C0009387075063F1E7020145EFF01F9D01CDDB
:10F8D0000545EF809FF6084085450505EFF0FFCF11
:10F8E0000145EFF01FF726856F206FC7EF224FC34A
:10F8F000A1642A8901449769FF1F9389E95CFD147B
:10F90000338AA500EF800FEF6344A4006F208FC4FB
:10F9100003A7090093172400BA979843658F4207FD
:10F920004183634C2701635A470123800700A3806A
:10F93000070023810700A38107000504E1B7EF2238
:10F94000CFBC83594500C547411163F537310441A8
:10F95000C1E533853401834785FF034795FF03489D
:10F96000B5FFA207D98F0347A5FFC2072207336758
:10F970000701D98F0347C5FF0348D5FF2207336727
:10F9800007010348E5FF0345F5FF420722083365F9
:10F99000A800498FB98F1767FF1F1307A750176873
:10F9A000FF1F130828523A85832807006384172B0A
:10F9B0001107E31B07FF1767FF1F1307A750184323
:10F9C0001318270042951CC10507A1473367F702AA
:10F9D0009767FF1F23A8E74E93F73500139747005B
:10F9E00083474601C16B368993F7F7FCD98F328480
:10F9F0002E8A230AF600814A176CFF1F130C0C3F56
:10FA0000FD1B976CFF1F938CAC26176DFF1F130D0A
:10FA10002D4CEF802FDF63C7AA00E15426854101FA
:10FA20006F206FB21308400EB3870A0303280C0B34
:10FA3000B30DF800638E0D2083D7CD01638A772143
:10FA400083A70C00014B639707169767FF1F9387E7
:10FA500067389C436390071683C7040003C70D04EF
:10FA600093F7F707631BF71ACA872287CE86268685
:10FA700093859D0613851D04EFF0BF85631F051850
:10FA800083D7CD01032709002320B4012312F400FA
:10FA9000FD572313F4008347170093F6F7078347B6
:10FAA000D40093F707F8D58FA306F40093F7F70770
:10FAB000B337F000B307F0402307F4008347170083
:10FAC0009D839396370083474401DD9BD58F230A9E
:10FAD000F4008347370083464700A207D58F83464B
:10FAE0002700C206D58F1CC88347770003478700CD
:10FAF000A207D98F2315F4000D476304EA00BD5413
:10FB000091DF93870710C207C1831307B00FBD545D
:10FB1000E376F7F0EF800FC98144E31105F09766B3
:10FB2000FF1F83C6A63A938716001767FF1F230F90
:10FB3000F7381767FF1F13072739231BD400939744
:10FB40002600144303578400E175BE96A16713860F
:10FB5000F7FFB377C70098426D8FD98F9CC21848C2
:10FB6000F18F3E07D98F9CC2EF80CFC89767FF1FE8
:10FB700083C7C73533F5A7029767FF1F2388A734CC
:10FB800071BD9307A004B308FB0283270D00BE9844
:10FB900003D7080083D7CD01631DF70083C7040096
:10FBA00003C7880093F7F707630BF70083C7FD01CE
:10FBB0009DEB050BEF804FD2E345ABFC71BD938508
:10FBC000980113859800CA872287CE86268646C666
:10FBD000EFF02FF0B24879F98347440193E74700EB
:10FBE000230AF40071BD83C7040003C7980293F78A
:10FBF000F707E310F7FCCA872287CE86268693850F
:10FC0000A8031385A802EFF0CFEC45F58347440124
:10FC100093E72700230AF400C1B783C7FD018DCB0A
:10FC200083C7040003C79D0993F7F7076312F70220
:10FC3000CA872287CE86268693852D0C1385AD092B
:10FC4000EFF02FE911E58347440193E7270049BF0F
:10FC5000850AC1B3FD54D9B3EF22AF8B79718354B8
:10FC60004500AA8B2E84B28AEF80CFBB5905634929
:10FC70009504B7E4040003A90407EF80AFBA59055F
:10FC80004205418102992A8905CD2AC6231801001F
:10FC9000EF804FB959052319A10061468145280815
:10FCA0009769FF1F938989144ACAEF200F8C23029A
:10FCB000810203A48900058819E4BC544A8582970F
:10FCC00045616F208F8874003008D6855E85EFF01F
:10FCD0001FC765F56800EF807FF1176AFF1F130AE1
:10FCE000AA4783270A00AA84035B010189CB8947BD
:10FCF0006397FA00835501025E85EF50203003556B
:10FD00002102EF704FC819E503552102EF708FD41F
:10FD10003334A000931764000344C1022C08680028
:10FD20001374F4FB5D8C23068102EF60B056E95733
:10FD30006314F5028356E1029767FF1F9387C71884
:10FD40009C43139726006176BA979843718F98C3A6
:10FD50009767FF1F238CD716831721026345F00096
:10FD600085476396FA00B25793F7070C95E7D24799
:10FD7000C2040347C102C180BE9426C62318610194
:10FD800013770703C147631DF700834751020547F7
:10FD900093F7F7076390E704B7E70400BC5739BF50
:10FDA00092570544A18393F7F707E377F4FE15C74D
:10FDB0008347C1021307000293F707036397E70025
:10FDC000EFB06FFC8547E319F5FC8347C10293F759
:10FDD000070389CFEFB0AFCA21A8EFB08FD7E309EF
:10FDE00085FCEFB04FFAE31985FAD9B7EFB0EFD839
:10FDF000AA8501460545EF707FF82A8451DD8347C7
:10FE0000C102414793F707036384E7023247834700
:10FE1000170093F707F8A300F7003247925783467D
:10FE20001700A18393F7F707FD17D58FA300F700FD
:10FE300003560101B245130BC4005A85EF80DFDF82
:10FE4000E24A130690058347C10283C4EA01918BFD
:10FE5000B384C40213851404569595C35444B387E0
:10FE60009A0083C7070403C70600137707F82380A7
:10FE7000E600584483460700D58F2300F700B257A9
:10FE800003A609008146858B1D8EDA85EFD0EF9B96
:10FE900015E9B25783A50900484413869406858B5B
:10FEA00056969D8DEFD0CF9411ED83270A0099EFE0
:10FEB000B257054791838D8B6387E7049DCF094730
:10FEC0006389E7042285EF80DFF8F9B5EFB0AFEB87
:10FED00085476309F5008347C102414793F707034C
:10FEE000E398E7FC835521025A85EF40907C69D165
:10FEF00083172102E35EF0FAF1B7EFB08FC57D15ED
:10FF00001335150061D1014681452285EF70FFEF61
:10FF100055BFEFB04FE7E5B7EF123FE29764FF1F21
:10FF2000938444EE2685EF809FEB2A8419E16F10BD
:10FF30001FE31305C40005468145EFF0FFD122857C
:10FF4000EF803FF1C5B7EF125FDF4111AE842A8425
:10FF500093079503130715019306F10005466C00FE
:10FF6000268523060100EFD0CFBE1DEDA6854146B4
:10FF70002285EF8030468347F100930514022685E1
:10FF80002308F400EFD06FC805E19767FF1F938740
:10FF9000A71C9C4389EF1306940497C50000938522
:10FFA000E5DB2685EFD08FD441016F105FDB1306B0
:10FFB000940297C500009385E5DA2685EFD00FD32C
:10FFC00079D9DDB7EF12DFD59767FF1F9387C7EFAA
:10FFD0008043AE84B289368AAA8AEF80AF81131635
:10FFE000250081452285EF105FD89767FF1F238F7B
:10FFF00007EC9767FF1F938767DF03A4070B13F7CF
:020000040001F9
:1000000014003E89230FE400CE8525C7130594080C
:10001000EFF07FF301C555556F10DFD38947A30F6C
:10002000F4009767FF1F938727139C4303278900DA
:10003000858093B7170086072300F402231E54011E
:100040009767FF1F23A447DB85889377B7FF99C085
:10005000936747001767FF1F232EF7D82285930762
:1000600000061767FF1F230FF7DEEFF08FD3014560
:1000700065B713050403EFF01FED45D569BFEF1217
:10008000DFCBFD572310F5002311050023120500D7
:10009000231305001306200481452105EF10FFCC32
:1000A0006F10FFCBEF12DFC74111AA84014417691B
:1000B000FF1F1309E9E19309A0042EC6EF80CF8149
:1000C000B2456344A40061550DA033053403832772
:1000D00009003E9583572500639CB70083570500B0
:1000E00063989700EFF0BFF9014541016F109FC67B
:1000F0000504E1B7EF12DFC29767FF1F938787CD33
:100100009C434111AA842E84B28903592500C1C39E
:100110009767FF1F83D747D0639B2707EF700F8632
:100120002A8903D5240093051002B305B40285473C
:100130002302F10093578900A302F1009357850031
:10014000A303F10083D744002304A100254613D75D
:1001500087002305F10083D76400A304E1004E85E6
:1001600013D78700A305E1002306F100138795004C
:1001700093879501A105B386B400A6974C002697F6
:1001800023032101EFD0EF9C41016F10BFBCEF6052
:10019000FFFE51BFEF12DFB84111AA840144176975
:1001A000FF1F1309E9D29309A0043AC636C432C22C
:1001B0002EC0EF707FF282451246A246324763445A
:1001C000A400615599A0B307340303250900AA9739
:1001D00003D8070003D5C4016310A80495E91DEEF8
:1001E00091CA03C6E401930510023306B602250640
:1001F0003E9690C2014511CB83C6E401130610025E
:10020000B386C602E506B6971CC341016F109FB4C2
:1002100003D52700E305B5FC050441BF83C5E40110
:1002200013051002B385A502BE9583C58500230082
:10023000B6007DB7EF12DFAE5C4141112A8403DACC
:100240002700C167FD17AE843289630CFA0026854A
:10025000EF807F9A8D4763EDA7007D5541016F10B8
:100260007FAF2E85EF803F999D47E3E2A7FEF5B76C
:100270005C40268583D54700EF809F90835584009E
:100280002685EF80FF8F8D452685EF803F8EAA89DA
:10029000EFF04FE0935705012380F9009357850055
:1002A000A380F9002381A9005840C167FD17834549
:1002B000A7006314FA0093E505082685EF801F8FD9
:1002C0009767FF1F938707B19C430840D9CF8347A7
:1002D000B400858BD9CB78003400130671008145BA
:1002E000EFF05FEB1DC98347B400184093069005FB
:1002F000F99BA305F4008347E701B387D702B30650
:10030000F70083C60604A303D100938617049387DE
:100310009706BA96BA9736C43EC61764FF1F1304F1
:10032000E4AC1C440C4026858983858B9D8D8347D6
:1003300071009E05DD8D93F5F50FEF803F871C441E
:10034000104022458983858BCA861D8EA685EFC005
:10035000DFCFE31505F01C440C403246898388400A
:10036000858B9D8DEFC0DFC8D5BD8347B4001307D3
:100370009005F99BA305F4008347E501B387E702E5
:100380003307F50003470704A303E10013871704AD
:10039000938797062A973E953AC42AC6BDBFEF12A7
:1003A0003F98032A45009307F00FAA840347AA0049
:1003B000AE89328436896316F700EFB06FAB230540
:1003C000AA00938AC9000146D6852685EFF09FE6EC
:1003D0002A8A21E51767FF1F130707D81843DC4057
:1003E00039C383C6A7000547638FE60283D547005C
:1003F0005685EF40102C05C9DC40839747006354B5
:10040000F00201CC1C4089C74A868145014582978C
:100410005C4081C7CA85014582974E85EF807FA3E6
:1004200052856F103F93DC4003D54700EF60BFD586
:1004300001E9DC4003D54700EF60DFE181471DCDD6
:1004400019C41C4089C74A868145014582974E855B
:10045000EF807F9FAA851765FF1F1305A59AEF8080
:10046000DF9511C45C4081C7CA8501458297176535
:10047000FF1F13056598EF60F0368547D840854625
:100480000346A700E30BD6F8031747006353E000C9
:10049000C9F74A86A2854E85EF703F97BDBFEF1220
:1004A0003F88AA8401441769FF1F130969A29309B1
:1004B000A004130A9508EF703FC26344A4000145ED
:1004C00035A033053403832709003E958357250063
:1004D00099E30504CDB70357050083D7C401E31A98
:1004E000F7FE52868545EFF0FFC065D56F109F86F9
:1004F000EF121F83AA8401441769FF1F1309499D46
:100500009309A004EF705FBD6344A4006F109F8443
:1005100033053403832709003E958357250081CF97
:1005200083570500639997009305950213061002FF
:100530002105EF80206A0504F1B7EF121F80034701
:10054000E5012A848347F5016307B70089E7814500
:100550002E856F10DF80230FB400054781C9E39813
:10056000E7FE8947A30FF4008545DDB7638BE702FB
:100570000947E39FE7FC2285EFF02FA59767FF1F50
:10058000938747859C4399E79757FF1F9387476E4B
:100590009C4389C70355C401EFF09FF5A30F0400E6
:1005A000E1B755D6C9BFEF12AFF7EFA0FFEE854711
:1005B0006312F508EF80EFCC1764FF1F1304C4B972
:1005C0001C4081CBEFA03FFC89476304F5001C4031
:1005D00082979757FF1F9387E77F9C43B9CF8297F6
:1005E0009757FF1F9387C7689C4391C382971754FF
:1005F000FF1F1304A47F8327040B83D4C701EF607C
:10060000FFB78327040BAA85144003C6E7011C44E7
:100610008983858B99C31366260026854169EF403F
:10062000C03D8144D9497D19EF705FB063CAA40011
:100630006F104FF2EF800FCA41B7EF705F884DB770
:10064000B38734030327840ABA9703D527006308C6
:10065000250103C6470183D50700EF40A03B850471
:10066000E1B7EF12EFEB01449754FF1F9384047836
:100670001309400EFD59EF70FF98634FA404014425
:100680009754FF1F9384847613098002FD59EF70FD
:100690007F98634CA40401449754FF1F938404750E
:1006A0005949FD59EF709FA8634AA40497F5FFFFCD
:1006B0009385450A1755FF1F1305057BEF60D0078B
:1006C00097050000938585851755FF1F1305C57293
:1006D000EF6050056F100FE83307240383A7040B66
:1006E0000504BA97239E370179B73307240383A7FC
:1006F000C40A0504BA972390370151BF3307240376
:1007000083A7840A0504BA972391370161BFD441B6
:100710000387350085473356F5026377E600A54821
:1007200099E7238006008280B387E702EDB733584C
:10073000F502038735003375F502B3D7E7021307D7
:10074000000363DA080103C6050013077003118A6A
:1007500019E21307700585064297A38FE6FEC9B715
:1007600018451C416376F7005C41BA972380B700B7
:100770001C4585071CC58280EF122FDC4111AA871A
:100780002E85B285368636C6829763480500B24606
:10079000158D3335A0003305A04041016F102FDCCB
:1007A000EF120FD8056941112A8A2320060001445F
:1007B0008149975AFF1F938A2A74056B7D1932C6A7
:1007C0002EC4EF703F85AA84EF70DF832695A24583
:1007D00032466346A4004E8541016F10AFD703A790
:1007E0000A0093171400BA9703D7070033776701FD
:1007F00001E71CC20504E1B703D707009356D700F1
:10080000858AE39946FF33772701E315B7FEBE8952
:10081000D5B7EF128FD201112EC6B2843689EFB050
:100820002FEE2A84615501C8B24589E9232E0400C0
:1008300023200402014505616F106FD2A1463008E4
:10084000CA852685EFF05FF37DF583578101035755
:10085000A101231EF4008357C1012310E4022311D8
:10086000F4028357E101D207D1832312F4028357A4
:10087000E1011397370163560700FD57231FF4006A
:100880005DBF231F040045BFEF128FC91754FF1F20
:100890001304C4558327040B03D7C701C167FD1791
:1008A000630EF7109767FF1F9387478B9C4381C7A1
:1008B0000545EF406077C1690149930A400EFD1973
:1008C000176BFF1F130B4B89EF70CFF3634BA90E10
:1008D0001757FF1F034707599307F00563E4E70223
:1008E000EF704FED93050006B3C5A502B7F73600CC
:1008F000938707E81755FF1F13050557B385F502C2
:10090000EF60A06F81451705000013058520EF609B
:10091000DFF8EFB0EFDE01CD0357C50109CB035778
:10092000E50111C78347050299C3EF60A06BEFB0E3
:100930006FDE31C51757FF1F0347875F9757FF1FAC
:100940009387075F0DCF03C717002304E50003C794
:100950002700A304E50003C737002305E50003C70C
:100960004700A305E50003C757002306E50003C7BA
:10097000670083C77700A306E5002307F5001C4442
:1009800093E717001757FF1F2326F7465C4085E7BC
:10099000EF708FEF0DC1EF702FEF44402A89EF7099
:1009A000AFEE33F5A4025C40FD17CA97898F175745
:1009B000FF1F232FF7420145EF70DF9F01456F10A6
:1009C0006FB9B30459038327040BBE9483D7C401C2
:1009D00063883703138A0403D2855285EFF0AFD6BC
:1009E00005E183C7F40199CF938594082E85EFF034
:1009F0008FD509C91306900581455285EF10EFB6D2
:100A00000509D9B583270B00268593B717008607FC
:100A10002380F402EFE0FFB8E5B7854763F8A7004D
:100A20009307F5FFBE953305A040E98D2E858280A2
:100A30009841C167BA9713D707016304A7009CC107
:100A400082804207998FE5BFEF122FAF41112EC66A
:100A50003284B684EFB00FCCE15701C9B24591E9B9
:100A60009757FF1F2386074C81473E8541016F1032
:100A70000FAF9D461756FF1F1306964BA68522857E
:100A8000EFF09FCFAA8775F105479756FF1F238187
:100A9000E64AE1BFEF12CFA8411191E99757FF1F36
:100AA00023A807340144228541016F10AFAAB685FF
:100AB00032858D467000EFF03FCC2A846DF5834778
:100AC000D1000347E1001759FF1F13092932A2077C
:100AD0004207D98F0347C100D98F1757FF1F23291A
:100AE000F730EF706FDA61D1EF700FDA83244900CD
:100AF000AA89EF706FD933F5A40283274900FD1747
:100B0000CE97898F1757FF1F2324F72E69BFEF1247
:100B1000CFA21C45AA8491CFD84B01CF83D74700E1
:100B200089CBEF601F92AA8509C588446105EF60F3
:100B3000C04C9757FF1F9387E7299C43014489EFD7
:100B40006F10EFA19C4813171400BA9703D5070044
:100B500019C1EFE0CFCF0504EF70CFC7E344A4FE87
:100B6000C5B7EF128F9D011185E9EF605FDA01448F
:100B70009757FF1F23A807309757FF1F23A607305B
:100B80009757FF1F23A407309757FF1F23A2073053
:100B9000228505616F10AF9CB6873285C94670000B
:100BA000BE85EFF07FBD2A8465F541469305E100DF
:100BB0001755FF1F1305052DEF80C0010355C10018
:100BC000EF608FD7F1B78DE19757FF1F23A0072262
:100BD0009757FF1F938787219C470145ED9B175728
:100BE000FF1F2329F7208280EF122F954111B68530
:100BF000328595463000EFF03FB815EDA247175704
:100C0000FF1F2325F71E9757FF1F9387271E944723
:100C1000B24713F7B6FF13F6170019C213E74600E1
:100C2000858393F7F7079756FF1F23A5E61C1757F1
:100C3000FF1F2309F72241016F106F92EF124F8EB1
:100C400003841500DC412A89AE8485070387F7FFFA
:100C500019C36340800C8387240091C763558000CB
:100C60007D14620461849C40370700FF0907F98FF7
:100C70003707001009076392E70A6355800079146B
:100C80006204618483C70400858B95E39379F40F34
:100C90004E8A93178A01E187634AF008A28763535B
:100CA000040081473384F9407D14620461848385A4
:100CB000240081C54A85EFF0BFAA9C40370700FF9A
:100CC0000907F98F370700100907639AE7069305AC
:100CD00000034A85EFF0DFA883C704009305800571
:100CE000918B99E3930580074A85EFF07FA783C72F
:100CF0000400858B81CB1374F40F93178401E18773
:100D00006347F004C04005048305F4FFA1E96F10B8
:100D10006F847D14620461840DBF370700080907E2
:100D2000E392E7F6E35080F67D1499BF9305000245
:100D30004A857D1AEFF0DFA2137AFA0F99BF3707C1
:100D400000080907E395E7FA9305000371BF9305CF
:100D500000034A85EFF0DFA07D1471BF4A85EFF0F4
:100D60003FA055B7EF027FFDEF70CFAA2A84EF7046
:100D70006FA9229589450605EFE02FC6E55711C5F5
:100D80009757FF1F23AAA71681473E856F003FFD97
:100D9000930700026306F5005D1513355500828048
:100DA00005458280EF02DFF74111AA892A891304E1
:100DB00019008304F4FF32C62EC42685EFF05FFDD0
:100DC000A245324659E19307D0026392F4088304A6
:100DD00004000548130429009377F6FEC9E793073A
:100DE0000003639FF40E830704001307800593F745
:100DF000F7FD6399E7068304140041460904B7062A
:100E000000806314080093C6F6FFB3FEC602814754
:100E1000254F654EFD5F33D3C602138704FD63681B
:100E2000EF06BA8463D5C408630DF5017D55636A86
:100E3000F3006394670063C69E000545B307F6029E
:100E4000A69705048304F4FFC9BF22898DB79307D1
:100E5000B0020148E392F4F8830404002A881304E2
:100E600029009DBF01CA8947E31BF6F893070003D9
:100E7000E397F4F8830704001307200493F7F7FDC2
:100E8000639BE70483041400094609048DBF13E73C
:100E900004021307F7F9636CEE009388F4FB130761
:100EA000700363741E0113077005998CA5BF7D57ED
:100EB0006300E50263040800B307F04091C519C15F
:100EC0009309F4FF23A035013E8541016F009FE89F
:100ED000B687FDF5D5BF9304000315F2214605B78B
:100EE00019FE294629BFEF02BFE3011161540DC568
:100EF0003284AE89414681453689EFF0BFEA9314CA
:100F00000501C180639E09002685EF30102B014446
:100F100001C58145EF205016228505616F009FE3D2
:100F20002285CD467000CA85EFF01F852A846DF5B5
:100F30002685EF30902809E90356C1008345E10179
:100F40002685EF20500B01C941469305E1001105AC
:100F5000EF705048D1B75D54C1B7EF027FDC01118B
:100F6000E15401CDB284AE89414681453689EFF026
:100F70007FE32A84639709008144268505616F0019
:100F80007FDD2685D1467000CA85EFF0EFFEAA848A
:100F90006DF58357C100EDD3EF700F8E42059317A7
:100FA00004014181C18363F9A702EFB08FB6420407
:100FB000E14741803304F40241460C082A941305AA
:100FC0004400EF7030418357E1002311F400835750
:100FD000C1002310F40055B7E55445B7EF025FD4C4
:100FE0007971E15415C53284AE8941468145B68494
:100FF000EFF05FDB1319050113590901639E090026
:101000004A85EF401065814401C58145EFB02FB19D
:10101000268545616F001FD4A685930630027000B7
:101020002285EFF06FF5AA8465F54A85EF4070627E
:101030002A8411E54A85EFB04F8C2A8431C5835745
:10104000C10023112401930964002310F400834795
:10105000E1009305F10041462302F4004E85EF7054
:1010600070371309740141469305F1014A85EF7009
:101070007036930554004E85EFC04FBF9305640151
:101080004A85EFC0AFBE69B7DD5459B7EF025FC9FB
:10109000797111E5E154268545616F00BFCBB284BB
:1010A000AE89414681453689EFF0DFCF131A05013D
:1010B000135A0A015285EFE06FCA2A846398090027
:1010C00071D98145EFB02FB48144F1B726859306DD
:1010D00010027000CA85EFF02FEAAA844DFD31C8D6
:1010E000B2479305D1004146858B230FF400B247E8
:1010F00013050403858393F7F707A30FF400EF703C
:10110000702D41469305D10113059408EF70902C82
:1011100059B73304690383A70A0B3E948357C4016C
:10112000638337030509EF60FFEDE344A9FEDD5457
:101130009DB7C1690149975AFF1F938A2ACB130BA8
:10114000400EFD19CDB7231E440159BF49CDEF0212
:101150003FBD4111B289AE8441468145368AEFF0E8
:101160007FC4931A050193DA0A010149175BFF1F37
:10117000130BCBC7EF601FE1634AA9000145ADCC5B
:1011800081441759FF1F130969C681A883274B0B98
:10119000131439003E9483570400638857050509EA
:1011A000D1BF8327490B139434003E948357040026
:1011B00085E72310540191467000D2854E85EFF0EB
:1011C000AFDB1DE9B24713978700E1832183858B4D
:1011D00058C02301F4000DA08504EF60BFDAE3C21C
:1011E000A4FC5D5511A861558280F1F4214681452A
:1011F0002285EF009FB7014541016F00BFB519710E
:10120000D2C4130AC10686CEA2CCA6CACAC8CEC60C
:10121000D6C2B6D6BAD8BEDAC2DCC6DE52C4638144
:101220000524FD151C102ACC2ECA02CE3EC89304FC
:10123000B0021549A94983050600130416009DE173
:10124000F2465247E24763FBE620B6972380070049
:101250007245F6406644D6444649B649264A964AFF
:1012600009618280930750026386F5004808EFF019
:101270002FCFF5A88357C10023070100014593F73D
:10128000C70F2316F10081450148014701468146F9
:101290009308D00213030003130E300205048307E2
:1012A000F4FF99C7638C970463C3F404638BC70589
:1012B00001CA0346C100858A799AD18E2306D100DE
:1012C000630908008346C100098BF59A558F2306F0
:1012D000E10019C12307B100138707FD1377F70F4A
:1012E000A54663E2E6068146A545294535A0E38784
:1012F00017FBE39F67FA0546FD564DB70545854543
:1013000071BF05487D5759BFB386A6020504830700
:10131000F4FFBA96E206E18613F7F70F130607FD0E
:101320001376F60F63E5C500138707FDF1BF1306BB
:10133000F7F91376F60F636EC902138797FAE30580
:1013400037FDA306D100130790066385E704634BBE
:10135000F706130780056384E70A6345F702E38114
:1013600007EE1307500293055002E381E7F022864F
:10137000D9B51307F7FB1377F70FE364E9FC13877D
:1013800097FC75BF130730066386E70A130740060C
:10139000E39FE7FC03250A00A947A307F100930A8E
:1013A0004A00635805009307D0023305A040230785
:1013B000F1006C00EFF0AFB56C004808EFF01F884B
:1013C000568A75B713073007638EE7066341F70245
:1013D0001307F006638EE70413070007E399E7F8A5
:1013E0000347C100136727002306E10009A813077C
:1013F0005007638BE70213078007E39AE7F69387AA
:1014000087FA414793B71700A307E1001397270016
:101410008347C100ED9BD98F2306F100930A4A0050
:101420006C0003250A0079B7A947A307F100FDB7AF
:10143000A147E5BF83050A004808930A4A00EFF078
:101440002FB2BDBF83270A006C0048083EC8EFF0EA
:10145000EFFE1C10930A4A003EC89DB7BA97FDB331
:101460000145C5BBEF027F8D2A883685834648003B
:10147000BA8703475800A206D98E328717B60000F4
:101480001306869089E517B600001306A690BE8560
:10149000EFF0FFD66F00BF8C9757FF1F9387C7A849
:1014A0009C4381CFEF027F89D843B2862E861847AE
:1014B000AA853E8502976F009F8A61558280EF0260
:1014C000DF878357050039712A84231EF100834783
:1014D00045009305650041461305F101230FF10016
:1014E000EF70406F9305740141461305F102EF70F0
:1014F000606E8356240017B600001306E691E5459A
:101500000A85EFF0DFCF6C08130630020A85EFF092
:10151000BFF821616F00BF84EF023F8239712A84D6
:101520009305050341461305D101EF70A06A9305A9
:10153000940841461305D102EF70C0698347E40166
:101540000347F4018356C401858B0607D98F17B66C
:1015500000001306268DE5450A85230EF100EFF005
:101560001FCA6C08130610020A85EFF0FFF2216112
:101570006F00EFFEEF02CFFA37040001B70400FF5F
:101580000111814A1759FF1F130949867D14938958
:10159000F4FF17BA0000130A6A8DEF60BF9E63C59F
:1015A000AA0005616F000FFB8327490B13973A00D0
:1015B0003E978347370095CF5C43A30107005286CF
:1015C000B3F687008247E5454800E58FD58F3EC0DA
:1015D00083462700B3F73701858AE206D58F835605
:1015E00007003EC0EFF0BFC111468A854800EFF00A
:1015F000BFEA850A5DB7EF024FF401468145EFF07F
:10160000BFE96F00CFF583576500638E071A1D7120
:10161000A2CCA6CACAC886CECEC6D2C4D6C2DAC0AA
:101620005EDE801013F717003289AA8431CBF99B54
:101630002313F500EF601F9906053D0541990A8BBC
:10164000C16A3301A1408A8B8149014AFD1AEF60CA
:101650007F97634CAA0C7947930604FB17A60000FA
:101660001306C67FCA852685EFF0DFDF638F090C7E
:1016700013961900DE85130504FBEFF0FFE15A8194
:1016800083D7640013F7270021CBF59B2393F40045
:10169000EF605F9406053D0541998A8A3301A140B8
:1016A0000A8B8149014AEF60FF926345AA0A6547A8
:1016B000930604FB17A600001306C67ACA85268582
:1016C000EFF05FDA6387090A13961900DA851305CC
:1016D00004FBEFF07FDC568183D7640013F74700EB
:1016E00005CBED9B2393F4006547930604FB17A6F7
:1016F000000013066677CA852685EFF0BFD69C44A6
:1017000081C703D747003DEB130504FBEFF0BFEEA5
:10171000130104FAF6406644D6444649B649264ABF
:10172000964A064BF25B25618280DC4413171A004F
:10173000BA9703D707006308570193971900DE97FC
:101740002390E7008509050A19B7130504FBEFF09C
:101750009FEA35B79C4813171A00BA9703D70700BA
:1017600019C793971900DA972390E7008509050AAE
:101770001DBF130504FBEFF01FE8B1BF2314E4FA0B
:1017800003D767008326C4FA2146520751832315E5
:10179000E4FA370700F0758F9447930584FA130530
:1017A00004FB92069182558F2326E4FA83C77700C3
:1017B00013F707018347F4FABD9BD98FA307F4FA07
:1017C000EFF09FCDB1B78280EF02AFD41744FF1F77
:1017D0001304C4610444797193F7F4FB1747FF1FA6
:1017E000232AF76093F70404A1C78588A1E097A98D
:1017F00000009389A967EF60EFF863DBA4028327F9
:10180000440B139934003E998356090091CE4E86BD
:10181000E5454808EFF0BF9E4808EFF0DFDD2146C0
:1018200081454A85EF006FD48504F1B7EFF09FD46E
:101830001C4413F7F7F79746FF1F23ADE65A93F7BB
:1018400007086397071E1C4413F7F7EF9746FF1F1F
:1018500023A2E65A13F707106318071E184493775C
:10186000F7DF9746FF1F23A7F6589376072095C604
:10187000058B630A072018408983858B3ACA034782
:10188000840715464C080607D98F17A500001305D5
:10189000A55A230CF100EFF03FC01C4413F7F7BF2B
:1018A0009746FF1F23A8E65493F707408DC383573D
:1018B00044000D464C08231AF1008357640017A515
:1018C00000001305A557230BF100EFF0FFBC1844EF
:1018D000FD749387F47FF98F9746FF1F23ACF65072
:1018E0009317470163DF0700EFA08FE119C9835603
:1018F000C5016391061A17A500001305A554EFF062
:101900009FCF1C447D777D177D8F9746FF1F23A3B4
:10191000E64E13973701635A0702858B6388071CCD
:10192000EFA04FDF1DC118458347E5001D463ACAA9
:101930000357C5004C0817A5000013052551231CAB
:10194000E100230DF100EFF03FB51844F977FD17E2
:10195000F98F9746FF1F23AFF6489317270163D9E6
:101960000700814517050000130525CAEF50FFF257
:101970001844E177FD17F98F9746FF1F23ACF64611
:101980009317070163D30702EFA0BF982A8481440D
:1019900017A900001309094CEF600FEE939704019B
:1019A0004205C183418163EAA71445616F00EFB925
:1019B00083A70A0093141900BE9483D7040033F759
:1019C00067011DCF1396170133F77701B3F637017F
:1019D0006352060417A600001306064409E717A67B
:1019E000000013062644E5454808EFF05F814808EB
:1019F000EFF07FC083D70400B3F747012390F400D2
:101A00000509EF602FE1AA84EF60CFDF2695E3415F
:101A1000A9FA15BD368519C7EF40A04361DDEFF087
:101A20001FAAC9BFEFD09FB371D5EFF0FFAED9B7F2
:101A300085697D7A0149974AFF1F938AEA4B056BB6
:101A4000896BFD197D1A75BF858B9DC7EF500FF30C
:101A5000231AA10041469745FF1F9385A542130510
:101A60006101EF70201749464C0817A500001305C7
:101A7000253CEFF07FA2DDB317A500001305453B21
:101A8000EFF07FB7E1BB17A500001305E53AEFF0D3
:101A90009FB621B50357E501C17785073E97835768
:101AA000A101FD14133717003207E58FD98F231DCD
:101AB000F100231AD100835605020357250221465F
:101AC000231BD100231CE100035745028566FD1648
:101AD000758FFD76F58FD98F4C0817A5000013057B
:101AE0006536231DF100EFF03F9B21BD17A50000D7
:101AF0001305C535EFF03FB089BD5C4813F7E7FF2C
:101B000058C8858B89CFA6864A86C9450A85EFF0D5
:101B10000FEF8357040099E70A85EFF0DFAD8504E6
:101B200061049DBD231AF1008357240093054400EE
:101B300041462808231BF100EF70C00951464C08AC
:101B40000A85EFF07F95E1BFEF022F9F8547339520
:101B5000A7009747FF1F938767299C47411181453D
:101B60005D8D9747FF1F23A7A7289377057085E30F
:101B700093576500858BA1CBC167938707887D8DBF
:101B800005EDEF606FD19305803EB305B5021745B3
:101B9000FF1F1305A5362EC6EF50A03BB24519C155
:101BA0006349B50085C51745FF1F13052535EF505F
:101BB000C04441016F00AF9AEF600FCE2A84EF60FE
:101BC000AFCEE360A4FCEF602FCE75BF0145EFF010
:101BD000BFBFC5B7EF026F967971AA860144174956
:101BE000FF1F1309A92036C6EF60CFB9B246635C68
:101BF000A4028327490B93143400BE9483D70400B6
:101C00006396D70285C617A6000013062626E5456B
:101C10004808EFF0CFDE4808EFF0FF9D21468145F0
:101C20002685EF008F9445616F006F93050465BFB3
:101C300019C223200600814701C59306D00389E518
:101C40003E8582808505050583870500030705001D
:101C500099CF6394E700E397D7FE8147D5B7930602
:101C6000D0038547E30ED7FC93371700D1BF930706
:101C7000F002E316F7FE854761D6050508C2C9B72D
:101C800099C123A0050081470DC11308D003130695
:101C9000F0023307F5008306070081CA6387060157
:101CA0006397C60099C1050798C13E858280850764
:101CB000CDB731C9EF02EF8541112E8A6C002A8918
:101CC000368BB28A97A400009384040EEFF05FFB7A
:101CD0002A8C0144A689B14B88406286CA85EF7080
:101CE000E01801ED0E044E945C403245DA865686CB
:101CF000D285829741016F004F850504A104E31D41
:101D000074FD6155C5BF7D55828099E5615582801E
:101D1000615505616F000F84EF028F802E8A2A843F
:101D200001118145B28452854146BA893689EFF066
:101D30006F8793150501C1811376F50FA181228567
:101D4000EF507FB12A8469D552854C08EFF05FF3DC
:101D5000524A2A8BE30E0AFA2A8697A50000938539
:101D6000E50F5285EF708010AA8A0DED7D5AEF6065
:101D70006FA563C5AA0099E8014561BF5C4413974C
:101D80001A00850ABA9723904701D5B74C442EC64E
:101D9000EF604FA3B245131615004E850299E34D2F
:101DA000A0FC85BF5A8697A500009385A50B528598
:101DB000EF70C00B0DE1032A0401EF60AFA1131611
:101DC000150081455285EFF05EFADDD40C482EC631
:101DD000EF604FA0C1B75A8697A500009385C5084C
:101DE0005285EF70A00841E11C44A5CF81ECD4439B
:101DF000370700E0758F9447D8C33707001F758FEA
:101E000098C701BFA1463008CE854A85EFE0DF962E
:101E1000E31105F01844835781017D762312F70002
:101E20008357A1019396470183576700D182F18FB1
:101E3000D58FF2467D767D16F182858AB206F18FC6
:101E4000D58F2313F7008347E1018356C101230592
:101E5000F7008347B7002314D700FD8BA305F700D5
:101E60004DBD7D557DB55A8697A50000938545F3F8
:101E70005285EF60B07FE31D05E81C4CE38A07E85C
:101E80009C43E38707E8CE864A86A685228582970B
:101E900049B5EFF29EEA3687B2862E86AA850545B9
:101EA000EFF0BFE66FF0BEEBEFF23EE93687B286A9
:101EB0002E86AA850145EFF05FE56FF05EEAEFF24E
:101EC0003EE6411199C123A005009747FF1F938764
:101ED000A704804381441DC82E89AA8931141DC4DA
:101EE0000C4070004E85EFF0BFD419CD81E8A2847C
:101EF000630C0900B2472320F90039A08C40084048
:101F00000146EFF0FFD265F5404869F826854101AA
:101F10006FF05EE4184111CBEFF23EE2AE873E85F2
:101F2000B285368602976FF09EE335558280EFF2D8
:101F3000DEE08357C50013D70501C205B387E7026A
:101F40001841C1814849BA95BE95EFF0BFFC6FF0CA
:101F50001EE1584111CBEFF25EDEAE873E85B285C1
:101F6000368602976FF0BEDF35558280184509CB63
:101F7000EFF2BEDCAE873E85B28502976FF03EDEA3
:101F8000355582805C4599C7EFF23EDB2E858297FE
:101F90006FF0FEDC35558280EFF29ED88329050074
:101FA000035AC5002A844849AE848145EFF09FFD5D
:101FB0002A890DE193D50401B38545030356C40076
:101FC0004848CE95EFF09FFA2A8909E548488545AB
:101FD000EFF05FFB4A856FF0FED7EFF27ED42A89DF
:101FE0000441035BC500484979712E848145B28A5A
:101FF000368AEFF03FF941E193590401B38969034F
:10200000420441802694A29903440901330480408C
:102010003374440111CC03254901A2865686CE852E
:10202000EFF03FF3AA8431E1330A8A40A299A29AE1
:102030008144630C0A025286D685080803244901AC
:10204000EF605039834609011C089305F00F338671
:1020500046413385470136C6EFF03ED1B2461008FF
:10206000CE852285EFF0FFEEAA8403254901854540
:10207000EFF05FF1268545616FF0DECDEFF2FECB2C
:102080002E864C41A1462A84EFF03FF5AA840345F1
:102090000401A145EFE07F985C403385A74048C02C
:1020A00026856FF0DECB814797A600009386C6CCCD
:1020B0006393C70082803387F500034707008507D5
:1020C000398D135745003697034707001205398DA0
:1020D0001375F50F13574500369703470700120590
:1020E000398D1375F50FE9B7EFF23EC52A84AA853D
:1020F0001D461305F00FEFF01FFB83477400338577
:10210000A7403335A0006FF09EC5EFF21EC341110A
:10211000A1463000EFF0BFE109ED03578100C16730
:10212000FD1705456317F7002800EFF0FFFB333577
:10213000A00041016FF0BEC2EFF29EBEAE848C41A2
:102140004111A1462A8903440501EFF05FDEAA8907
:1021500039E9A1452285EFE05F8C9C400357C90017
:102160002A8AAA97939607019CC0C182098F639C13
:10217000E602C16513D70701B385B74011E7835560
:10218000E900FD15C205BE958CC0A1460A864A85A8
:10219000EFF0FFD9AA8901E90A85EFF0FFF401C940
:1021A000832749009CC04E8541016FF0BEBA03579A
:1021B000C9008357210080403307474163DBE700B4
:1021C00033FA470363170A004177798C3E9480C045
:1021D000D9BF03450901A145417AEFE01F84098C6D
:1021E000AA8A80C0337A4401417B63648A008149B2
:1021F0005DBFA1463000A2854A85EFF05FD3AA8972
:102200005DF12800EFF05FEE11E98357A10003575D
:10221000C100337A6A0180C0BA973E9A33045441B0
:10222000E9B7EFF29EB12A84AA851D461305F00F87
:10223000EFF07FE7A303A4006FF07EB2EFF27EAD74
:102240002A84034505015D71A145EFE00FFD5C4067
:102250002A8B0355E4004179B3F727016C003EC691
:10226000EFE00FFD8355C400B247A1463008BE958C
:10227000B385654122852EC8EFF07FCBAA84634BDE
:1022800005002808EFF05FE611C9B2452285EFF09E
:10229000BFD0AA84268561616FF03EABC247035769
:1022A000A101417C338B6741B3F72701BA973EC840
:1022B00010100C082285C24BEFF01FE8AA8479F9B0
:1022C0000810EFF07FE22DE95C403ECA30104C0868
:1022D00022855249EFF05FE6AA844DFD0357810243
:1022E000835701026316F7002810EFF0FFDF09C5DE
:1022F0005840D247E31CF7FC63902B0583574102FB
:1023000085CF83572102B3FA8B010810BE9A1C4473
:102310002311F102EFF0FFF083490401035A410257
:10232000B309304193F90902631B0A000C1022859E
:10233000EFF0DFD4AA8439FDE31C7BF7B9B74E89EF
:1023400063733A015289CA861018D6852285EFF048
:102350001FBEAA8421F1630909000C44CA86101823
:102360002285EFF09FC7AA8403450401CA85EFE0E8
:10237000CFEA1C443E9508C4E39E04F0330A2A4188
:10238000CA9A5DB7EFF2DE99411191E5FD542685B9
:1023900041016FF03E9CC44983D725014CC904C15B
:1023A0002316F50003C705012A842317E50003C59A
:1023B000150193160701130700022308A400C18228
:1023C000E366A7FCE1D7B3E4F402E9F08547E3FF55
:1023D000D7FAA145EFE06FE4AA89014A0149835782
:1023E000C400931509012285BE95B38535412EC2DF
:1023F000EFF0BFD119ED0355E4004C00050AEFE002
:102400002FE39245420A2285135A0A01EFF0FFCFCB
:1024100009E905098357E400420913590901E360FA
:10242000F9FC8357E40063944701D1548DB763945A
:1024300027039245A1463000B38535412285EFF050
:102440001FAF35E12800EFF03FCA11C50355E40086
:102450004C00EFE0EFDD9247C17A3387374158C037
:102460004177F98F1CC44C401C4463EEF500A14633
:1024700030002285EFF0BFAB1DE52800EFF0DFC68E
:10248000032A44001DC15C400355E4004179B3F7C1
:1024900027014C003EC2EFE0AFD992452285EFF014
:1024A000DFC6635C0502AA84DDB512450359A100AD
:1024B000035BC10033F5AA002A9903450401DA85BC
:1024C000EFE0AFD54A9508C46314450163130B04CC
:1024D000330A3A412322440179B709C58547A30845
:1024E000F40075B54C402285EFF01FAB4DFD484020
:1024F0008357C40086093375A9003E9533053541DD
:1025000048C03375250108C42285EFF03FD379D543
:1025100059BF4D5549BF83471501C9CFEFF26EFF33
:102520002A840345050141112E8AA145BA893689BD
:10253000328BEFE08FCE8357C4000605898F7D551F
:1025400063E727075C4081443EC230004C0022858F
:10255000924AEFF07FBE21ED835B810063994B01CE
:102560002800EFF07FB801E58504C204C18058401F
:102570009247630BF702E3FA99FC8356C100615559
:102580009DC663E63403C175B3FABA006373D9001C
:10259000CA868355A1005A862285D695EFF03F99C9
:1025A00019E50355C10021A06155E3884BFD4101A8
:1025B0006FF0AEF949558280EFF22EF80147EFF047
:1025C0009FF56FF0CEF9EFF24EF73284B2862E8689
:1025D000835545000841EFF03FFE635385002A8490
:1025E00022856FF0CEF7EFF24EF283471501397175
:1025F000C954BDC7034B05012EC62A84A1455A857F
:102600003689328AEFE06FC10D473307E502835701
:10261000C400AA8DFD54998F63E427056304090063
:1026200063000A045C403ECA30084C082285524DC3
:10263000EFF09FB0AA8945ED835781013247639738
:10264000E7002808EFF05FAA630605105840D2475C
:10265000E31CF7FC8144631B090019A0814499E73E
:10266000268521616FF02EEEE35CA0FE5A85CA85B7
:10267000EFE0AFBA014B11C5330BB501420B135B51
:102680000B01014D7D5CC17B930C44008357E4003A
:102690006380A70D1C4444403307FB0063EBE40454
:1026A00032472311F1020810FD572310E1022312D3
:1026B00021032303F102EFF0DFB6630909000C44A4
:1026C000CA8652862285EFF05F91AA8903450401EC
:1026D000CA85EFE08FB41C443E9508C46399090095
:1026E0000C102285EFF09F99AA89CA8435D9CE842F
:1026F00085BF03450401A145EFE02FB2B387A400D5
:102700002311F1028357C400B3F474012310810331
:10271000BE94898C44C0081023120102EFF07FB0F0
:102720000C102285EFF09F95AA840355E400E685FE
:10273000EFE00FB05C40B3F777011CC4E39204F202
:102740002285EFF0BFAFAA84E31C05F0050D3DBF65
:10275000C15439B78357C101E30209F0E39827F167
:10276000C177034C0401B377FD00035DA101330C75
:102770008041137C0C023E9DD28ACA8CE28B63F3AB
:102780008C01E68BDE861010EA852285EFF02FFAA9
:10279000AA84E31B05EC5E860C105685EF60204191
:1027A000AA84E31505ECB38C7C415E9DDE9AE39729
:1027B0000CFC7DB5EFF26ED881460146EFF0BFE22A
:1027C0006FF0EED9638C050EEFF2AED45D71054D5E
:1027D00019C213BD160003590502B68B328B0509C9
:1027E0004209135909012E8A2A84CA89216C930A45
:1027F0008500E15C9304F9FFC204C180638F840506
:102800009306A0045000A6855685EFF0FFDA6357C3
:10281000050063139501A6892689E9BF9C083E95AA
:10282000230A05FA4C005285EFF0AEDE75F563041D
:102830000D0883570402639597089387F4FF2310CC
:10284000F402894613060402A1655685EFF0BFD94C
:102850006358050661616FF04ECF0145E31C0DFE24
:102860000549B1675D55E387F9FE9165CE959304FF
:102870008400C205DE865A86C1812685EFF0BFD668
:10288000630D09005285EF60405DAA865286CE85B1
:102890002685EFF05FD5E34F05FA8357040263FF07
:1028A000370323103403894613060402A1652685E5
:1028B000EFF07FD325A0A689014965B77D558280B9
:1028C000A6855685EFF01FEFE34605F89165FD15E7
:1028D000CA95C205C1815685EFF0DFEDE35CA0F635
:1028E00001458DBFEFF2EEC203540502916A1D71DE
:1028F000050442042A89AE894180A16B130A850030
:10290000FD1A130B05029304F4FFC204C180639DFA
:102910007405916B2164130A8900850B170C000064
:10292000130CACCA8357090293041400C204C1807B
:1029300085076383F40E5E949306A0045008A68571
:1029400052854204EFF05FC74180AA8A854613068C
:102950007100A2855285EFF03FC62A8B634750076E
:102960006347A00626847DBF56949306A0045008B2
:10297000A68552854204EFF03FC441802A8C8546EB
:1029800013067100A2855285EFF01FC3634C8003CC
:10299000E351A0F883570902E39D97F69387F4FF6C
:1029A0002310F90289465A86A1655285EFF0BFC30C
:1029B000A6855285EFF01FE0A2855285EFF09FDFDC
:1029C000268491B7E358A0FCA9B7634BA000A68565
:1029D0005285EFF03FDEA2855285EFF0BFDD59B79B
:1029E0009C10BE9A238A0AFA639109022C004808B7
:1029F000EFF0EFCC25D91C45224552C623188100A3
:102A000074006286DA858297B1BF0146CE85480898
:102A1000EFF00FA261FDB9B7014525616FF0EEB28D
:102A2000EFF2AEB19737FF1F9387074F8043814482
:102A300009C42A893114814401E426856FF02EB23D
:102A4000631809005C4481EF404865D83114EDB744
:102A500008400146CA85EFF0AF9D6DF5F5B7829746
:102A6000E5F4AA84D5B7EFF24EAD9737FF1F9387F1
:102A7000274B8043AA8409EC2685EFF07FFAAA84CD
:102A80000144EF502FD0636CA40026856FF02EAD6B
:102A90005C402285A6859C4382970040E9BF0504DF
:102AA0001374F40FF9BFEFF24EA90145EFF0BFFB2D
:102AB0006FF0EEAA9737FF1F9387874623A0070082
:102AC00023A207008280EFF24EA79737FF1F93875C
:102AD000A74423A0070023A20700EFF0BFFD6FF07B
:102AE0000EA8EFF28EA54111130985002A84EF503C
:102AF000CFE5AA854A85EFF0FF88AA8419ED8946BB
:102B00001306E100A1654A85EFF01FABE17763444E
:102B100005008357E1002310F402268541016FF080
:102B20000EA49737FF1F9387A73F90430147B286B4
:102B300091EE05E3DC4310C11737FF1F2322A73EA8
:102B400085EF9737FF1F23AFA73C828036879442DB
:102B5000C5B7144385E2DC432320050091EB97378A
:102B6000FF1F23A1A73C9737FF1F23ABA73A828003
:102B700088C3C1BF14C108C38280EFF20E9C173412
:102B8000FF1F130424352285EFF0BFF5AA8405E565
:102B9000179900001309492722859737FF1F23AD96
:102BA0002733EFF01FF89737FF1F23A727339737F7
:102BB000FF1F23AB873626856FF06E9A9737FF1F6E
:102BC00083C7C736795599EFEFF22E97EFF0BFEF35
:102BD000EFF0BFFA11E585471737FF1F2308F734D9
:102BE0006FF0EE978280EFF24E959737FF1F938735
:102BF000A73280432A89BE8419C0311415E0D84019
